:020000040800F2
:100000000000022045B800083DB800083DB80008CF
:100010003DB800083DB800083DB8000800000000E9
:100020000000000000000000000000003DB80008D3
:100030003DB80008000000003DB8000829B80008DD
:100040003DB800083DB800083DB800083DB80008BC
:100050003DB800083DB800083DB800083DB80008AC
:100060003DB800083DB800083DB80008E52100088B
:100070003DB800083DB800083DB800083DB800088C
:100080003DB800083DB80008293100083DB8000817
:100090003DB800083DB800083DB80008153100081B
:1000A0003DB800083DB800083DB800083DB800085C
:1000B000BD300008652F00083DB80008292600085B
:1000C000BD2300083DB800083DB800083DB8000851
:1000D000DD300008452E00083DB800083DB8000896
:1000E0003DB800083DB800083DB800083DB800081C
:1000F0003DB800083DB800083DB800080D200008D4
:100100003DB800083DB800083DB800083DB80008FB
:100110003DB800083DB800083DB800083DB80008EB
:100120003DB800083DB800083DB800083DB80008DB
:100130003DB8000800000000000000003DB80008C5
:100140003DB800083DB800083DB800083DB80008BB
:100150003DB800083DB800083DB800083DB80008AB
:100160003DB800083DB800083DB800083DB800089B
:100170003DB800083DB800083DB800080000000088
:10018000000000003DB80008000000000000000072
:100190003DB8000800000000000000003DB8000865
:1001A0000000000000000000000000003DB8000852
:1001B0003DB800083DB800083DB800083DB800084B
:0401C0003DB800083E
:10020000344A0368904210B455D0B0F1804F29D0E1
:10021000A2F57C44A04237D004F5806C604533D011
:100220000CF5806290422FD002F57844A0422BD08A
:1002300004F5705C604513D00CF5806290420FD0DD
:1002400002F58064A0420BD0A4F5983C604507D02D
:100250000CF58062904203D002F58064A04209D17F
:10026000CA6804E04C68CA6823F07003234323F48F
:100270004073134303608A68C26209688162012483
:1002800044615DF8044B70474C68134A23F07003D7
:100290002343CC6823F44073234303608C68C46217
:1002A0000B6883629042EAD10969016301244461C9
:1002B0005DF8044B70474C68CA6823F07003234311
:1002C00023F44074144304608A68C2620B6883623A
:1002D000EAE700BF000001400004014030B4494A91
:1002E0001368D96821F00100D8601C6A41F2111529
:1002F0002C420AD1186A40F2444C10EA0C0F04D187
:10030000196821F001041C6013683F4D1120D06072
:10031000AB42196867D0B3F1804F29D0A5F57C4C6A
:1003200063454DD00CF58064A34249D004F5806547
:10033000AB4245D005F57840834241D000F5705C72
:10034000634513D00CF58064A3420FD004F580659B
:10035000AB420BD0A5F59830834207D000F5806CF6
:10036000634503D00CF58064A34209D1156904E00C
:100370009068156921F07001014321F4407129430F
:100380001960D5685468DD629C62106895681469CC
:1003900001215961036823F070032B4323F4407556
:1003A000254305601468D0685268E062A26261610A
:1003B000E3680B43E36025680D43256030BC70475C
:1003C00090681469114D21F07001014321F44070CF
:1003D00020431860D4685168DC62AB429962D4D182
:1003E00051691963D1E79568106921F070012943BB
:1003F00021F4407404431C60D568DD625068986243
:10040000EEE700BF40000120000001400004014071
:100410002DE9F04FDFF8D8C1DFF8D8E16E4FDFF8F3
:10042000D89183B0002603E00136102E00F0B3808F
:1004300001230A68B3401A409342F5D14D6825F074
:100440001004022C15D1F50800EB850806F007040E
:10045000D8F82050A4004FF00F0B0BFA04FA25EA4D
:100460000A0B0D6905FA04F444EA0B05C8F820509C
:100470004D68D0F800A04FEA46084FF0030B0BFA86
:1004800008F405F00305E44305FA08FB04EA0A054D
:100490004BEA050505604D6825F0100A0AF1FF35A5
:1004A000012D12D8856804EA050BCD6805FA08FA13
:1004B0004AEA0B0585604D68D0F804B0C5F3001515
:1004C000B5402BEA03032B434360C5688B682C407F
:1004D00003FA08F52543C5604C68E300A4D5002362
:1004E0000193DCF8445045F48044CCF84440DCF8F7
:1004F000443026F0030808F1804A03F480450AF5E9
:100500009C3B019506F00304019BDBF80880A500E5
:100510000F23AB40704528EA030A18D048453DD068
:100520002E4B984240D02E4B984243D02D4B9842B0
:1005300046D02D4B984249D02C4B98420CBF4FF0DF
:1005400006084FF0080808FA05F54AEA050ACBF84C
:1005500008A04D683B68D443ED0354BF23401343C8
:100560003B604D687B68AD0354BF234013437B6001
:100570004D68BB68ED0254BF23401343BB604D6818
:10058000FB68AD0206F1010654BF23401343102E51
:10059000FB607FF44DAF03B0BDE8F08F012404FA97
:1005A00005F84AEA080AD2E7022404FA05F54AEAFD
:1005B000050ACCE7032404FA05F84AEA080AC6E764
:1005C000042404FA05F54AEA050AC0E7052404FAFA
:1005D00005F84AEA080ABAE7003C01400008024070
:1005E000000C0240001002400014024000180240BB
:1005F00000380240000002400004024070B4174B73
:10060000DC68C4F30223C3F10705042D03F10406DB
:1006100028BF0425062E19D9033B4FF0FF369E4014
:1006200022EA06044FF0FF32AA4021EA020101FA51
:1006300003F525432C01431CE6B20AD000F16040CB
:1006400000F5614C8CF8006370BC704700242346B1
:10065000E8E7024B83F8236070BC704700ED00E0D0
:100660002DE9F04F8BB0C64CC64800250395236B8F
:1006700043F002012163226B02F002060396039B02
:100680000295276B47F002032363216B01F00202FE
:100690000292029B0195266C46F400172764236C96
:1006A00003F400110191019B0095226B42F40016A6
:1006B0002663276B079507F400134FF012084FF0DD
:1006C000010A00934FF04009042605A9CDE90598D9
:1006D000009AAC4FCDE908A6FFF79AFECDE908A62F
:1006E0008020DFF8C0E20590CDE906852946D04696
:1006F000A4464FF00F090131102900F09380059BAB
:1007000008FA01F003409842F5D1069A22F010064B
:10071000022E14D1CD08AC0004F1804A0AF5013450
:1007200001F0070B5D46266AAD0009FA05FA26EAD4
:100730000A0B099E06FA05F545EA0B0626624C00EF
:1007400003253E68A54002F00302ED432E40A2407F
:1007500032433A60069A22F0100A0AF1FF36012E5F
:1007600010D8BE6805EA060B089EA64046EA0B06AE
:10077000BE607E68C2F300128A4026EA0000104381
:100780007860069AFE6807983540A0402843F860D4
:10079000D000B0D500240494DCF8445045F48046E1
:1007A000CCF84460DCF8440021F0030A0AF1804BE5
:1007B00000F480450BF59C34049501F00306049D7C
:1007C000A568B00009FA00FA25EA0A0608FA00F559
:1007D0003543A560DEF80040D843D20354BF04403F
:1007E0001C43CEF80040069EDEF80420B60354BF3A
:1007F00002401A43CEF80420069CDEF80860E502A9
:1008000054BF06401E43CEF80860DEF80C50A40228
:1008100001F1010154BF05401D431029CEF80C50D1
:100820007FF46DAF584B5949D3F89C40D9630225EA
:1008300083F871500F684FF0007227F001064020D6
:100840004FF480671A645864DF64032500274FF46F
:1008500000024FF400105D669A66D86689460E6005
:100860009F64C3E91477C3E916771F6683F8707035
:1008700005E0D3F89C20171B052F00F29281D9F8D0
:100880000060F207F5D4D3E91024D3E9120522431E
:100890000243D3E914702A43D3E916643A4302436E
:1008A0000D683B4F186E324322432F40042842EA22
:1008B000070200F07D81DD6B0A60196E6A69042908
:1008C00022F0070040EA010000F077815FFA85FB23
:1008D000304F6861ABF1100CA7FB0C210E092E48BC
:1008E00025F47F75845DC3F8984025F00302032E3C
:1008F00088BF04323F27A74000210126C3F8942077
:100900009760C3F8901083F871602449D3F89C5025
:10091000234F022483F829410A68C3F8F41022F017
:1009200001044FF000760C60002207F16400C3F868
:10093000D470C3F8F8604FF480674FF40036C3F802
:10094000FC20C3F80021C3F80821C3F80C21C3F828
:100950001021C3F8182183F82821C3F80471032259
:10096000C3F814614FF400074FF4001658678A4625
:10097000C3F81C21C3F82071C3F824611AE000BF3A
:10098000003802400004024040000120B8600240EC
:100990003F8010F0ABAAAAAA00BD00081060024078
:1009A0007C000120003C0140D3F89C20571B052F00
:1009B00000F2F080DAF80020D607F5D4D3E93E271C
:1009C000D3F80051D3F80441D3F808613A432A43DD
:1009D000D3F80C71AD4D22433243D3F81061D3F8F4
:1009E00014413A4332430F68D3F8186122433D4023
:1009F000042E42EA050205D1D3F82041D3F8247130
:100A00003C432243D3F8F4600A60D3F818117269AA
:100A1000042922F0070444EA010400F0E3805FFAAD
:100A200086F89B4F7461A8F11004A7FB04252909DF
:100A3000984F26F47F767C5CC3F8504126F0030281
:100A4000032988BF04323F21A14000250127C3F8B4
:100A50004C219160C3F8485183F829718E498F4D1C
:100A6000CA68C3F82C01C2F30227C7F107000428A3
:100A700007F1040628BF0420062EC3F8D85040F220
:100A80008680FD1E4FF0FF33AB40D94301F00104D7
:100A90004FF0FF328240D74307F00200A8402043C6
:100AA00006017F4C7C4D5FFA86FB4FF4004384F8CF
:100AB0002FB36360E968C1F30222C2F10707042F74
:100AC00028BF04274FF0FF36101D06FA07F406284A
:100AD0006FEA04058CBF033A002205F0020393403D
:100AE00019016F4A6C4FC8B24FF4006482F80B03CF
:100AF0001460FD68C5F30221C1F10703042B01F165
:100B0000040228BF0423062A3ED9CF1E06FA07F0A6
:100B1000C44304F001064FF0FF3505FA03F1CB435F
:100B200003F00202BA40324316015D4F5A48F1B257
:100B3000012487F820137C60C368C3F30222C2F14A
:100B40000700042802F1040628BF0420062E0746E9
:100B500017D9D41EA540E94301F002054FF0FF3339
:100B6000BB40DA4302F00200A04028434C4F06018C
:100B7000F5B24FF0004487F81F533C600BB0BDE85E
:100B8000F08F00252C46E9E700263746C3E700240E
:100B900025467DE720260324C3F8486183F82941D0
:100BA0005CE720260320C3F8906083F87100ACE670
:100BB000D3E91A64264332437DE65F6E5E6D3843A7
:100BC0008EBB012F46D002D3022F7FF47FAE9C6EE6
:100BD000E7017FF57BAE40200125C3F8900083F844
:100BE000715092E6D3F81C71D3F80C513C438DB987
:100BF000012F43D002D3022F7FF411AFD3F820216D
:100C0000D1017FF50CAF40260124C3F8486183F879
:100C1000294123E7B5F5005F22D0022FF3D9032F36
:100C20007FF4FDAEEAE7B6F5005F05D0022FD2D91A
:100C3000032F7FF44BAECAE7032F3FF647AE01A464
:100C400054F827F0D70B0008CF0B0008D70B00088B
:100C5000550C00089A6EB2F1C07F7FF437AEBAE748
:100C6000032F3FF6DCAE01A555F827F0070C00086E
:100C7000FD0B0008070C00087D0C0008D3F82011BC
:100C8000B1F1C07F7FF4CBAEBDE700BF3F8010F075
:100C9000ABAAAAAA00BD000800ED00E034010120C3
:100CA00000E100E070B41B4DD5F8A0406369DE435D
:100CB0001FFA86FC1CEA000311D0666916F48063F3
:100CC00010D1D5F89C60B61AB142EFD22022C5F8F7
:100CD000D03085F8DC3085F8DD20032000E01846B0
:100CE00070BC7047206840F400712160D5F8A060A6
:100CF0006FF480647461002304214FF0200CC5F868
:100D0000E0100120C5F8D03085F8DC3085F8DDC072
:100D100070BC704740000120F0B4134ED6F8A050CC
:100D2000070C012F0CBF6C69AC69E4431FFA84FC0B
:100D30001CEA000F0CBF4FF0010C4FF0000C8C456B
:100D400002D00020F0BC7047D6F89C40E41AA242C2
:100D5000E7D200232022C6F8D03086F8DC3086F8AF
:100D6000DD200320EEE700BF4000012070B4394DC4
:100D7000D5F8CC30D5F8A040042B08D0012B06D0F4
:100D800013F5803F03D0D5F8D060122E05D123682B
:100D900043F480762660D5F8A0406369DE070ED460
:100DA000D5F89C60B31A9942F7D200212022C5F8E9
:100DB000D01085F8DC1085F8DD20032046E0D5F85A
:100DC000B060B6F5804F17D1C0B220616369DE43D1
:100DD00016F0020C3CD0606910F480631BD1D5F88A
:100DE0009C60B01A8142F1D22022C5F8D03085F83B
:100DF000DC3085F8DD2023E0F023236166693307CA
:100E0000E2D4636913F4806305D1D5F89C60B61A07
:100E1000B142F3D2E8E7216841F400702060D5F8D0
:100E2000A00000236FF4806404264FF0200C44617E
:100E3000C5F8E06085F8DC30C5F8D03085F8DDC055
:100E4000D5F8E050042D0CBF0120032070BC704782
:100E50006046FBE74000012010B41A4CD4F8A01003
:100E600008E04A6912F0100C0CD1D4F89C301A1A20
:100E7000012A18D84B6913F04003F2D000205DF826
:100E8000044B70476FF0100048614FF0200CC4F81D
:100E9000E0300120C4F8D03084F8DC3084F8DDC0C4
:100EA0005DF8044B7047D4F8E00084F8DCC040F0F3
:100EB00020012023C4F8E010032084F8DD305DF821
:100EC000044B70474000012030B41A4CD4F8A010F5
:100ED00008E04A6912F480650BD1D4F89C301A1AE4
:100EE000012A16D84B6913F08003F2D0002030BCE1
:100EF00070476FF48060486104252022C4F8E050F8
:100F00000120C4F8D03084F8DC3084F8DD2030BC17
:100F10007047D4F8E00084F8DC5040F020034FF034
:100F2000200CC4F8E0300320C4F8D05084F8DDC0B1
:100F300030BC704740000120002941D0013930B455
:100F4000421E10FA81F54BF6AD24002012F8013F45
:100F500080EA032001B28BB20029ACBF5B0084EAB7
:100F6000430398B2030454BF400084EA400083B2B4
:100F7000190454BF5B0084EA430399B20B0454BFC5
:100F8000490084EA410188B2010454BF400084EA68
:100F9000400081B20B0454BF490084EA41018BB286
:100FA000190454BF5B0084EA430398B203044CBFA6
:100FB00084EA40004000954280B2C7D130BC7047FF
:100FC0000846704730B40E4C0D2304F10E054FF067
:100FD000000C034003F00F0293B22AB100225A40E2
:100FE0005B08FCD102F0010242EA4C01A5421FFA63
:100FF00081FC02D034F8023FEBE7604630BC70471A
:1010000008BD000830B41B491B4A4B6992F859517E
:1010100092F8584183F0400C4CF48003A5428B6158
:1010200002D092F884510DB930BC704792F85A4101
:10103000D2F8541141F8240092F85A3192F858012C
:1010400092F859110133DCB2A04205F1FF3582F864
:101050005A415FFA85FC9CBF002482F85A4102EB9A
:101060008C034C1C82F884C182F85941D3F85C018E
:1010700030BC70470000024040000120034AD2F813
:1010800088310133C2F88831704700BF4000012029
:101090000120704700207047024B19780170012031
:1010A000704700BF00000020024B93F88C110170C4
:1010B0000120704740000120044B93F88D110A1C59
:1010C00018BF012202700120704700BF40000120BC
:1010D000224BB3F890110A0A42EA01210180B3F8C9
:1010E00092110A0A42EA01214180B3F894110A0AD6
:1010F00042EA01218180B3F896110A0A42EA0121ED
:10110000C180B3F898110A0A42EA01210181B3F8BB
:101110009A110A0A42EA01214181B3F89C110A0A94
:1011200042EA01218181B3F89E110A0A42EA0121B3
:10113000C181B3F8A0110A0A42EA01210182B3F881
:10114000A2110A0A42EA01214182B3F8A421130A3A
:1011500043EA022181821620704700BF400001202F
:101160002F4B5978002957D0F0B42E4A32F8024B51
:101170000123250A45EA04264F1E9942068007F0FE
:10118000030C44D94FFA8CF4ECB1012C10D0022C92
:1011900006D032F8025B2B0A43EA0526468002237A
:1011A00032F8027B3C0A44EA072520F81350013349
:1011B00032F8026B370A47EA062C20F813C00133D5
:1011C000DCB2A14223D915465C1C35F8027B3E0AED
:1011D00046EA072720F8137057883E0A46EA072791
:1011E00020F814706E889C1C350A45EA062720F802
:1011F0001470D588DE1C04332C0A5FFA83FC44EAA1
:101200000527614502F1080220F81670DBD8480076
:1012100000F0FE00F0BC7047480000F0FE00704790
:1012200000000020E8010120F0B44B4B04460D46BD
:10123000164693E8070084B00DF1040CACE80300F7
:1012400001AFACF800200DF10E00002130F8022DA6
:10125000490014EA020389B206D000225A405B0812
:10126000FCD102F0010211438742EFD179BBC4F3F4
:101270004032C4F3C02C4CEA4203C4F3802747EA4F
:101280004300C4F3402242EA4007C4F3C01C4CEAC6
:101290004703C4F3801040EA4302C4F3401747EA0F
:1012A0004200C4F3001C4CEA4003C4F3C00242EA0B
:1012B0004307C4F3800040EA470CC4F3400444EA07
:1012C0004C03012031802B8004B0F0BC70470F2903
:1012D0003BD9A1F110070120308017F0FF0605D09F
:1012E000C6F1100C00FA0CF14C40A4B2C4F3403229
:1012F000C4F3C02343EA4207C4F3802040EA470610
:10130000C4F3402141EA460CC4F3C01242EA4C0344
:10131000C4F3801747EA4300C4F3401646EA40018D
:10132000C4F3001242EA410CC4F3C003C4F38000CA
:1013300043EA4C0740EA4706C4F3400444EA460146
:101340000120298004B0F0BC70474FF6FF740020E4
:10135000348004B0F0BC704718BD0008F0B4284ECB
:101360000025A6F1080736F8024D04406D00E4B2EE
:10137000ADB2A3B234B100245C405B08FCD104F0F0
:1013800001042543B742EED19DB9C0F3401CC0F320
:10139000C00343EA4C04C0F3800646EA4407C0F3A6
:1013A000400040EA470C15800120A1F800C0F0BCC5
:1013B0007047072D1ED9A5F108060127178016F0E2
:1013C000FF0205D0C2F1080C07FA0CF5684080B2A4
:1013D000C0F3C004C0F34013C0F3800744EA4306DF
:1013E00047EA4602C0F3400040EA42050D80012072
:1013F000F0BC70474FF6FF701080F0BC00207047C3
:101400002CBD000830B40F4C40F2D56304F11E052A
:101410004FF0000C0340C3F30A0293B22AB100223A
:101420005A405B08FCD102F0010242EA4C01A5429D
:101430001FFA81FC02D034F8023FEBE7604630BC73
:10144000704700BF2CBD00081E4A92F8E83103B96E
:1014500070472DE9F0411C4841695C1EE4B281F4FB
:10146000007545F00076122C82F8E841866110D8AC
:10147000164D174E6700EA1996F805C092F84C8091
:10148000C44513D83D44707B95F84D50A84202D80E
:101490003475BDE8F0813169012011F8351004F090
:1014A00031FA0028F4D035733475F2E7B3680020C0
:1014B00013F8381004F026FA0028E3D086F80480E8
:1014C000E0E700BF400001200008024000BD000826
:1014D000000000201D4A92F8E831112B00D9704716
:1014E0002DE9F0410133DCB2194F1A4982F8E84185
:1014F00065007819184E4B6990F84C8096F805C035
:1015000083F4807242F08070C445886112D83D44F3
:10151000777B95F84D50AF4202D83475BDE8F08125
:101520003369012013F8351004F0ECF90028F4D0E9
:101530003573F2E7B168002011F8381004F0E2F9D1
:101540000028E4D086F80480E1E700BF40000120D5
:1015500000BD000800080240000000200020704785
:10156000264B5A78597D01328B1A48BF03339A10A3
:10157000013212F0FF033DD010B4214AB2F8EC4121
:10158000210241EA1424012B04802DD9B2F8EE4146
:10159000210A41EA0424022B448025D0B2F8F0410C
:1015A000210A41EA0424032B84801DD0B2F8F241C1
:1015B000210A41EA0424042BC48015D0B2F8F44176
:1015C000210A41EA0424052B04810DD0B2F8F6412A
:1015D000210A41EA0424062B448105D0B2F8F8110F
:1015E0000A0A42EA012484815B0003F0FE005DF8F0
:1015F000044B7047580000F0FE00704700000020C8
:1016000040000120012070470020704701207047F2
:10161000002070470120704701207047012070476B
:101620002DE9F04F83B00026814CDFF80882DFF807
:1016300008920190B34637464FF40075D4F8FC2168
:10164000D4F800329A42F9D094F88C01D4F8882169
:1016500050B1D4F8041439B1D4F80834D01A14288D
:1016600000D88847C4F80474D4F80C34D4F8FC11BA
:10167000D4F8002201339142C4F80C3400F0CE803B
:10168000D4F80032D9B2043104EB410CBCF8FC218F
:10169000D4F8003290B20FFA80FA0AFB0AF1013353
:1016A0000BEBA13BC4F80032D4F81034D8F818C0C2
:1016B0000133013DC3F30E0209EB4201ADB25644C2
:1016C000C4F81034C8F81810ACF80000002DB5D1DB
:1016D00086FB0667B60B46EA8744670A5846C31777
:1016E000BBEB070863F1000218EB080142EB0205AF
:1016F000002975F1000306DA40F2FF164FF00009E9
:10170000891945EB09054C0A44EAC552002A4FEAFB
:10171000652575F10003C0F286806FF00047002652
:10172000974276EB05034FF001087EDA900840EA15
:101730008570A9104FEA480387425FFA83F876EB79
:10174000010302460D46F1DB5FFA88F84FF000090D
:10175000AC0344EA9245002694034FF08047B0085A
:1017600040EA8776B4424FEAA70775EB0703F6DB3A
:1017700032463B46134356D000200021B208B24601
:1017800036184FEAA70E42EA877CBB464F41B44267
:1017900075EB070309DB1AEB0A0A4BEB0B0210EBA4
:1017A0000A005141A41B65EB0705624673464910C8
:1017B0004FEA3000134366467746DFD100FB09F35A
:1017C000C11708FB013CA0FB0889E14418EB0802A3
:1017D00049EB090512EB080445EB090046016701D6
:1017E000391946EAD46B4BEB000A18EB010249EBBE
:1017F0000A05002A75F1000315DB12F5005345F1C7
:101800000004980B40EA8446FF2E28BFFF26F7B25B
:10181000019901200F7003B0BDE8F08F4FF0FF3A3F
:101820004FF6FF7040E70027F2E74FF000098FE71F
:1018300040000120000000204000002000207047F0
:101840000020704700207047002070474379042B28
:1018500001D001207047D0F80620064B0648074902
:1018600012BA03FB02F3A0FB03239809C1F8140486
:1018700001207047400D0300D34D6210400001204D
:10188000094B0A4AD3F814144FF47A7303FB01F39B
:101890009909A2FB012399090A0202F47F0343EA92
:1018A000016101600420704740000120632D3E0566
:1018B0004379012B01D001207047827922B9054874
:1018C00080F88D21012070470249012081F88D3177
:1018D000704700BF40000120002070471E4A92F868
:1018E0001834032B2ED870B41C491D4D8C69817996
:1018F00082F81814661B00237410B0F8075082F8A1
:101900001934C2F81C34C2F81044B0F809602B0A2C
:10191000300A43EA052540EA062628B20028ACBF73
:1019200080B24FF400401FFA86FC8445A2F820C420
:1019300088BFA2F820040129A2F8220404D00120C3
:1019400070BC70470020704782F81914C2F81C441C
:10195000084670BC704700BF400001200000002016
:1019600040000020034B1322197D017042700220B9
:10197000704700BF0000002001207047054B06495A
:10198000DB69064A591A8B1002FB03F3037001202E
:10199000704700BF0000002074BD0008ABAAAAAACF
:1019A0004379012B01D001207047807904289CBF26
:1019B000024A82F824040120704700BF4000012041
:1019C0004379022B01D001207047C2880848094999
:1019D00053BA9AB200FB02F0A1FB0010830C802BDB
:1019E00098BF05494FF0010098BF0B84704700BFB6
:1019F000400D030083DE1B43000000202DE9F84367
:101A0000134B1C8C6201161B4FF000054FF00001B8
:101A100061EB05077B02720243EAD657161947EBC2
:101A200005014FEA8118B30148EA96699E1B69EBEC
:101A3000010780463019074A4FF0000347EB0501C4
:101A400006F060FD40BAA8F800000220BDE8F88367
:101A500000000020400D03004379012B01D001203C
:101A6000704780790A289CBF024A82F82504012029
:101A7000704700BF40000120034B0B2293F8251450
:101A800001704270022070474000012030B4084BC2
:101A900000211D795C7901701A7B5B7B4570012107
:101AA0008470C1700271437130BC0620704700BF62
:101AB000000000204379022B01D00120704710B4B0
:101AC00083799A08911E06290BD80F4C6178013151
:101AD00003F0FC03B2EB910F6375BCBF03F1FF335E
:101AE0006370C07901308408A21E062A08D806480F
:101AF00090F815C0B4EB9C0F02D8A1004B1E4370A8
:101B000001205DF8044B70470000002010B4074B23
:101B10005A78597D0170531C8C089B108470427058
:101B2000C3705DF8044B0420704700BF0000002024
:101B300010B4074B002493F8241093F82520047068
:101B400001234170C27083705DF8044B042070471C
:101B5000000000204379012B01D0012070478079DB
:101B6000421E072A9CBF024A10700120704700BF26
:101B7000000000204379012B01D0012070478079BB
:101B8000421E632AF9D88305044905483233A1FB74
:101B90000312530983620120704700BF1F85EB5178
:101BA00000000020084B9A6A642101FB02F111F544
:101BB000001304D503F57F1C0CF57F533F339A15B2
:101BC00002700120704700BF000000204379012B04
:101BD00001D00120704780790228FAD8084A0128EC
:101BE00082F82604F5D192F8271421B9054B4FF05D
:101BF00000609861EDE703494FF400628A61E8E70D
:101C00004000012000080240024B93F826140170A6
:101C1000012070474000012000207047024B012046
:101C200083F82804704700BF40000120002070475F
:101C300001207047034BB3F82A144ABA02800220ED
:101C4000704700BF40000120024B93F82F14017031
:101C5000012070474000012001207047BFF34F8FE3
:101C60000549064BCA6802F4E0600343CB60BFF34A
:101C70004F8F00BFFDE700BF00ED00E00400FA0554
:101C800008B5FFF7EBFF00BF08B5024B024A1A6028
:101C9000FFF7E4FF00C00120AD700DB030B4694B18
:101CA0006948D3F88811D3F8382601314FF08064A1
:101CB000C3F888118461D3F83054D3F834048542D2
:101CC00084B048D0D3F83054D3F83444A5423FD040
:101CD000D3F83404C1B2043103EB4105B5F8304404
:101CE000D3F8340401301FFA84FCC3F83404574D90
:101CF000A3F890C6A91CD3F89C40C3F86856C3F853
:101D00007016D3F89C0004E0D3F89C50291A64297B
:101D100045D89468A507F7D5B3F89036D36000206E
:101D20000190D568019591680191019B54684848DC
:101D300044F040035360156845F04001116042696A
:101D400082F0200444F40013836104B030BC704777
:101D50004FF6FF7CCBE793F8941671B33D4DD3F863
:101D60009C00C3F8685603F29264D3F89C50C3F801
:101D7000704691688C0741D4D3F89C40611B64295C
:101D8000F7D9354B08254FF40064402080214FF4EB
:101D900080529D619C61986199619A61FEE72E4B2A
:101DA00008254FF40064402080214FF480529D614B
:101DB0009C61986199619A61FEE703F29265274CF4
:101DC000D3F89C00C3F87056D3F89C50C3F868460B
:101DD000916889072CD4D3F89C10481B6428F7D944
:101DE0001D4B08254FF40064402080214FF48052A1
:101DF0009D619C61986199619A61FEE700234FF4AF
:101E00000040D0600293D568029594680294029BCA
:101E1000516841F040005060136843F04005156080
:101E20000B4A546984F0400141F4800090618CE7D2
:101E30000023D3600393D068039094680394039BBA
:101E4000E6E700BF4000012000040240D006012068
:101E5000000802408CBD0008000002408EBD000852
:101E6000F0B46149614B4A6982F0800040F400049B
:101E70008C61D3F888510135C3F88851B3F8926664
:101E8000D3F81857D3F88841F7001FFA87FCACF550
:101E9000804188B293F8951602B203EB4106002AFE
:101EA000B8BFCCF58042B6F99876B8BF12B2A6F8A2
:101EB0009826D21BD3F81C672A44013101F03F0C4D
:101EC000B24282B083F895C6C3F818275DDAB3F83A
:101ED00022576F1EBAB22126A3F82227A3F8206743
:101EE00042B94349C3F8084440F20124C3F804143A
:101EF000A3F82247D3F8FC51D3F80072EA1BB2F5DD
:101F0000807F3AD0D3F8FC51EFB2043703EB470C93
:101F1000ACF8FC01D3F8FC210132C3F8FC21354EAA
:101F20003548364CC3F868064FF00071B161D3F8FC
:101F30009C10C3F87046D3F89C60D3F8382604E0B0
:101F4000D3F89C00841B642C38D89568A907F7D572
:101F50004AF6AA270023D7600193D66801969068B5
:101F60000190019B546844F040015160156845F0B0
:101F70004007176002B0F0BC70471B48466986F402
:101F8000806141F080648461C9E7D3F824178A42F4
:101F900022DDB3F820777A1E96B240F2012CA3F826
:101FA0002067A3F822C7002EA4D11549C3F808441E
:101FB0002124C3F80414A3F820479BE7114F0825F8
:101FC0004FF40066402380214FF48052BD61BE6112
:101FD000BB61B961BA61FEE7212440F20125A3F893
:101FE0002047A3F8225785E700080240400001205F
:101FF000D51400080004024090BD0008D20601205C
:102000004914000800000240704700BFF0B5704A54
:10201000704BD2F8D440DE6A83B0D4E91673002046
:1020200001903D68082202FA03F1294203D0216899
:10203000086840077ED4684A9A40154204D0216857
:102040004869010600F19C80644A9A40154204D018
:1020500020680168880700F18C8010229A401542A0
:1020600003D021680868010771D4202000FA03F129
:102070000D4215D025682A68D50611D5B96094F8A7
:102080003530052B35D027683868400340F186800D
:102090003F68390340F19280E16B09B120468847DF
:1020A000606D002844D0656DEA071BD522684C4955
:1020B000052384F835301768A1FB061627F00100C8
:1020C0001060B50A03E022681768FB0704D5019B7E
:1020D00001339D420193F6D20021012084F834108F
:1020E00084F83500E36C1BB3204603B0BDE8F04034
:1020F00018472668356825F016023260216848695D
:1021000020F080034B61266C002E5CD022681168A1
:1021100021F008001060E66D3F23B340BB60236DE3
:102120000027012584F8347084F83550002BDBD16A
:1021300003B0F0BD0B6823F004000860E16D8A4035
:10214000BA60626DE36D42F00100606573E7BA60EA
:1021500023681A6850031AD41968CA0503D418688A
:1021600020F008021A60216C09B120468847E36D0F
:102170007BE7BA60626DE36D42F0040060656CE776
:10218000BA60626DE36D42F0020161655CE71B6855
:102190001903E8D5A16C0029E7D1E8E7396811F403
:1021A00080757FF479AF3A684FF0010C22F010038C
:1021B0003B6084F8345084F835C06DE7616C0029C9
:1021C0007FF46CAF6CE7A56C002D9FD1A3E700BF37
:1021D0004000012000000020010080000400800079
:1021E000B5814E1BF0B5704A704BD2F8D840DE6A0C
:1021F00083B0D4E91673002001903D68082202FAEA
:1022000003F1294203D02168086840077ED4684A58
:102210009A40154204D021684869010600F19C806B
:10222000644A9A40154204D020680168880700F18A
:102230008C8010229A40154203D02168086801075B
:1022400071D4202000FA03F10D4215D025682A68C8
:10225000D50611D5B96094F83530052B35D02768EF
:102260003868400340F186803F68390340F192802E
:10227000E16B09B120468847606D002844D0656D48
:10228000EA071BD522684C49052384F835301768C6
:10229000A1FB061627F001001060B50A03E02268D2
:1022A0001768FB0704D5019B01339D420193F6D2C9
:1022B0000021012084F8341084F83500E36C1BB34E
:1022C000204603B0BDE8F04018472668356825F081
:1022D000160232602168486920F080034B61266C49
:1022E000002E5CD02268116821F008001060E66DB5
:1022F0003F23B340BB60236D0027012584F8347071
:1023000084F83550002BDBD103B0F0BD0B6823F00F
:1023100004000860E16D8A40BA60626DE36D42F0CE
:102320000100606573E7BA6023681A6850031AD425
:102330001968CA0503D4186820F008021A60216CD5
:1023400009B120468847E36D7BE7BA60626DE36DB3
:1023500042F0040060656CE7BA60626DE36D42F0C4
:10236000020161655CE71B681903E8D5A16C0029CF
:10237000E7D1E8E7396811F480757FF479AF3A68FE
:102380004FF0010C22F010033B6084F8345084F8C5
:1023900035C06DE7616C00297FF46CAF6CE7A56C0C
:1023A000002D9FD1A3E700BF4000012000000020C6
:1023B0000100800004008000B5814E1B70B5964C72
:1023C0009648D4F8A02053695168034203F4813041
:1023D0002DD0CD052BD5D4F8E0506FF4807645F0A4
:1023E0000105C4F8E0505661002800F09E80D4F842
:1023F000E0506FF4007045F0020613F4823FC4F819
:10240000E060506103F4843025D160B1C9050AD57C
:10241000D4F8E000D4F8A02040F008056FF4006381
:10242000C4F8E0505361D4F8E01099BB70BD58B1C6
:10243000CE05DCD413F4823F03F48430E5D0D4F825
:10244000E0100029F2D025E013F4823F03F4843039
:10245000DBD0CD05E7D594F8DE50B4F8CAC094F8C7
:10246000DD10D4F8D060202D1FFA8CF3C9B262D0F1
:10247000D4F8E06046F00403C4F8E030116841F499
:1024800000751560D4F8A0606FF480627261002856
:10249000BED1C8E794F8DD60A6F12900012867D90C
:1024A00094F8DD20602A4FF000051CBF202284F83C
:1024B000DD20C4F8D05084F8DE50D4F8A060336832
:1024C00023F400603060D4F8A0502A6812051AD4B2
:1024D00094F8DD10602904BF202184F8DD1094F801
:1024E000DD20282AA2D1D4F8E0104B079ED5002089
:1024F0004B4EC4F8CC602023C4F8D00084F8DD3003
:1025000084F8DE0070BD6E6826F400636B60D4F85A
:10251000D400A8B390F83550424A0265022D34D059
:102520008025456500F0F6FED9E713F4823F03F4F9
:10253000843090D169E7002B9AD101F0F705212D65
:1025400003D0282994D1212E92D194F8DDC0D4F85B
:10255000CC1004295FFA8CF320D008291ED0212B3F
:1025600039D06FF48065556100287FF451AF5AE788
:1025700000214FF0280CC4F8D01084F8DDC09CE78F
:10258000D4F8D8000028C5D1A9E70668052180F84D
:102590003510306820F001033360A0E7282BDED12E
:1025A0001F4BC4F8CC3055686FF4806125F4E066A9
:1025B000566051611368002123F480664FF0200CAF
:1025C0001660C4F8D01084F8DDC084F8DE1000284E
:1025D0007FF41EAF27E7124EC4F8CC6094F8DDC03C
:1025E00094F8DE300CF003010B4320250026C4F8DC
:1025F000D03084F8DD5084F8DE6053686FF4806179
:1026000023F4E0655560516116680E40166000289D
:102610007FF4FEAE07E700BF40000120000101008B
:102620000000FFFF15330008F0B4AA4BD3F8A02038
:1026300095695169546893F8DE00C6B2102E8AB0CD
:1026400049D0402E47D0A44F0F40002F00F0DF802C
:10265000A70500F16C81A14FA14E2F400E40002F25
:1026600000F008819F4D0D40002D00F0638165054D
:1026700040F16081002E40F0608193F8DD40B3F8B6
:10268000CA108EB2E7B21EB3D3F8C400451CC3F81B
:10269000C45004781461B3F8CAC00CF1FF318EB293
:1026A000A3F8CA60B3F8CA0085B28DB9292F0FD13B
:1026B000576827F48064546093F8DDC093F8DE20F7
:1026C0000CF003010A432826C3F8D02083F8DD600C
:1026D0000AB0F0BC704711F0011F40D0A00500F116
:1026E000098181480840002843D07C4A7C482A4020
:1026F0000840002A5CD07B4D0D40002D53D065056D
:1027000051D5002800F05981A005E1D5D3F8CC407F
:1027100093F8DD70212FDBD1B3F8CA60D3F8A000A5
:10272000B2B2002A40F05F82042C05D0082C03D0FE
:1027300014F5803F40F0EA82416821F4E06545608D
:1027400004680027202244F400760660C3F8D070A5
:1027500083F8DD2093F8DE2083F8DE70B8E7624866
:10276000084030B1A705C0D5D3F8E470FEB21661B9
:10277000BBE7594F0F40002FB7D0A605B5D593F84A
:10278000DE00D3F8CC70D3F8D0C093F8DD60222EF1
:10279000C0B200F0868100270197566901969269C0
:1027A0000192019AA1E70028AED10AB0F0BC7047AF
:1027B0004E4D0D4035B3610524D5002800F0308121
:1027C000A20585D5D3F8CC40B3F8CA70D3F8A010D1
:1027D000BEB2032E00F0A681B3F8CAC01FFA8CF275
:1027E000022A00F0B581D3F8C4700E697A1CC3F8D0
:1027F000C4203E70B3F8CAC00CF1FF3081B2A3F818
:10280000CA1065E70028DBD10AB0F0BC7047384831
:10281000084000283FF41FAFA6057FF51CAF93F8D2
:10282000DDC0556825F4E061516009975469099449
:10283000166846F001001060D3F8A050099A296884
:102840005FFA8CF2A2F1280421F48066022C2E603B
:1028500040F24A81D3F8D070222F02D0222A7FF48E
:1028600037AF00202025C3F8D00083F8DD5083F86F
:10287000DE002DE71D480840002876D0600574D59D
:10288000002E75D193F8DD40B3F8CA50A9B2E7B273
:1028900000293FF41DAFD3F8C4601269701CC3F85F
:1028A000C4003270B3F8CAC00CF1FF34A5B2A3F86B
:1028B000CA50B3F8CA108EB2002E7FF409AF2A2F87
:1028C0007FF406AFD3F8A0707A6822F48060786055
:1028D000F2E600BF400001200200010004001000E9
:1028E0000400010080000100080001004000010018
:1028F0001000010093F8DE00402800F00181D3F8B9
:10290000B070B7F5804F4BD0D3F8F060002E00F0D8
:102910000081D3F8F00001287FF4E7AED3F8E4702B
:10292000FE1106F0060C4CF0F1001061DDE6936933
:102930009369CDE6002E3FF4CBAEA4057FF5C8AE7B
:10294000B3F8CA40A1B200293FF4C2AED3F8C460C4
:10295000771CC3F8C47030781061B3F8CAC00CF1AA
:10296000FF3295B2A3F8CA50B2E6002E3FF4B0AEE3
:10297000A1057FF5ADAEB3F8CA40A5B2002D3FF476
:10298000A7AED3F8C41012694F1CC3F8C4700A7004
:10299000B3F8CAC00CF1FF36B0B2A3F8CA0097E68C
:1029A00093F8DD70D3F8E460212F16BF46F00106DE
:1029B00006F0FE06F6B2166197E693F8DD70B3F8FE
:1029C000C86093F8DEC0D3F8CC50FAB25FFA8CF14D
:1029D000002E40F00481212A00F0488140297FF434
:1029E00077AE222A7FF474AEB3F8CA40A0B20028B2
:1029F00000F0358193F8DE70402F00F0C481D3F8E9
:102A0000C470D3F8A060781CC3F8C4003D78356169
:102A1000B3F8CAC00CF1FF3291B2A3F8CA1057E65E
:102A200093F8DD20222A7FF453AEB3F8CA00D3F81E
:102A3000A01085B2032D3FF6D6AEAC1E012CD3F804
:102A4000CC7040F2FF800E68022F14BF26F480661F
:102A500046F480660E60D3F8A020516821F4E0604F
:102A60005060D3F8C45014696F1CC3F8C4702C7044
:102A7000B3F8CAC00CF1FF36B2B2A3F8CA2093F87B
:102A8000DD1093F8DE0001F0030528432024C3F88D
:102A9000D000002783F8DD4093F8DE2083F8DE7055
:102AA00016E6D3F8F06016B9402800F0FD80D3F8A0
:102AB000F0602EB9D3F8B000B0F5404F00F0FB80C5
:102AC000B3F8CA60B0B2002840F0A38006905669FF
:102AD0000696906906900698176847F40076166087
:102AE0000022C3F8F02000E6BA49C3F8CC104FF03A
:102AF000200CC3F8D07083F8DDC083F8DE70E7E502
:102B0000D3F8F000E8B9D3F8E47007F0FE061661D8
:102B1000EBE5D3F8E470FE1106F0060C4CF0F00083
:102B20001061E2E5042C05D0082C03D014F5803F99
:102B30007FF459AE0F6827F480660E60D3F8A010BA
:102B400051E6D3F8E47047F00106F0B21061CCE52D
:102B5000042C56D0082C54D014F5803F51D00F6867
:102B6000022C14BF27F4806747F480670F6093F846
:102B7000DD1093F8DE6001F003021643C3F8D06065
:102B8000D3F8C450D3F8A0006F1C0469C3F8C47014
:102B90002C70B3F8CAC0D3F8C410D3F8A0600CF1FD
:102BA000FF3290B2A3F8CA0035694C1CC3F8C44088
:102BB0000D70B3F8CA70D3F8A060791E1FFA81FCBB
:102BC000A3F8CAC07268202022F440757560002402
:102BD00083F8DD0093F8DE2083F8DE4078E5212AD3
:102BE0003FF402AFFAE6D3F8C460721CC3F8C42005
:102BF00031780161B3F8CA506C1EA0B2A3F8CA00C4
:102C000066E51220C3F8D0000D6845F400740C602E
:102C1000B6E7B3F8CA60B0B201285CD0B3F8CA70A6
:102C2000BEB2022E00F09780106840F480671760F3
:102C3000D3F8A02000260296506902909769029767
:102C4000029A4DE7022F0E6800F0DD8026F48060C6
:102C50000860D3F8A0100D6845F400640C60D3F848
:102C6000A040636823F48061616031E5042DD3F8EE
:102C7000A07005D0082D03D015F5803F40F0978057
:102C80007E6826F4E06078603D68002645F40072B6
:102C90004FF0200C3A60C3F8D06083F8DDC093F8A1
:102CA000DE2083F8DE6013E5089657690897966979
:102CB0000896089A19E5079650690790976907974B
:102CC0000798166846F480701060D3F8F02001323F
:102CD000C3F8F02009E5042F2BD0082F29D0BCF130
:102CE000120F26D0D3F8CC001768022814BF27F49F
:102CF000806747F480671760D3F8A0200026059608
:102D00005069059097690597059AE9E6416821F4AD
:102D1000E065456093F8DDC093F8DE400CF00300F9
:102D200004432027C3F8D04083F8DE2083F8DD7009
:102D3000CEE4166826F480601060D3F8A020002747
:102D4000049756690496906904900498176847F4AC
:102D500000761660C4E6D3F8CC601068022E4ED020
:102D600020F480661660D3F8A000026842F4006781
:102D70000760D3F8A0200026039650690390976956
:102D80000397039AACE6D3F8F0602EBBD3F8EC407F
:102D9000D3F8A010D3F8E870012C38D0C7F3072679
:102DA0000E61D3F8F0000130C3F8F00090E47C68C5
:102DB00024F4E061796093F8DD7093F8DE0007F0A9
:102DC000030528432022C3F8D00083F8DE6083F88F
:102DD000DD207DE40000FFFFD3F8F050012D1ED070
:102DE000D3F8F020022A7FF473AC93F8DD10222987
:102DF00021D093F8DD40212C7FF46AACFFE540F44C
:102E000080671760B5E746F480620A6027E7FDB285
:102E10000D61D3F8F0200232C3F8F02058E4D3F863
:102E2000E860D3F8A000F5B20561D3F8F0200132D4
:102E3000C3F8F0204CE4D3F8A040236843F4807733
:102E4000276045E470B5454CD4F828371A68D9682E
:102E5000950601D5880627D4160619D50D0617D56F
:102E6000D4F84827511CC4F8481710785860B4F8B3
:102E70004EC70CF1FF35AEB2A4F84E673EB9DC6820
:102E800024F08002DA60D96841F04000D86070BD5B
:102E90005006FCD54A06FAD5D868202520F0400611
:102EA000DE6084F8615770BD2D4DD4F86C27286B17
:102EB0005B68111ADBB2882984F868370DD94FF0A6
:102EC000000C102BC4F86C0784F870C784F871C725
:102ED000DDD1012284F8712770BD94F8716796B333
:102EE000022B94F870670DD0032B14D0102B27D130
:102EF000002ECCD0501C00251370C4F86C0784F849
:102F0000715770BDA6B9012584F87167C4F86C07C4
:102F100084F8705770BD002EB9D0052908D94279C0
:102F20008B1F9A4204D1D4F8741701B188472863E3
:102F30000026C4F86C0784F8706784F8716770BD68
:102F4000002EF5D1A3E7102BC3D094F8700700280A
:102F50009DD0511C1370C4F86C1770BD4000012047
:102F6000000000204E4B1869C10700D470474D4B3C
:102F700093F878274AB193F8792762B94A494FF410
:102F800080508861013283F87927454A136923F01C
:102F900001011161704793F87A17481CB2EB400F9A
:102FA0007BDA4148416981F4805C4CF08051816159
:102FB000122AE7D910B493F8B84783B00022012C45
:102FC00001925ED00120D3F87C1783F8B8078C6893
:102FD000E20714D4354A364CD26A8868A4FB024210
:102FE000940C04EB440240F0010088600192019CC3
:102FF0002CB1019A501E0190019C002CF9D18A68D5
:10300000D4073ED5D3F8BC0720F4E06424F0010CCB
:103010004CF48072C3F8BC274868400507D5D3F844
:10302000BC4724F4405C4CF48052C3F8BC27D3F86E
:10303000BC0710F4805418BFD3F8C0471D4818BF10
:1030400024F006044FF0000C6FF0220283F8B8C79A
:10305000C3F8C0470A60D3F87C174C6844F0806C12
:103060004CF020024A604068C20602D0124CA142D5
:1030700007D18A6812F0405F03D1886840F080442D
:103080008C60074A002183F87917136923F0010047
:10309000106103B05DF8044B7047042988D180E7C4
:1030A0000004004040000120000002400000002019
:1030B00083DE1B43002301400020014010B54FF088
:1030C00080442369DB0706D50348416B88472269A2
:1030D00022F00103236110BD0000002010B40B4B4F
:1030E0000B4AD3F83806D3F87016C4680C80D3F8AE
:1030F00038164B684FF4007423F040034FF480609F
:103100004B60946190615DF8044B70474000012072
:1031100000040240034B5A69D00544BF4FF480704D
:1031200058617047003C0140794AD2F87C371968F1
:103130005868890701D580065BD419685868490723
:1031400001D500061CD419685868C90701D5410685
:1031500007D419685868890602D5410100F18F80AB
:1031600070471968C807F4D5D2F8BC176FF0010092
:1031700041F48031C2F8BC171860D2F87C37E8E718
:10318000D2F8BC17C90605D4D2F8BC0740F40051E8
:10319000C2F8BC17986810F4401F24D1996B11F441
:1031A000401F02D0986840051DD4596849051AD4BB
:1031B000986810F0405F16D1D2F8941799B9586802
:1031C00020F080015960D2F8BC0720F48051C2F889
:1031D000BC17D2F8BC07C00505D4D2F8BC1741F023
:1031E0000100C2F8BC076FF00C011960D2F87C37FF
:1031F000A9E7D2F8BC17C90605D4D2F8BC0740F439
:103200000071C2F8BC17986810F0405F44D0D86CC9
:1032100044F27C7180B201FB00F1C1F30F3C42F635
:103220001F318C45A2F82AC468D942F62D40844546
:1032300067D942F6E5518C4566D943F2C7208445EB
:103240008CBF4FF0040C4FF0030C92F8B81782F8C3
:103250007AC701290DD0012082F8B807996821F0BA
:10326000010098609968C80733D54FF0000C82F8C8
:10327000B8C76FF012011960D2F87C375DE7D2F859
:10328000C0176FF0200041F00201C2F8C0171860AB
:10329000D2F87C2710607047D2F894170029B6D175
:1032A000D86A10F4700F25D1586820F020015960B9
:1032B000D2F8BC0720F48071C2F8BC17D2F8BC0762
:1032C000C104A4D4D2F8BC1741F00100C2F8BC0775
:1032D0009DE7586820F0806C2CF020015960D2F8EE
:1032E000BC0720F4885C2CF0010141F00100C2F819
:1032F000BC07BAE79968480589D4D5E74FF0000CB8
:10330000A3E74FF0010CA0E74FF0020C9DE700BFD0
:1033100040000120836B19680A6822F4806008600D
:10332000596B00225A850A65986B0265202093F834
:103330003D1083F83D0083F83E20704710B4836B46
:10334000186802680021202422F4806202605985F6
:1033500083F83D4083F83E10186C40F0100119646A
:103360005DF8044B704700BF836B93F83D2093F8E2
:103370003E10D0B22128CAB227D0222823D0196803
:10338000086820F480620A601968086840F40072D6
:103390000A601968486820F480524A6019684A68CF
:1033A0004FF0000C22F400604860A3F82AC01A6CA9
:1033B00042B9202183F83D1093F83E0083F83E2067
:1033C000402811D07047202AD9D119684A6822F4C0
:1033D000006048601A684FF0000CA3F82AC05368D8
:1033E00043F4407151607047704700BF2DE9F041D0
:1033F0009C4A936803F00C01042982B000F0D58048
:10340000946804F00C05082D00F0CB80954FBA6845
:1034100002F00C030C2B00F0FA80934C934A914974
:10342000012525704668D2F89C40002E00F081806E
:103430000E68B60308D4D2F89C703B1B642B00F2D4
:10344000AC800E68B603F6D501688A0735D5854C81
:10345000A26812F00C0F00F0AF80A56805F00C0612
:10346000082E00F0A5807F498B6803F00C040C2C1B
:1034700000F0ED80C568002D00F0D8807C4E7B49BF
:10348000784A01273760D1F89C7005E0D1F89C306C
:10349000DC1B022C00F2818013689D07F6D51468AE
:1034A0004FF0F80898FAA8FC0569BCFA8CF18D4039
:1034B00024F0F8063543156001680F0714D54669F6
:1034C000002E00F084806B4F684A664901263E60FA
:1034D000D2F89C4004E0D2F89C60351B022D5CD8E9
:1034E0004B6F9E07F7D501684A0726D48769BFB19D
:1034F0005C4A916801F00C05082D64D0022F5E4EE5
:103500005A4900F0A98000203060D1F89C7004E096
:10351000D1F89C30DD1B022D3FD81468A301F7D4ED
:10352000002002B0BDE8F081D2F89C301D1B642D54
:1035300033D80F68BD03F7D486E74A4D4F490022C0
:1035400001922C6C494A44F080572F642E6C06F08F
:1035500080530193019B0D6845F480740C60D2F890
:103560009C5004E0D2F89C305F1B022F15D80F68E6
:10357000FB05F7D5424E017A31708368D2F89C5032
:10358000384941F28838002B46D00B6F9F07ADD4E5
:10359000D2F89C60741B4445F7D9032002B0BDE803
:1035A000F081566873027FF531AF2E490B684BE707
:1035B00067687B023FF557AF2A4D2E68B60716D5D0
:1035C000C168012913D0012002B0BDE8F08129496A
:1035D000264A0E60D2F89C40224E04E0D2F89C307D
:1035E0001D1B022DD9D8776FBD07F7D47BE71D4F80
:1035F0004FF0F8083C6898FAA8FC0369BCFA8CF212
:1036000024F0F80593402B433B60016855E7796847
:103610004F027FF502AFC8E70F6FBE077FF566AFB9
:10362000D2F89C40661B4645F6D9B6E7104E0F4AC5
:103630003560D2F89C400B4904E0D2F89C301D1B49
:10364000022DAAD80F68BB07F7D4016835E74A688E
:1036500057023FF50FAFAFE700243460D1F89C402C
:1036600015E000BF0038024002380240400001204F
:1036700000004742800E4742600047420070004011
:1036800070380240D1F89C301F1B022F85D8166875
:10369000B501F7D447F6C07797FAA7F34FF4403552
:1036A000B3FA83F895FAA5F44FF07066B4FA84FE85
:1036B00096FAA6F74FF0E043B7FA87F793FAA3FC20
:1036C000D0E90954D0E9073605FA08F8334364080D
:1036D000D0E90B56013C04FA0EF043EA0803BCFAA9
:1036E0008CF4034305FA07F73B4306FA04F5094E49
:1036F00009482B43012453603460D1F89C2005E035
:10370000D1F89C50AE1A022E3FF647AF0768BC01B5
:10371000F6D505E76000474200380240094B4FF4F8
:10372000E0529B6892FAA2FC07490848BCFA8CF266
:1037300003F4E053D3400B44C06A93F89410C8409C
:10374000704700BF0038024000BD000800000020A4
:1037500070B40668B40707D5894A8468936823F073
:10376000F005254395600668F2072BD54568012DC5
:1037700000F0B580AA1E824C012A236840F2FC802A
:103780009C0740F188807E4B7E4C9E6826F00302A9
:103790002A439A604268D4F89C50012A41F2883C3E
:1037A00000F08180022A00F08980032A06D190E08F
:1037B000D4F89C60721B624500F2DB809A6812F0BC
:1037C0000C0FF5D1704C236803F00F058D425BD8C8
:1037D0000468620707D56A4DC168AB6823F4E056F8
:1037E0000E43AE600468230707D5654A00699568F3
:1037F00025F4604141EAC0039360614EB46804F06F
:103800000C02082A00F092800C2A6ED05F4B5C4EAE
:10381000F025B16895FAA5F45D485E4AB4FA84F6DD
:103820002940F14001445C4C91F89410CB40A2FB3C
:1038300003108209561EB6F1807FE36208D2574B0F
:10384000574C5E600021072084F82350996018606F
:10385000534DEA68C2F30226C6F10701042906F1B6
:10386000040328BF04214FF0FF308840062B8CBF93
:10387000033E0026C543B5402E01494AF1B282F805
:103880002310002070BC7047CEB22670226802F070
:103890000F04A1429CD0012070BC7047D4F89C60FA
:1038A000721B624565D89E6806F00C02042AF5D1A9
:1038B00088E7D4F89C60721B62455AD89E6806F06F
:1038C0000C02082AF5D17DE7D4F89C60721B624592
:1038D0004FD89E6806F00C020C2AF5D172E7284EEC
:1038E000326893033FF54FAFD5E77568706871682C
:1038F00005F03F0C47F6C07090FAA0F6B6FA86F4D1
:1039000001401F48214B4668B3FBFCF521FA04F245
:1039100005FB02F54FF0E04C9CFAACF1B1FA81F4F2
:1039200006F0E042E240B5FBF2F370E773687068BE
:10393000766803F03F0547F6C07090FAA0F1B1FA3F
:1039400081F4064026FA04F20D4E104B7468B3FB66
:10395000F5F54FF4403005FB02F590FAA0FCBCFAF7
:103960008CF104F44032CA4001325300B5FBF3F34A
:103970004DE7032070BC70479E013FF504AF8AE716
:103980000038024040000120003C02400024F400C6
:1039900000BD0008D34D62100000002010E000E0E0
:1039A00000ED00E0094B4FF460429B6892FAA2FCE4
:1039B00007490848BCFA8CF203F46043D3400B4437
:1039C000C06A93F89410C840704700BF00380240A6
:1039D00000BD0008000000202DE9F84F4F4A504E6E
:1039E0005369DFF84C8183F0020141F400349461A3
:1039F00005464FF42A7206F2C470002107F098FEC3
:103A0000DFF830C1002286F86C2A1446A800A6F818
:103A1000702A06F6942706F67429ACF1A40E5CF819
:103A2000041B57F804B091F800A00EEB8A0307EBD3
:103A3000040AD3F8AC5005443D518B78DAF80410F1
:103A40000EEB8303D3F8AC3003448B4263D0CAF847
:103A50000430344D49F8142005EB040B04EB080343
:103A6000ABEB030AAAF11001090909EB4405013186
:103A700011F007016A60AA60EA6022D001291BD018
:103A8000022916D0032911D004290CD0052907D00A
:103A9000062902D0C3E900221033C3E90022103303
:103AA000C3E900221033C3E900221033C3E9002226
:103AB0001033C3E900221033C3E9002210339B45C1
:103AC00015D01A67C3E90022C3E90422C3E908221A
:103AD000C3E90C22C3E91022C3E9142203F1700ADE
:103AE000C3E9182280339B45CAF80420E9D1083481
:103AF000102C94D109480C4AC6F824270427876162
:103B000043690A4CC6F81C4783F0020646F40035A8
:103B10008561BDE8F88F5D45E9D09AE7000802406D
:103B20004000012058440120DB1B0400B9A2010021
:103B300058240120A4BD00082DE9F04FDFF8708360
:103B400098F8A52A0023A1B088F8A43A002A00F02A
:103B50005683D248069300F517610791D04C98F828
:103B6000AC7A257D98F8AD9AD8F8A86AAF4228BFFC
:103B70002F464022A94506EB050338BFA946002180
:103B80000DEB0200C8F8A83A88F8AC7A88F8AD9A2C
:103B900007F0CEFD98F8AE0A98F8AFBA0130C3B27C
:103BA0009B4588F8AE3A00F0F782BE4CBB4FE11857
:103BB00091F884C091F878E00CEB4C0222447244F6
:103BC00092F8905092F89C6007EB850A07EB860903
:103BD000DAF8AC40D9F8AC00B24D08902B44099407
:103BE00093F887B093F88A1093F88DC093F87B60B0
:103BF00093F87EA093F881900BEB4B0E01EB4107FD
:103C00000CEB4C022A44AE442F44B6445744914432
:103C1000A24E9EF8905097F890009EF89C4097F81E
:103C20009CB099F89C3099F8907006EB850C06EBE7
:103C3000830906EB840E06EB800A06EB8B0106EB8C
:103C40008702D9F8AC30DCF8AC50DEF8AC40DAF8DA
:103C5000AC00D1F8AC70D2F8AC60CDE90A45CDE942
:103C60000C70CDE90E364FF40079E0E0D8F8002270
:103C7000D5B2043508EB450CBCF8FC41D8F800027D
:103C80001FFA84FB0FFA8BF303FB03F70130BE131B
:103C9000C8F8000282490A988A69D8F81074A2F814
:103CA00000B0DDE90854B0F90210B4F902C0B5F96A
:103CB00002E035F904BB34F9042B089503FB01F14C
:103CC00003FB0BF503FB0CFB4BF38F3C41F38F3BEA
:103CD0001099099445F38F3503FB02F4691844F3F6
:103CE0008F32DDE9115403FB0EFE30F904AB029173
:103CF00022444EF38F3E009210910EEB0501DDE958
:103D0000132E03FB0AFAD8F8B04A159D05914AF321
:103D10008F3A01373444119162440099624E1291F6
:103D2000F2440BEB05010A90D8F8B45A1392C7F38A
:103D30000E00CDF850A0C8F81074594FC8F8B04A1A
:103D400006EB4000B861DDE90B70B7F902C0179CC3
:103D5000B0F90260DDF838E0159103FB0CFB4BF382
:103D60008F3BA344CDF85CB037F904BB0B9703FB42
:103D70000BFB169FBEF902401D444BF38F3B5F4483
:103D8000C8F8B45A0D9D30F904BB169703FB06F62C
:103D9000199F0C90AC4646F38F36B5F9025003FBE1
:103DA0000BF0374440F38F3B03FB05F51B98199745
:103DB000189F3CF9046BCDF834C045F38F353EF9BC
:103DC00004CBCDF838E05F44054418971A981B954A
:103DD000DDE91CB503FB04F403FB06F644F38F3462
:103DE0002C4446F38F360F9D03FB0CF7064447F334
:103DF0008F3E1A96B5F9026035F9047B1E980F952F
:103E0000F34403FB06F6CDE91CB403FB07F31F9C48
:103E100009F1FF3746F38F3C43F38F336444034487
:103E20001FFA87F9CDE91E34B9F1000F42D0D8F856
:103E3000FC11D8F800228A4222D098F88C11D8F8C8
:103E4000883159B1D8F8042442B1D8F808545C1B21
:103E5000142C00D890470698C8F80404D8F80C74BD
:103E6000D8F8FC61D8F8001201378E42C8F80C74FB
:103E70007FF4FCAE00264FF0FF334FF6FF7B09E7DF
:103E80000A4D2C6924F00400286130BFD8F8FC7179
:103E9000D8F80062B742D0D1F2E700BF00BD0008F9
:103EA00000000020F8CD00084000002000ED00E0F8
:103EB0004000012098F8B84AC448DDF808B0DDF8A1
:103EC00014E098F8A49A0D46082156468161002C0A
:103ED00000F087808EFB0E01870B82FB02238BFB99
:103EE0000BBCCDE9022347EA8141009F029A4FEAC9
:103EF0009B3343EA8C4087FB07AB039B970B4FEA4E
:103F00009A3A08EB491C47EA83474AEA8B4B01443B
:103F10005F44012CCCF8BC1ACCF8C07A61D9DDE939
:103F2000161081FB01AB80FB00234FEA9A3747EA6A
:103F30008B40920B85FB05AB86FB065642EA834716
:103F4000A90B4FEA9A3343EA8B4A41EA8645384443
:103F50005544022CCCF8C80ACCF8C45A41D0DDE94B
:103F60001876DDE91A2087FB07AB86FB0667B10BE5
:103F700041EA874582FB026780FB00014FEA9A33E2
:103F8000B60B43EA8B4E46EA874B870B47EA8142E2
:103F900075445A44032CCCF8CC5ACCF8D02A20D003
:103FA000DDE91C3183FB03ABDDE91E604FEA9A3A81
:103FB0004AEA8B4581FB01AB4FEA9A3747EA8B42CD
:103FC00086FB066780FB00ABB30B4FEA9A3143EAEE
:103FD000874641EA8B4B2A445E44CCF8D42ACCF87D
:103FE000D86A98F8A55A794B09F10100C7B24FF485
:103FF0000022BD4288F8A47A9A613FF6AFADA2468E
:10400000724C1026A661BAF1000F00F0D680DFF8DE
:10401000C891B8F8C85B99F800B0DFF8C0E1D9F8EA
:1040200038700BF1FF3C5FFA8CF12024A81C0AF1D8
:10403000FF32013514FB014650FA82FA0696A8B207
:10404000DEE900561FFA8AF300220593AEF5827C62
:104050000292CDE90056BBF1000F00F09B80069C58
:10406000A4F120035E090136002316F0030519466A
:10407000624604EB0C0A53D0012D1CD0022D0DD04A
:10408000DCE90024A242CBBF121BA21A1C46012469
:10409000002AC4BF114623460CF12002D2E9005683
:1040A000B542CBBFAE1B761B002501258E42C4BF97
:1040B00031462B462032D2E90045AC42CBBF651BCE
:1040C0002D1B0024012420328D42C4BF29462346E3
:1040D000924525D13AE0541B00228C42C8BF2146AC
:1040E000D6E90845C8BF1346AC42CBBF641B2C1BA6
:1040F000002501258C42C8BF2146D6E91024C8BF3F
:104100002B46A242CBBF121BA21A002401248A42D2
:10411000C8BF114606F16002C8BF2346924515D0BC
:10412000D2E90064A642CBBF341BA41B00260126A3
:104130008C42C8BF334602F12006126A7568C8BFB8
:104140002146AA42C7DCAC1A0122C6E7DDE90045D8
:10415000641845EBE175CDE900454FFA83FA3B78E9
:104160004AEA430110F0070A397007D1184E0137A7
:10417000BD1BB5F5897F33D201240294421C0599F9
:1041800093B28B420CF1080C0DD01846BBF1000F16
:104190007FF465AFDA46E2E7069B88F8AE3A0D4851
:1041A000079C002318E5DDE90056CEE90056029E83
:1041B0000EB1C9F83870A8F8C80B04484FF480173E
:1041C0008761012021B0BDE8F08F00BF00080240E8
:1041D0000C0C012070BE000800000020000C012023
:1041E000B8F8A441A8F8C80BDDE900BC0134C9F84F
:1041F0003870CEE900BC5046A8F8A441E2E798F830
:10420000B8AAFDE607490023C1F89031C1F89431FE
:10421000C1F89831C1F89C31C1F8A031A1F8A4319E
:10422000012070474000012008B5402200210248CB
:1042300007F07EFA012008BDE801012005490023AE
:10424000C1F8EC31C1F8F031C1F8F431A1F8F8311E
:1042500001207047400001202DE9F04FC94ACA4BA8
:10426000CA4CCB4DB1B002F58051009003F500600F
:1042700002F500660C9004F5006709920A9110A8F7
:10428000802200210E9408930D960B970F9507F04E
:104290004FFAC04C4FF40078D4F8FC21D4F8003227
:1042A0009A42F9D094F88C51D4F888015DB1D4F8D1
:1042B000046446B1D4F80814471A142F00D8B04744
:1042C0000022C4F80424D4F80C34D4F8FC51D4F8F7
:1042D000000201338542C4F80C3400F06181D4F847
:1042E0000062F1B2043104EB410ABAF8FC71D4F86F
:1042F00000221FFA87F901320FFA89F3C4F800226D
:10430000A5490A988A690B9FA2F80090DDE9086523
:10431000B6F902B036F9042BB5F902E0109935F977
:1043200004AB089603FB02F2B0F90260099542F370
:104330008F323D46114403FB06F6119A109103FBA0
:104340000BFB35F9041B46F38F3C4BF38F3B30F9E5
:10435000046B0A905A4403FB01F103FB06F003FBD4
:104360000EF9129E119203FB0AFED4F8102441F3B9
:104370008F3B13994EF38F3A49F38F3940F38F3EB9
:1043800001325644494485481296DDE9159AC2F334
:104390000E0613911499C4F8102400EB46027E4EC9
:1043A0007144E144D344B2611491CDE9159BDDE938
:1043B0000C010B95B1F90250B0F902A030F904EBF1
:1043C000B7F90260179F0C90DDE90E2C03FB05F591
:1043D00003FB0EF903FB0AFA45F38F3E219DB2F968
:1043E000020003FB06FB4AF38F3A664655444BF343
:1043F0008F3B5F442195209D36F904BB179749F305
:104400008F3931F9047B0D914D4403FB07F1209561
:1044100032F9047B0E9203FB0BF5239A45F38F3A96
:10442000229D41F38F3129447244269D239203FB40
:1044300000F0259A229103FB07F7249940F38F306F
:1044400047F38F3710440F44554425902497269501
:104450000F96BCF90260279803FB06F308F1FF37BB
:1044600043F38F3303441FFA87F82793B8F1000F03
:104470007FF412AF009CA446C4F800804CF8048F6F
:1044800010AA0C3406920794CDF814C00599DDF8F3
:1044900018E0A1F1040B0BF102050495F446DCE9E8
:1044A000006086FB065680FB0034AF0B9B0B47EA8F
:1044B000864143EA8444621877D44FEAA2494FEA1E
:1044C00082384FF080430022950845EA8372904578
:1044D0004FEAA30379EB0301F6DB52EA03014FF045
:1044E000000035D0CDE900230021CDF808B0DDE98A
:1044F0000045A208A24624184FEAA50742EA85769D
:10450000AB464D41A04579EB05030ADB1AEB0A0ADD
:104510004BEB0B0210EB0A005141B8EB040869EBBE
:104520000509CDE90067DDE9003449104FEA3000A4
:104530002343DCD1642101FB00F00028DDF808B042
:1045400004DA00F57F1000F57F503F30C0F387504C
:104550000BF8010B049FBB450CF1080C9FD1059E85
:10456000B3450EF1100E96D1069D079B0BF1040486
:104570004035A3420594069588D1082031B0BDE8A6
:10458000F08F00BFA0DE0008A0CE0008A0F6000853
:10459000A00601084000012000000020400000208B
:1045A0004FF0FF334FF6FF79AAE60020D0E700BFB7
:1045B0002DE9F04FADF2A44DC37845790090014646
:1045C000C3F3800044000444DFF8D890344FA400C3
:1045D0000DF10C0809EB04062A4606314046FE613F
:1045E00004F010F90C2D5FD8002D00F05E82681EDB
:1045F0000DF10D0757FA80FBC44600231CF8011B80
:104600004B4013F0800F4FEA430218BF82F097022D
:10461000D3B2580013F0800F18BF80F09700C7B2D4
:10462000790017F0800F18BF81F09701CAB25300CC
:1046300012F0800F18BF83F09703D8B2470010F034
:10464000800F18BF87F09707F9B211F0800F4FEA7B
:10465000410218BF82F09702D3B213F0800F4FEAE5
:10466000430018BF80F09700C7B217F0800F4FEAE1
:10467000470118BF81F09701DC45CBB2BED124AF12
:1046800038464FF40272002108F8053007F050F860
:1046900019F80440002D40F00382AE46A9465EE0C2
:1046A0000000002074BD0008691E0DF10D0212FA11
:1046B00081FAC34600234BF6AD201BF801CB83EAF9
:1046C0000C2E0FFA8EF7BBB2002FACBF5B0080EA56
:1046D000430399B20F0454BF490080EA41018AB2F2
:1046E000170454BF520080EA420293B21F0454BF21
:1046F0005B0080EA430399B20F0454BF490080EA8B
:1047000041018AB2170454BF520080EA420293B2B8
:104710001F0454BF5B0080EA430399B20F044CBFEF
:1047200080EA41014900DA458BB2C6D11A0A08EB8A
:10473000050A24AF08F8052038464FF4027200211C
:104740008AF8013006F0F4FF4FF0020A19F804402D
:104750001FFA85F9CA441FFA8AF94FEAC90EA6441E
:104760000EF1FF3292FBF4F3002B98F800C040F3F7
:10477000C98000218E4680229A4601954FF00003A1
:1047800027F81E3007EB4E05002C00F0B3801CEA22
:10479000020F04F1FF3014BF01230023520800F080
:1047A000030B07D10131C9B289458CBF18F801C08C
:1047B000944680220120A04280F09B804FFA8BFB20
:1047C000BBF1000F41D0834528D0BBF1020F12D0BE
:1047D0001CEA020F03FA00F318BF43F00103C240C2
:1047E0009BB207D10144C9B289458CBF18F801C0FA
:1047F0009446802201301CEA020F4FEA430318BF9F
:1048000043F0010352089BB207D10131C9B2894577
:104810008CBF18F801C09446802201301CEA020FB8
:104820004FEA430318BF43F0010352089BB207D17C
:104830000131C9B289458CBF18F801C09446802265
:1048400001305FFA80FBA34553D21CEA020F4FEA06
:10485000430318BF43F0010352089BB207D1013153
:10486000C9B289458CBF18F801C0944680221CEA61
:10487000020F4FEA430318BF43F001035FEA520BF4
:104880009BB200F1010008D10131C9B289458CBF4A
:1048900018F801C0DC464FF0800B1CEA0B0F4FEA02
:1048A000430218BF42F001025FEA5B0B93B208D1EA
:1048B0000131C9B289458CBF18F801C0DC464FF000
:1048C000800B1CEA0B0F4FEA430218BF42F00102B3
:1048D00093B25FEA5B0207D10131C9B289458CBF4F
:1048E00018F801C09446802203305FFA80FBA3458C
:1048F000ABD32B800EF101051FFA85FEF2453FF781
:104900003DAF019D0DF5267840464FF4027200211F
:1049100006F00EFF4FF0000ADDF800900AE0726822
:1049200037F81B009047624B28F81B00DE6999F8A6
:10493000055034781FFA8AFB2DB10D2D34BF0123A9
:1049400002231D44ED002544681E90FBF4F4A345AA
:104950000AF1010AE3DB76780127731E9F40B9B2A2
:10496000A4B2002900F09880621E1FFA82F90DF2AD
:104970009A2C504A0CEB49050023002C00F089804A
:10498000A5EB080EAEF102004708013717F003004F
:1049900046463ED0012828D0022811D036F8027BA6
:1049A00092F800B0394203F1010314BF0127002738
:1049B000DBB2082B47EA4B00107004BF0023013222
:1049C00036F802AB92F8009011EA0A0F03F10103E6
:1049D00014BF4FF0010A4FF0000ADBB2082B4AEA7D
:1049E0004907177004BF0023013236F8020B92F812
:1049F00000C0014203F1010314BF01200020DBB21B
:104A0000082B40EA4C00107004BF00230132B5426D
:104A10003FD0304692F800E030F8026B013331426B
:104A200014BF01260026DBB2082B46EA4E0717709A
:104A3000B0F800B004BF01320023167811EA0B0F62
:104A400003F1010314BF4FF0010B4FF0000BDBB279
:104A50004BEA4607082B177001D100230132B0F84A
:104A6000029092F800A011EA090F03F1010314BFAC
:104A70004FF001094FF00009DBB249EA4A06082B62
:104A8000167008BF002300F1060608BF01328088B7
:104A9000ADE749087FF471AF0DF2A44DBDE8F08F8A
:104AA0001FFA85F94FF0010A54E62B46E7E500BFEF
:104AB000000000202E0D01202DE9F04FDFF808B393
:104AC000BE4CDBF83C20ADF2AC4D20200192A06141
:104AD00056793EB94FF400150120A5610DF2AC4D99
:104AE000BDE8F08F019BB648DC78C4F380077A00FC
:104AF0003A449300A0F1740898440D2E98F87490ED
:104B000098F8757034BF012502253544034409EB3C
:104B1000C505A8AC691ECBF81C3091FBF9F50393D1
:104B20002046ABB200216A00029306F001FE039B0F
:104B3000002F00F0A6800298421E91B20DF2A22A28
:104B40000AEB41089F494FF0000E8022002D00F033
:104B50009180A8EB040CACF102004FEA500909F176
:104B6000010A1AF0030C204639D0BCF1010F23D002
:104B7000BCF1020F0FD00878B4F8009002424FEA5F
:104B8000490A204618BF4AF0010A20F802AB520831
:104B900004BF01318022B0F800C091F800904FEAC4
:104BA0004C0A12EA090F18BF4AF0010A20F802ABBA
:104BB000520804BF01318022B0F800C091F8009083
:104BC0004FEA4C0A12EA090F18BF4AF0010A5208CC
:104BD00020F802AB01D10131802240454AD0B0F823
:104BE000009091F800A0844612EA0A0F4FEA4909A2
:104BF0000CBF484649F001002CF8020B5208E14670
:104C000008BF013139F8020B91F800A008BF8022DB
:104C100012EA0A0F4FEA400018BF40F001005208A4
:104C200029F8020C01D180220131BCF8020091F870
:104C300000A04FEA400912EA0A0F18BF49F0010923
:104C4000520808BF0131ACF802900CF1060091F84F
:104C500000A0BCF804C008BF802212EA0A0F4FEA85
:104C60004C0918BF49F00109520820F8029CB2D043
:104C70004045B4D10EF1010E5FFA8EF087423FF647
:104C800065AF002D00F09481029ADFF84091DFF8C3
:104C90002CA1511E8DB26E000DF2A22C0CEB060859
:104CA00026AF18F0020F01963E4640F09180314643
:104CB0000DF112029B6834F8020B9847B51C0DF1F8
:104CC00012022946AE1C002800F0AB80BDF812305D
:104CD000A3B1DBF83CC0B9F8A0E19CF88800184407
:104CE0008CF88800DAF8145085F0400C5EFA83F3F3
:104CF0004CF48000A9F8A031CAF81800DBF81C5069
:104D000034F8020BAB689847002800F08A80BDF8A1
:104D10001250A5B1DBF83C10B9F8A0E191F8882059
:104D20002A4481F88820DAF8140080F040015EFA05
:104D300085FC41F48003A9F8A0C1CAF818304445A5
:104D4000DBF81C30B3D10DF114088222404600215B
:104D5000029306F0EDFC029C94F80090012609F104
:104D6000FF3506FA05F2019D07F1020A1FFA82FEDD
:104D700000235544724644461E46AE46C2B13F88A3
:104D8000B446114639424FEA430318BF43F00103CA
:104D90000CF007050136072D1BB2B6B2C1F34F0167
:104DA00009BF23709BB200230134B4460029E9D126
:104DB000F245574646D00AF1020ADFE700080240F2
:104DC00074BD00081A0C01200000002040000120E2
:104DD00020889C680DF112023946A0470DF2A224EA
:104DE000F8B1BDF81230A3B1DBF83C10B9F8A0E17E
:104DF00091F88800184481F88800DAF8142082F0CD
:104E000040055EFA83F645F48003A9F8A061CAF86C
:104E100018304445DBF81C3007F102067FF447AF39
:104E200091E7674D674F6B69B7F8A24183F0800146
:104E300041F400060134AE61A7F8A2410DF2AC4D79
:104E4000BDE8F08FDBF83C40019466790C2E6CD8FD
:104E5000751EEFB2FD2F51D80DF115029119C44600
:104E600000271CF8014B67407B0017F0800F18BF2C
:104E700083F09703D8B2450010F0800F18BF85F07B
:104E80009705EFB27A0017F0800F18BF82F09702F3
:104E9000D4B2630014F0800F18BF83F09703D8B228
:104EA000450010F0800F18BF85F09705EFB217F09E
:104EB000800F4FEA470218BF82F09702D4B214F075
:104EC000800F4FEA440318BF83F09703D8B210F065
:104ED000800F4FEA400518BF85F097056145EFB296
:104EE000BFD1B8B250B1374EB6F89E210020013282
:104EF000A6F89E210DF2AC4DBDE8F08F0198414619
:104F00000630324603F07EFC6EB10C2E94BF0122B7
:104F1000022200211644884601E01FFA81F8464526
:104F200001F10101F9DC264CD4E50DF595608219FB
:104F3000A2F2924BC14600204BF6AD2519F8017B39
:104F400080EA072A0FFA8AF18BB20029ACBF5B0016
:104F500085EA43039CB2220454BF640085EA4404FA
:104F6000A0B2070454BF400085EA400087B23A046B
:104F700054BF7F0085EA4707BAB2170454BF5200F6
:104F800085EA420291B20A0454BF490085EA410110
:104F90008BB21F0454BF5B0085EA43039CB222041A
:104FA0004CBF85EA44046400D945A0B2C6D199E754
:104FB0000DF1140829464046822206F0B9FB45E768
:104FC00000080240400001202DE9F04F7F4C94F88A
:104FD000F86D94F8F93DB34289B0054639D094F89C
:104FE0008401B0B3E97801F00303012B00F0C7801E
:104FF000022B00F09A80AA787F2A32D094F8FA1D0A
:10500000D4F8F40D40F8215094F8FA5D94F8F89D26
:105010000135EAB2914584F8FA2D1ED994F8F93D8C
:1050200094F82674013384F8F93D012F05D16849BD
:1050300084F827744FF400678F6194F8845145B168
:10504000681E5FFA80F804EB880C84F88481DCF831
:105050005C51284609B0BDE8F08F002684F8FA6D4F
:10506000DCE769790029C9D06B7894F82F0498425D
:1050700001D0FF2BC2D1D5F806A094F82674D5F83C
:105080009010D4F8988E9AFA8AF2022F029205F1C3
:10509000060900F08F800391DFF840B1D4F8882131
:1050A0000192A1EB0801A1FB0B014A4A002303F086
:1050B00029FA029BC01A00EBD0724FEA620C0198E9
:1050C000ACF1220121EAE173A0EB0802A2FB0B0183
:1050D00093FA83F83F4ACDF81080002303F012FAC8
:1050E000039B01993B4AC91A90FA80FC0023A1FB5B
:1050F0000B01CDF814C003F005FA00BACDE9060A99
:105100000DF1100ABAE80F004FF0100BC9F80000BB
:10511000C9F80410C9F80820C9F80C3085F805B0A2
:1051200094F8F92DB24280D068E794F82F746A7829
:10513000BA4202D0FF2A7FF45EAF94F88D110029A5
:105140007FF459AF01269822234884F8FC6D06F0BD
:10515000EFFAD5F8941084F8007E2B7895F8048047
:1051600084F8013E08BA7F274FF00409C4F8060E00
:1051700084F8048E84F8027E84F8059E3EE795F854
:1051800001A094F82FB4D3457FF435AF98220021C5
:1051900004F5606084F8FC3D06F0CAFA84F800BEAD
:1051A0002E782F7984F8016E7F2384F8023E84F8EC
:1051B000047E23E70648436983F4006242F00063FB
:1051C0008361D5F89000039066E700BF400001209E
:1051D00000080240400D0300400E012040420F0035
:1051E00030B4064C05460FCC247828602C746960D6
:1051F000AA60EB60112030BC704700BF3C1203086E
:105200004379012B01D0012070478179BB4A080204
:1052100083B2000446BF4BF6AD2383EA41235B0013
:1052200098B25FEA004C46BF4BF6AD2C8CEA4000CA
:10523000400082F82F1481B2080446BF4BF6AD2C13
:105240008CEA410149008BB25FEA034C46BF4BF642
:10525000AD2C8CEA43035B0099B2080446BF4BF6C1
:10526000AD2C8CEA4101490088B25FEA004C46BF90
:105270004BF6AD2C8CEA4000400083B2180446BFC8
:105280004BF6AD2C8CEA43035B0098B2010446BF99
:105290004BF6AD2181EA40004000B2F82D341FFAF0
:1052A00080FC6345AFD0F0B4FF2492F8DD50A2F843
:1052B0002DC486B082F82C44D2F82C64CDF8056059
:1052C0000027202D8DF8047003D0012006B0F0BC1B
:1052D0007047D2F89C4092F8DD109DF805009DF8CB
:1052E00006309DF807C09DF8085082F89C7E052680
:1052F000202982F89D0E82F89E3E82F89FCE82F889
:10530000A05E82F89C6FE0D1D2F8A07005E0D2F8E0
:105310009C60301B192800F2DB80B969C84310F08B
:105320000203F4D092F8DC50012DCED0012682F891
:10533000DC603868724920F400633B604FF0210C58
:105340001027002582F8DDC082F8DE70C2F8E05038
:10535000C2F8CC10D2F8CC60D2F8A030042E00F005
:10536000AD80012E00F0AA8016F5803F00F0A680E7
:10537000D2F8D000122806D1A0E0D2F89C100F1B62
:10538000012F00F2AE805D69E807F6D5D2F8B06073
:10539000B6F5804F10D0F02018610AE05F6917F46D
:1053A000806740F0B180D2F89C502E1B012E00F295
:1053B000C18059690907F1D5A02018610AE05D692B
:1053C00015F4806740F0A080D2F89C60301B012863
:1053D00000F2B0805969CF4317F00205EFD1009574
:1053E0005E690096986900900099464E052508E090
:1053F000586910F4806032D1D2F89C100F1B012F35
:1054000045D8596911F08001F2D037781F615F6982
:10541000681E7F0781B206F1010046D40D4606469C
:1054200008E05F6917F4806019D1D2F89C100F1B57
:10543000012F2CD85F6917F00401F2D0002DE0D1C4
:105440001C6844F4007018602026012082F8DD609A
:1054500082F8DC5082F8DE5006B0F0BC70476FF482
:10546000806704244FF0200C5F61C2F8E04082F8AE
:10547000DC10C2F8D01082F8DDC0D2F8E020042A97
:105480007FF423AF186840F4007119601DE7D2F86B
:10549000E04082F8DC0044F020052026C2F8E0500D
:1054A000C2F8D00082F8DD60E7E771B1A5F1020C27
:1054B00075781D6102361FFA8CF5BBE7196841F457
:1054C00080771F60D2F8A0305DE706460D46B1E751
:1054D0004FF0200CC2F8D03082F8DC3082F8DDC00A
:1054E000F3E600242023C2F8D04082F8DD30002506
:1054F000D2F8E03082F8DC50E7E600BF400001203F
:105500000000FFFFDC0E01201C6844F400711960EC
:10551000D2F8A0706FF48065042600204FF0200CB4
:105520007D61C2F8E060C2F8D00082F8DDC0D2F838
:10553000E030DCE72023C2F8D07082F8DD30F6E7F7
:1055400070B42D4E2D492E4A2E4D2F4C03463068F7
:1055500018600E68C3F8036003CAC3F80600C3F8F6
:105560000A1003CD128818615961284DDA8103CCE5
:10557000274E284A2C68284D126898613068C3F875
:105580002240D961C3F82500C3F82B2007CD312470
:10559000224DB68883F821404FF03A0C204CA3F8F6
:1055A000296083F820C0C3F82E00C3F832102968A0
:1055B000C3F83B1003CCC3F83620C3F83F00194AA8
:1055C00019482578C3F84310048883F8475003CA64
:1055D000C3F84D10A3F8504093F85010C3F8490099
:1055E0002C26B14283F83A6083F848600CBF502003
:1055F000512070BC704700BF5012030854120308BA
:105600005812030864120308701203087C1203087E
:1056100080120308881203088C1203089C120308E6
:10562000A4120308B0120308B812030808B5094B06
:10563000094A93F8241400F8011B02EB810C7E2226
:10564000DCF8C01D06F0BEF803F07AF90130C0B2F4
:1056500008BD00BF40000120E00001082DE9F0472F
:105660009B4B9C4C08229A6182B0D4F88851FAF77F
:1056700035FE72B6984E9948706362B672B60021D4
:10568000C4F83014C4F8341462B6954F4FF4803324
:105690000222BB61BA61D4F88801D4F888110F1ACC
:1056A000B7F5487F0BD28F4A136923F004011161CB
:1056B00030BFD4F888713B1AB3F5487FF4D394F81F
:1056C000DD00202824D0D4F83826116841F00203E8
:1056D0001360D4F83806076847F001020121026020
:1056E00084F89416FAF7FAFD72B67F4B736362B6CC
:1056F000D4F88861751BB5F5166F3ED3784C7449A4
:1057000004204FF40022A0618A6102B0BDE8F08756
:105710000021764F94F8258400914744D4F89C20CA
:1057200094F8DD0097F8D49D84F89D9E4FF0020A0E
:10573000202884F89C1E84F89CAFC4D1F36A6C4F77
:10574000D4F8A010D808A7FB00031F0A07EB870CAA
:105750000CEB8C00009003E0886910F0020321D06C
:10576000009B5F1E0097002BF6D12027C4F8D03095
:1057700084F8DC3084F8DD70A5E7D4F88801D4F82B
:105780008871C5F5166C3A1A9445B7D955490B6915
:1057900023F004060E6130BFD4F888512F1ABC459F
:1057A000F5D8ABE794F8DC70012F8CD0012784F892
:1057B000DC700868DFF83C91DFF83C81DFF83CC121
:1057C000DFF83CE120F400600860D4F8D410C4F89D
:1057D000C4C04FF0210A102084F8DDA084F8DE0058
:1057E000C4F8E03091F834A00B650220BA45A4F863
:1057F000CA00C1E91133C1E90F93C1F84C80A4F884
:10580000C800C4F8CCE03CD091F8359081F83470F1
:10581000B9F1010FD4F8A070D1F858E04FD1D1F808
:10582000008081F835004B65D8F8003023F48023E0
:10583000C8F800300B68586088680B68402807F18A
:1058400010073FD0C3F808C00868C760C86D3F2381
:105850008340CEF808300F68386840F016033B608C
:105860000F68786940F080037B610F6C27B108688E
:10587000036843F0080707600968086840F00103FF
:105880000B6023215A20FBF771FA28B10020D4F8CD
:10589000E02084F8DC0016E7D4F8A07001907A6963
:1058A0000192B9690191019A7B6843F480727A6030
:1058B000796841F400637B6084F8DC0003E781F8D9
:1058C0003430DEE79F600F68C7F80CC0BEE700BF4A
:1058D0000008024040000120000000207D10000868
:1058E0000000024000ED00E09D1C0008E0000108FF
:1058F00089B5F814693300083D330008DC0E012037
:105900000000FFFF012801D90020704760B901297C
:1059100000D970476C486D4B80F8241099B94FF44A
:1059200080319961012070472DE9F041684C664B48
:1059300094F8DD2083F82510202A82B006D00020BC
:1059400002B0BDE8F081012098617047002000900E
:10595000D4F89C2094F8DD5084F89D1E202D4FF043
:10596000020184F89C0E84F89C1FE8D1DE6A594F2E
:10597000D4F8A010F308A7FB0305280A00EB800861
:1059800008EB8806009603E08B6913F002030CD045
:105990000098471E00970028F6D12022C4F8D000B6
:1059A00084F8DC0084F8DD20CAE794F8DC50012D8F
:1059B000C5D0012584F8DC500868DFF82081DFF8C5
:1059C00020E1454EDFF81CC120F400670F60D4F8D9
:1059D000D410C4F8C4602120102784F8DD0084F8B6
:1059E000DE70C4F8E03091F834700B650220AF42ED
:1059F000A4F8CA00C1E91133C1E90F83C1F84CE032
:105A0000A4F8C800C4F8CCC037D091F8357081F83C
:105A10003450012FD4F8A050D1F858804DD10F68E0
:105A200081F835004B653B6823F480233B600F68A9
:105A3000786088680B68402805F1100540D09E60AA
:105A40000E68F560CF6D3F20B840C8F808000E68BA
:105A5000336843F0160535600F68786940F08006BA
:105A60007E610B6C23B10D682F6847F00800286039
:105A700009680E6846F001030B6023215820FBF7EC
:105A800075F9024628B10020D4F8E03084F8DC0033
:105A900056E7D4F8A05001906F690197A86901906A
:105AA0000199696841F480766E606B6843F4006721
:105AB0006F60012084F8DC2042E781F83430DCE7B5
:105AC0009D600D68EE60BDE7000000200008024008
:105AD0004000012089B5F814DC0E0120693300086C
:105AE0003D3300080000FFFF38B54379022B01D099
:105AF000012038BD81790129FAD8084CC57904EB19
:105B0000C1046279AA42F3D9A368084613F8351094
:105B1000FFF7F8FE0028EBD02571E9E70000002030
:105B20004379012B01D0012070472DE9F0418479A0
:105B3000122C10D8144D154E6700EA19707992F89E
:105B40004C80404515D83D4496F80DC095F84D5011
:105B5000AC4503D834750120BDE8F08133690120DC
:105B600013F83510FFF7CEFE0028F3D035733475E7
:105B7000F1E7B168002011F83810FFF7C3FE0028E4
:105B8000E1D086F80480DEE700BD000800000020B8
:105B90004379012B01D001207047827942B92D4908
:105BA0002D4881F88C214FF4000383610120704758
:105BB0002DE9F041274C284E94F8E85184F88C31B7
:105BC0008027B761002D37D184F8E8311D46A846FB
:105BD0000126224F7979B14224D8787B404514D8E8
:105BE0003D7540F2012C4FF0400800211C4D1D4F27
:105BF000A4F822C7A4F82087C4F80414C4F82457D2
:105C0000C4F81C770120BDE8F0810FFA88F63A69E4
:105C1000012012F83610FFF775FE0028E0D087F853
:105C20000C80DDE7BB68002013F83610FFF76AFE32
:105C30000028D2D03E71D0E7112D07D80A4A02EBD6
:105C4000450898F84C6098F84D80C2E7112584F813
:105C5000E851BCE7400001200000024000000020A5
:105C6000DB1B0400B9A2010000BD00082DE9F043D0
:105C7000BA4B082283B09A6172B6B94C0020C4F8BE
:105C8000FC01C4F8000262B694F89416002900F0F2
:105C9000E780D4F88861D4F88851D4F88831591B4A
:105CA00063290AD8AF4A106920F00407176130BF92
:105CB000D4F88831591B6329F5D9A84DAA4F4FF460
:105CC00000204FF48022A861BA61D4F88811D4F87A
:105CD00088315D1A632D0AD8A24F386920F004027A
:105CE0003A6130BFD4F888315D1A632DF5D99E49E9
:105CF00001278F61D4F88801D4F88821131AB3F5ED
:105D0000C87F0BD2974D296921F004072F6130BF5E
:105D1000D4F88821131AB3F5C87FF4D394F88C0112
:105D2000924D70B929796F798F4200F21081287BEA
:105D30006B7B834205D9296911F830100120FFF7E8
:105D4000E1FD8948854F08224FF400334FF480214C
:105D5000BA6183610027816184F89476FAF7BEFA0C
:105D600072B68348686362B6824A8349834BC4F83B
:105D700068164FF080679761C4F87036D4F89C308D
:105D8000D4F83836D4F89C1005E0D4F89C00471AB3
:105D9000642F00F2948098688207F6D50022DA60BA
:105DA0000192D96801919F680197019A586840F063
:105DB00040025A60196841F040071F60D4F88831EA
:105DC0009E1BB6F5166FC0F08E8094F88C0170B3F0
:105DD00094F8E861002E40F0A8804FF0010984F8A3
:105DE000E89194F8E861664F95F805C04FEA4609D6
:105DF00007EB090E9EF84C80C44500F28A804F44A0
:105E00006A7B97F84D70BA4200F2968040F2012CFE
:105E1000402000272E755B4B5B4EA4F822C7A4F8E8
:105E20002007C4F80474C4F82467C4F81C37D4F8F5
:105E30003826116841F002001060D4F8384627680F
:105E400027F001062660FAF749FA72B64F4B6B63EA
:105E500062B6424D4FF40022AA6103B0BDE8F08360
:105E6000414D4FF480260127AE61AF61D4F888011F
:105E7000D4F888311A1AB2F5C87F0BD239490D69A6
:105E800025F004060E6130BFD4F888713B1AB3F5D3
:105E9000C87FF4D394F88C01344D002898D1297927
:105EA00095F80580884518D82E7B687BB042BED90E
:105EB0002F69012017F83610FFF724FDB7E72A4BAA
:105EC00008254FF40064402680214FF480529D61E4
:105ED0009C619E6199619A61FEE7AA6812F831108F
:105EE000FFF710FDE0E7D4F88801D4F88821C6F563
:105EF0001667111A8F427FF668AF1A4B1E6926F09B
:105F000004021A6130BFD4F888110E1AB742F5D8CE
:105F10005BE7AB68002013F83810FFF7F3FC0028AC
:105F20003FF46DAF85F8048069E7112E7FF65BAF13
:105F3000112784F8E87154E72969012011F8371016
:105F4000FFF7E0FC00283FF461AF2F735EE7AA681B
:105F500012F83110FFF7D6FCE9E600BF0008024056
:105F60004000012000ED00E00000024000000020A1
:105F70007D100008000402408EBD0008D2060120FA
:105F800000BD0008B9A20100DB1B0400611E00086F
:105F90002DE9F04FDFF854A2904ABAF89031044648
:105FA0004FF400619DB0916101334FF4897200217B
:105FB0000AF54E60AAF8903105F0BAFBFFF74EFBE8
:105FC0002068A5880C900020ADF834500CAEAAF8DB
:105FD0009E0F0DF1360916F8017B7840420010F053
:105FE000800F18BF82F09702D3B2590013F0800FD0
:105FF00018BF81F09701C8B2450010F0800F18BF9C
:1060000085F09705EFB27A0017F0800F18BF82F085
:106010009702D3B2590013F0800F18BF81F0970197
:10602000C8B210F0800F4FEA400518BF85F0970501
:10603000EFB217F0800F4FEA470218BF82F09702C5
:10604000D3B213F0800F4FEA430118BF81F09701DC
:106050004E45C8B2BFD100210DF1520C9DF8305011
:106060008DF83600CDE91511CDE91711CDE91911DB
:106070001B9166460DF16E0B4FF0800E21E02F4014
:10608000FAB25800002A18BF40F00100CEF387078B
:1060900083B2002F40F07E820131C9B206296DD84B
:1060A0001CAF0F4417F8405CC5F3C01343EA400827
:1060B000C5F3801242EA48004FF0200E5E45308062
:1060C00037D005EA0E075FFA87F818F10003CEF320
:1060D000470706F1020618BF0123002FCFD1013177
:1060E000C9B2062903D81CAD0D4415F8407CC7F38E
:1060F000C01040EA4302C7F3801E4EEA42034FF04D
:10610000200817EA080F4FEA430018BF40F00100CB
:106110005FEA580540F05F820131C9B206294FF0AD
:10612000800ECBD81CAD0D445E4515F8405C308028
:10613000C7D10021CDE90E11CDE91011CDE9121121
:10614000274814913CF8025F264A0D274FF0000EB5
:106150002F4007F00F0399B23BB14FF0000B81EADB
:106160000B0B4908FBD10BF0010343EA4E079042A9
:106170001FFA87FE04D032F8027FE9E73D4693E735
:10618000B44529F802EFDDD1BDF83A00BDF84C2046
:10619000BDF84E10BDF83860BDF85030079004923D
:1061A000BDF84800BDF852200391082108960293DB
:1061B00001920691BDF83C80BDF83EE0BDF840C0BC
:1061C000BDF84270BDF84460BDF84650BDF84AB015
:1061D000054B0590002280210994A3E000000240B5
:1061E00016BD000808BD0008200D01204000012058
:1061F0001878079C4FEA4009901C2142C4B218BF8E
:1062000049F00109082C83F8009040F0E7815C78A0
:1062100011EA080F14BF0122002242EA440211EAE7
:106220000E0FD0B214BF0124002444EA40045C7075
:10623000022201331C78013211EA0C0F4FEA4400AC
:10624000D2B218BF40F00100082A187040F0E78170
:1062500058780F4214BF0122002242EA40020E4247
:10626000D4B214BF0120002040EA4400587002223A
:106270000133187801320D424FEA4004D2B218BF00
:1062800044F00104082A1C7040F0E7815A78059810
:106290005200084218BF42F0010211EA0B0FD0B2BF
:1062A00014BF0124002444EA40045C70022201333C
:1062B0001C780498013201424FEA4404D2B218BF5C
:1062C00044F00104082A1C7040F0E88103985A78D1
:1062D000014202984FEA420218BF42F00102014215
:1062E000D2B214BF0124002444EA42045C700222AA
:1062F000013301981C78084202F1010214BF4FF0EB
:1063000001094FF00009D2B249EA4400082A187086
:1063100001D1013300220698441E4FEA5101069430
:1063200000F0A3801878089C4FEA4009501C2142D5
:10633000C4B218BF49F00109082C83F800907FF41B
:1063400057AF079A5878114214BF0122002242EA3F
:10635000400411EA080FE2B214BF0120002040EA15
:1063600042005870022201331C78013211EA0E0FEC
:106370004FEA4400D2B218BF40F00100082A18705A
:106380007FF458AF5C7811EA0C0F14BF0122002291
:1063900042EA44020F42D0B214BF0124002444EA6E
:1063A00040045C7002220133187801320E424FEA39
:1063B0004004D2B218BF44F00104082A1C707FF4D4
:1063C00058AF5C7805980D4214BF0122002242EAC2
:1063D00044020842D2B214BF0124002444EA420419
:1063E0005C70022201331878013211EA0B0F4FEA78
:1063F0004004D2B218BF44F00104082A1C707FF494
:1064000057AF04985A78039C014214BF0120002022
:1064100040EA42002142C2B214BF0124002444EAEF
:1064200042005870022201331C7802980132014266
:106430004FEA4404D2B218BF44F00104082A1C7089
:106440007FF457AF019A93F8019006980A4214BF5F
:106450000122002242EA49045C700122441E1344D6
:106460004FEA510106947FF45DAF099EB5787379C8
:106470007F2D00F09181002B40F072810024C049F3
:10648000CA69487D92F800B0557807905C44671E51
:1064900097FBFBFC15FB0CF37033AAF89E3F00281A
:1064A00000F096810021B748B74C0594CDE9021160
:1064B000A0F1E802B54DB64C049101928B46894695
:1064C0004FF0200E01274FF0800806909AF824C460
:1064D0000198CCEBCC03C3EBC3063744764400EB06
:1064E000460200EB4701B1F9AC0DB2F9AC1D0991C0
:1064F0000E460644C317F717990332463B4641EA56
:106500009041800301F0AEFF08900998C3179903EA
:1065100032463B4641EA9041800301F0A3FFDDE9AA
:106520000527089E07F2FE3C00FB0BFB06FB09B3A8
:106530009B130FFA83F9B9F5804FC0F2D7804FF65D
:10654000FF7E06E0C5F81880216921F0040323616D
:1065500030BFDAF83034DAF834145B1AB3F5807FE0
:10656000F0D0DAF83014CBB204330AEB430B6745B2
:10657000ABF830E4DAF830144FF4000301F1010114
:10658000CAF83014AB6100F0BE8037F9029F32F9CF
:1065900002BFC9E74FEA43083D420CBF474648F0F7
:1065A0000107CEF3C708BBB2B8F1000F11D101311A
:1065B000C9B206290BD80DF1700E8E441EF8405C4E
:1065C000C5F3C01242EA47004FF0400E76E545465B
:1065D000F6E72F4695E5AE463D466FE5187803325F
:1065E00011EA080F4FEA4004D2B218BF44F0010488
:1065F000082A1C707FF4B8AE587811EA0E0F14BF49
:106600000122002242EA400411EA0C0FE2B214BF58
:106610000120002040EA42005870022201331C7819
:1066200001320F424FEA4400D2B218BF40F00100DD
:10663000082A18707FF4B8AE5C780E4214BF0122AD
:10664000002242EA44000D42C2B214BF01240024D9
:1066500044EA42045C70022201331C78059801323E
:1066600008424FEA4404D2B218BF44F00104082A99
:106670001C707FF4B8AE5878049C11EA0B0F14BF5D
:106680000122002242EA40022142D0B214BF01247A
:10669000002444EA40025A700222013303981C7815
:1066A000014202F1010214BF4FF001094FF000094D
:1066B000D2B249EA4400082A18707FF4B5AE029AB3
:1066C00093F801900198114214BF0122002242EA7E
:1066D00049040842E2B214BF4FF001094FF000092B
:1066E00049EA42045C700222013314E619F5804F36
:1066F00006DB03F580418BB259001FFA81FE28E7C3
:106700004FF0000E25E7029838B3039F002187F071
:10671000010603960291049B079A0133D8B2824284
:10672000049357D91B4B0299039A03EB810C019BED
:10673000DCF8A460B018B75C90F802E003EB870BBC
:1067400003EB8E09DBF8E81CD9F8E86C0691059696
:10675000B1F90090B6F900B0B8E601220292DAE78A
:106760003046FDF725FF7679002E3FF487AE0C2EDC
:106770008CBF4FF002084FF001084644F4007EE65B
:1067800000000020C0120108C00E010800080240ED
:1067900000ED00E000BD0008002B3FF46FAE304676
:1067A000DAF88871FDF704FFD6F80620DAF88831A8
:1067B0006049C7EB430014BA051B0023A5FB010188
:1067C0005D4A01F09FFE07BAC6F80670737952E67B
:1067D0005A4E01965A4F5B4D5B4C05974FF0000B9C
:1067E0006FF42B666FF4D663CDE902BBB919F818C4
:1067F0000491D94613224FF00E0E4FF080080690F8
:106800009AF824740199C7EBC706C6EBC60CE64498
:10681000944401EB4C0201EB4E0EB2F9AC1DBEF9F3
:10682000AC0D08910E460644C217F71791033B467C
:10683000324641EA9041800301F014FE0790089827
:10684000C317990332463B4641EA9041800301F069
:1068500009FE069F049A079E07F2FE3C00FB09F919
:1068600006FB0B939B130FFA83FBBBF5804F29DBD1
:106870004FF6FF7E06E0C5F81880216921F0040379
:10688000236130BFDAF83034DAF834145B1AB3F528
:10689000807FF0D0DAF83014CBB204330AEB43092E
:1068A000BC45A9F830E4DAF830144FF4000301F1E4
:1068B0000101CAF83014AB6111D037F902BF32F9C7
:1068C000029FCBE71BF5804F06DB03F580418BB2BF
:1068D00059001FFA81FED5E74FF0000ED2E702986B
:1068E000002837D0039E1948059B86F00107002138
:1068F00098420397029133D013F8010B144E05937D
:1069000006EB800C039BDCF8A470019E17F803E0F3
:10691000F91806EB8E0B8A78DBF8E80C069006EB8C
:106920008209B0F900B0D9F8E87C0497B7F9009073
:1069300066E700BF40420F00400D0300D811010878
:10694000712101080008024000ED00E074210108F7
:1069500000BD00088F48059B012298420292CBD1CE
:106960008D4CBAF89E2F2578069500268027DFF8F3
:1069700038828A4D8A4C049602970396BB46039947
:10698000914280F04C81029898F800703842844619
:1069900014BF4FF0010C4FF0000C5FEA500E8DF861
:1069A00030C040F0998198F80160F709C6F380196A
:1069B0008DF8317008F101088DF83290202798F891
:1069C00000301F4214BF0123002378088DF83330B4
:1069D000029003D1802108F101080291039E069BD9
:1069E0000436B7B20397002BC9D000220792CDF826
:1069F0002C80019B9DF830C0049E9DF83190694920
:106A00009AF82404059003EB8C078A1903EB890993
:106A1000D7F89C0F92F8841008901E46D9F89C3F36
:106A200009939DF83280089B92F887C09DF833E067
:106A300092F8789092F88A7092F88D0001EB4101FB
:106A4000194406EB8808099B0CEB4C0C06EB8E0EE8
:106A50006344D8F89C6F92F87B800A9611F809C0BD
:106A6000DEF89C6F13F8081092F87E9092F881E09F
:106A7000059B07EB47020A9F00EB4000BA18C3EBE7
:106A8000C307C7EBC7033044019E12F8092010F872
:106A90000E8003EB0C095F1806EB490006EB470775
:106AA00006EB8101B0F9AC0DB7F9AC7D059703EBAE
:106AB000020E06EB4E0E06EB8C0C03EB0809D1F828
:106AC000E81C0F9106EB880806EB82020599BEF9D7
:106AD000AC7DDCF8E83C0E9306EB4906D8F8E83CC0
:106AE000B6F9AC6D119301EB0008B844B044C3177C
:106AF0004FEAE879D2F8E82C1092990342464B46C7
:106B000041EA9041800301F0ADFC05991590CB1747
:106B100005984FEA833C4CEA904142464B4680033D
:106B200001F0A0FCFB179903169042464B4641EA40
:106B30009741B80301F096FCF2179103179041EAD0
:106B40009641B00342464B4601F08CFC002718905A
:106B50004FF40006DDE90EE8109B3EF90700159999
:106B6000DA5F38F90790169B01FB00F103FB091C63
:106B70001199179831F907E0189B00FB02C803FB35
:106B80000E82911308B2B0F5804FC0F29A804FF692
:106B9000FF7012E07421010800000020000802408C
:106BA00000ED00E0F8CD0008200D0120C5F818B078
:106BB000236923F00402226130BFDAF83034DAF8B6
:106BC0003424991AB1F5807FF0D0DAF83014CBB2C2
:106BD00004330AEB43090237A9F83004DAF8300429
:106BE000B7F5806F00F10100CAF83004AE61B1D191
:106BF000049E079A069B0136F7B20132032FD1B2E9
:106C000008BF00278B42079204973FF6F2AEBAF80E
:106C10009E2F0399DDF82C809142FFF4B4AEDAF890
:106C20003004DAF83424831AB3F5807F10D1414E52
:106C3000414F8024B4613D6925F00401396130BFC2
:106C4000DAF83004DAF83424831AB3F5807FF1D00F
:106C5000DAF83064374FF4B204340AEB440B4FF4E3
:106C60000045ABF83054DAF830044FF4000101303D
:106C7000CAF83004B961DAF83024DAF834349A42C8
:106C80000DD02D4E1025BD61346924F00400306113
:106C900030BFDAF83014DAF834249142F3D1254FBA
:106CA000264E4FF48013BB614FF00065DAF888413F
:106CB000B561CAF8984EFEF7D9FF01201DB0BDE8B6
:106CC000F08F10F5804F05DB01F580439AB251003B
:106CD00088B272E7002070E702991EEA070F14BF1E
:106CE0004FF0010E4FF0000E8E088DF831E00DD1FF
:106CF00098F801302021DF09C3F3801008F1010862
:106D00008DF832708DF83300029167E63E42029BA7
:106D100014BF012700278DF83270DF087FF44FAED3
:106D200098F801004026C1098DF8331008F10108D8
:106D3000029653E60008024000ED00E00000024029
:106D40002DE9F04FC379ADF20C4D8346002B40F096
:106D5000F48001221346C27115469BF8080010B951
:106D600001218BF808109BF80660754C002E40F04E
:106D7000D080312797FBF3F29303DFF8D491CDF85D
:106D800000B00DF1060E1F46DB17019409F2FE3A22
:106D9000A9F6A4760022F3464C469846A4EB090CCB
:106DA0002B46002005E0D1F8E81C2B4431F90C20DB
:106DB0009BB2302B06EB83011044F4D9C31799031F
:106DC00041EA90413A468003434601F04BFBA2451D
:106DD0002BF8020F02D034F9022FDFE7DDE900AB18
:106DE000FEF73CFC9AF80850002D48D0554C564808
:106DF0004FF000080DF2064180260DF1060C4FF40D
:106E000000093CF902EFBEF5804F7DDA1EF5804F98
:106E10007DDB0EF58047BAB253009DB2DBF83074CB
:106E2000DBF834E4A7EB0E02B2F5807F0DD1A6614A
:106E3000036923F00407076130BFDBF83024DBF877
:106E40003434D71AB7F5807FF1D0DBF83024D3B2D1
:106E500004330BEB430E8C45AEF83054DBF8305462
:106E600005F10105CBF83054C4F81890C9D108F1E8
:106E700001079AF808201FFA87F84245BDD8DBF8C9
:106E80003044DBF83404211AB1F5807F10D12D4E47
:106E90002D4D8027B7612B6923F004022A6130BF92
:106EA000DBF83044DBF83404211AB1F5807FF1D0EF
:106EB000DBF83064234DF7B204370BEB470A4FF48D
:106EC0000043AAF83034DBF830244FF400040132D8
:106ED000CBF83024AC61DBF83004DBF834148142A9
:106EE00007D01026AE61DBF83074DBF834349F42F3
:106EF000F8D1144D4FF48012AA61FEF7B7FE0120BD
:106F00000DF20C4DBDE8F08F4FF6FF7586E70025BA
:106F100084E794F824040D4EC0EBC0010023C1EBBC
:106F2000C10718463A1806EB42082844B8F9AC9D48
:106F300080B230284B44F5D91FE79DB20DE700BF62
:106F4000400001200008024000ED00E0D8110108D7
:106F50007C2101084379032B01D000207047EFE624
:106F60004379012B01D0002070472DE9F047DFF86D
:106F700070818279554808FB02F1A0FB0134A50914
:106F800005F580764FEA5628B8F1030F4CD84FF03C
:106F90000408FEF763FBDFF84CA14D4A4D484E490B
:106FA0004FF0000E80254FF00009B9F5804F4B4E91
:106FB0004FF4000C35DA19F5804F3BDB09F58043BF
:106FC0009CB26700BCB2D2F83034D2F83494A3EB50
:106FD0000907B7F5807F0DD185610B6923F00407A0
:106FE0000F6130BFD2F83034D2F83474DB1BB3F504
:106FF000807FF1D0D2F83074FBB2043302EB430946
:107000005645A9F83044D2F8304404F10104C2F8DE
:107010003044C0F818C00FD036F9029FB9F5804F40
:10702000C9DB4FF6FF74CEE740F2D137B84528BF31
:10703000B846AEE70024C6E70EF1010E1FFA8EF641
:10704000B045B0D8D2F83004D2F83414451AB5F5AA
:10705000807F10D11F4F204C8026BE61236923F012
:107060000400206130BFD2F83014D2F834544B1BE6
:10707000B3F5807FF1D0D2F83074164EFCB20434F0
:1070800002EB440A4FF40048AAF83084D2F83014D6
:107090004FF400000131C2F83014B061D2F830541E
:1070A000D2F834349D4207D01027B761D2F830446B
:1070B000D2F834148C42F8D1064E4FF48012B261EB
:1070C000FEF7D4FD0120BDE8F08700BFD34D62106C
:1070D000400001200008024000ED00E07C2501088E
:1070E00080841E007A2901082DE9F84F4379022B8C
:1070F00002D00020BDE8F88F594F8346FEF7AEFA64
:10710000584A59485949A7F6E8484FF0000E8024DC
:1071100000254FF4000C3E689BF80690735FB9F1B0
:10712000000F40F08980B3F5804F80F2828013F524
:10713000804FC0F2918003F58046B3B25E001FFA23
:1071400086F9D2F83034D2F834A4A3EB0A06B6F5A7
:10715000807F0DD184610B6923F004060E6130BF7E
:10716000D2F83034D2F834649B1BB3F5807FF1D071
:10717000D2F83064F3B2043302EB430A0235AAF8C2
:107180003094D2F83064B5F5806F06F10106C2F88C
:107190003064C0F818C0BED19BF8075055B3002624
:1071A0004FF400454FF4000C05E084610B6923F0B7
:1071B00004030B6130BFD2F83034D2F83494A3EB1F
:1071C000090ABAF5807FF0D0D2F83034DBB204334C
:1071D00002EB43090136A9F83054D2F830340133B8
:1071E000C2F83034C0F818C09BF807A0B6B2B6EBAE
:1071F0004A2FE0DB0EF1010EBEF1310F07F104075B
:1072000086D1D2F83064D2F83454AE4208D0164950
:1072100010278F61D2F83044D2F834048442F8D178
:10722000114B4FF480129A61FEF720FD0120BDE85A
:10723000F88F4FF6FF7984E792F82464C6EBC60610
:10724000C6EBC60AF24408EB4A09B9F8AC6D16FB66
:1072500003F343F38F3366E74FF0000971E700BF94
:10726000C01E0108400001200008024000ED00E0BF
:107270004379022B01D0002070472DE9F041857938
:10728000302D00F2A580C079002800F08E8064289F
:1072900000F2A180524A534E534C8103A2FB0137A6
:1072A0004FEA571806EB8506FEF7D8F94F4D504ABE
:1072B000D6F8E8EC002780264FF4000C3EF90710C2
:1072C00008FB01F3981301B2B1F5804F7BDA11F599
:1072D000804F7BDB00F5804398B2410088B205E027
:1072E000AE61116921F00403136130BFD4F830346A
:1072F000D4F834145B1AB3F5807FF1D0D4F830148D
:10730000CBB2043304EB43010237A1F83004D4F8C4
:107310003004B7F5806F00F10100C4F83004C5F8FF
:1073200018C0CBD1D4F83054D4F83424AF1AB7F500
:10733000807F10D12D4E2E4D8020B0612B6923F01F
:107340000401296130BFD4F83024D4F83474D31B3D
:10735000B3F5807FF1D0D4F83064244DF0B204301E
:1073600004EB40084FF40041A8F83014D4F830740E
:107370004FF400020137C4F83074AA61D4F83064C5
:10738000D4F834349E4207D01020A861D4F83014C9
:10739000D4F83474B942F8D1144C4FF48015A56177
:1073A000FEF764FC0120BDE8F0810F4C0D4E94F80F
:1073B00024C4CCEBCC0ECEEBCE032B4406EB430027
:1073C000B0F9AC8D6EE74FF6FF708FE700208DE7C8
:1073D0000020BDE8F081034E034C4FF4804861E784
:1073E0001F85EB51D8110108400001200008024020
:1073F00000ED00E04379022B01D001207047827933
:10740000012AFAD8C17952B90129F6D86A4B6B48DA
:1074100083F8241091B94FF480328261EDE72DE9B1
:10742000F041674C644894F8DD5080F82510202D19
:1074300082B006D0012002B0BDE8F0810121816157
:10744000DBE700260096D4F89C2094F8DD7084F8E1
:107450009C3F202F84F89D1E84F89C6EEAD1C36A5D
:107460005849D4F8A000DD08A1FB0516370A07EB40
:10747000870808EB8803009303E0866916F002038F
:107480000CD0009D691E0091002DF6D12026C4F875
:10749000D05084F8DC5084F8DD60CBE794F8DC70E1
:1074A000012FC7D0012684F8DC600168DFF81C8159
:1074B000DFF81CE1444DDFF81CC121F400670760D0
:1074C000D4F8D410C4F8C4502120102784F8DD006B
:1074D00084F8DE70C4F8E03091F834700B65022057
:1074E000B742A4F8CA00C1E91133C1E90F83C1F85A
:1074F0004CE0A4F8C800C4F8CCC037D091F835707F
:1075000081F83460012FD4F8A060D1F858804BD1B5
:107510000F6881F835004B653B6823F480233B609E
:107520000F68786088680B68402806F110063ED026
:107530009D600D68EE60CF6D3F20B840C8F8080030
:107540000D682B6843F016062E600F68786940F0CE
:1075500080057D610B6C23B10E68376847F0080029
:10756000306009680D6845F001030B602321582045
:10757000F9F7FCFB28B10020D4F8E02084F8DC0007
:1075800058E7D4F8A060019072690192B769019739
:10759000019A716841F480757560736843F4006204
:1075A000726084F8DC0045E781F83430DEE79E60E5
:1075B0000E68F560BFE700BF000000200008024031
:1075C0004000012089B5F814DC0E01206933000861
:1075D0003D3300080000FFFF2DE9F04F99B0002770
:1075E000DFF85CB30597DBF83010DFF858A3CE4E18
:1075F000CE4C41F00100CBF83000DBF8302002F037
:107600000103059305990497DBF8305045F002011A
:10761000CBF83010DBF8300000F00202049204993D
:107620000397DBF8303043F00405CBF8305018AD49
:10763000DBF8301015974FF0010845F8148D01F074
:107640000400039029465046039B1697CDF85080BE
:10765000F8F7DEFE4FF48032CAF8182002231393A5
:107660000193F8F7D5FE4FF40032CAF8182004232E
:107670001393F8F7CDFE4FF48020CAF818004FF4AA
:1076800000624FF0006930461392CDE914871697D7
:10769000F8F7BEFE5046C6F8189008231393CDE9BC
:1076A00014871697F8F7B4FE4FF40022CAF8182092
:1076B0004FF400631393F8F7ABFECAF8189040221A
:1076C0001392F8F7A5FE4FF48003CAF81830802211
:1076D0001392F8F79DFE4FF40003CAF818304FF4E8
:1076E00080521392F8F794FE4FF08053CAF8183086
:1076F0004FF01009CDF84C90F8F78AFE8C4ACAF882
:1077000018904FF4807CCDE913C2CDE91577F8F7D6
:107710007FFE3A4639461720F8F770FF0297DBF8EC
:10772000301041F00400CBF83000DBF83030CDF8F9
:10773000508003F00402304629464FF480630292E1
:10774000DDF808C01393CDE915781797F8F760FEB8
:10775000019A1392F8F75CFE04231393F8F758FE8E
:1077600008221392F8F754FECDF84C90F8F750FE2B
:1077700020231393F8F74CFE40221392F8F748FEAB
:1077800080231393F8F744FE4FF480721392F8F7B6
:107790003FFE4FF400731393F8F73AFE4FF40033B3
:1077A0004FF0806EC6F818E0B3614FF48023B361E8
:1077B0004FF400104FF400234FF4801AB3614FF0E0
:1077C0000072C6F818A04FF08071B0614FF400034A
:1077D0004FF48000B061B361B161B26194F83920B7
:1077E000276111264FF018094FF08040C4E9027656
:1077F000C4E90009002A00F0CF834E4F4E494FF0F4
:107800000208012684F83980F8F7FAFC4AF6C870B5
:107810004FF4FA7384F83960C4F84886B862FB62A2
:10782000FE604FF482733E60082094F88926C4F805
:107830003C3600234149C4F85406C4F840360720BA
:10784000C4F84C36C4F86036C4F85836C4F85C3610
:107850004FF4007B4FF40063C4F8381602F0FF07C2
:10786000C4F86406C4F84436C4F850B6002A00F0E0
:1078700014830E464FF0020C84F889C63068DFF896
:10788000C8E020F040033360D4F84076D4F83C36AA
:10789000D4F84466D4F84806D4F84C26D4F85416E4
:1078A0003B431E433043D4F85836D4F86066D4F8CE
:1078B0005076104301431943314307F40070D4F864
:1078C000382608431060B4F85276D4F85C16D4F821
:1078D0003866C4F828E707F004030B437360F069C7
:1078E000002320F400620127F261C4F88C3684F88A
:1078F000897694F86127C4F830374FF4E1300C21D1
:10790000C4F83437C4F83837C4F84037C4F84437BB
:1079100002F0FF06C4F82C07C4F83C17002A00F058
:1079200072821F4612E000BF0008024040000120A2
:107930000000111000040040440001200038004005
:107940000038024000000240001001404FF0240BBC
:1079500084F861B7DEF80C3023F40052CEF80C2026
:10796000DEF81000D4F8346720F440513143CEF8EB
:107970001010D4F83C27D4F83837D4F84407DEF890
:107980000C601343034326F4164A3B432AF00C07CA
:107990003B43CEF80C30DEF81410D4F8402721F425
:1079A00040731343CEF81430D4F84407B0F5004FB9
:1079B00000F0CE81CE4EB64500F0628106F58067BC
:1079C000BE4500F05D81FBF7A9FED4F82C174FF0FF
:1079D00019098B004FF0640809FB00F2B2FBF3F0C9
:1079E000B0FBF8F6FBF79AFED4F82C7709FB00F110
:1079F000BA00B1FBF2FBFBF791FED4F82C3709FB80
:107A000000FC9800BCFBF0F7B7FBF8F108FB11B2E3
:107A100013013233B3FBF8F000F0F007FBF77EFE02
:107A2000D4F82C1709FB00F38A003601B3FBF2FAF5
:107A3000FBF774FED4F82C1709FB00FE8800BEFB90
:107A4000F0F9B9FBF8FC08FB1CA31A013232B2FBB7
:107A5000F8F101F00F003843D4F828773044B860CB
:107A6000D4F82877A34E3869A34AC4F8A46020F458
:107A7000904139617B69C4F8A02023F02A00786125
:107A8000FB68002143F400504FF02009F860C4F86F
:107A9000641784F8619784F8629794F8DD30C4F82D
:107AA000B4104FF480405E26FE27C4E92F1103F086
:107AB000FF08C4F8B000C4F8A800C4F8AC60C4F86B
:107AC000B870002B00F09A8211464FF0240B84F816
:107AD000DDB00A68894F8A4E22F001030B60FBF784
:107AE0001DFED4F8A010A7FB0032920C4A60D4F817
:107AF000A430B34200F212815E00B0FBF6F3C3F390
:107B00000B00013203280A6298BF0423CB61D4E939
:107B10002F7217430F60D4E92B61D4F8A070794B12
:107B20003143B960D4E92D200243FA603E687648BB
:107B300046F0010139604FF0200A0027C4F8E070D8
:107B400084F8DDA0C4F8D07084F8DE70D4F8BC6787
:107B5000C4F88477C4F88C77C4F89477C4F89C7719
:107B6000C4F8A877C4F88877C4F8AC774FF48032AB
:107B70000127C4F87C37C4F88027C4F8A407C4F8E8
:107B80009077002E00F0D182D4F8BC77FA0640F14D
:107B9000458200270125109784F8B8571E695B4A73
:107BA000C4F8A45F26F0E0611961186940F000761E
:107BB0001E61596B21F01F0058635E6B46F008018F
:107BC00059634FF40060082393614026906180213F
:107BD0004FF4805096619161906194F8DD2084F8B3
:107BE000B877202A4FF00207C4F8A03FC4F8A87F56
:107BF00000F0D082464D2846FF270025012184F859
:107C00002F5484F82C74F9F797F9A4F82D043F4EFB
:107C10004FF480024FF00063B261B361F8F75EFB8E
:107C200072B63C483C49416362B64FF480354FF42C
:107C300000374FF480220023B56184F82534B76102
:107C400084F89436B261B561B761B26172B6C4F8B6
:107C50003034C4F8343462B672B6C4F8FC31C4F8B7
:107C6000003262B6FEF702F84FF400244FF4000031
:107C70004FF08051B461B061B16119B0BDE8F08FCF
:107C8000FBF790FED4F82C674FF019094FF0640809
:107C900009FB00F0B700B0FBF7F1B1FBF8F31E01F0
:107CA000FBF780FED4F82C2709FB00FB9000BBFB00
:107CB000F0FAFBF777FED4F82C7709FB00F1BB0054
:107CC000B1FBF3F2B2FBF8F008FB10A73901323137
:107CD000B1FBF8FC0CF0F007FBF764FED4F82C378E
:107CE00009FB00FB9A00BBFBF2FAFBF75BFEA1E687
:107CF00000100140801A06000054004083DE1B4340
:107D0000A0860100002001400100000F0000024099
:107D10006F040120000000207D1000084FF49677CA
:107D2000D4F8A86007FB02F24FF47A7CB2FBFCF2B5
:107D300001320A62002E40F0208203EB4306B0FBC2
:107D4000F6F7C7F30B02002A40F0C3820123DDE6F9
:107D500000F1804808F51046B64500F0818206F52E
:107D6000806AD64500F07C82FBF7D8FCD4F82C273B
:107D7000192653004FF0640906FB00FBBBFBF3F12F
:107D8000B1FBF9F04FEA0018FBF7C8FCD4F82C77E8
:107D900006FB00F07A00B0FBF2FAFBF7BFFCD4F868
:107DA0002C3706FB00F05900B0FBF1F0B0FBF9F7FF
:107DB00009FB17A2D3003233B3FBF9F1480000F4FA
:107DC000F87BFBF7ABFCD4F82C7706FB00F07A00CD
:107DD000B0FBF2F7FBF7A2FCD4F82C3706FB00F05F
:107DE0005E00B0FBF6F2B2FBF9F009FB1077F90088
:107DF0003231B1FBF9FE0EF007034344D4F8286793
:107E00005B44B3602CE6814B0F961A6B84F8606775
:107E10003A431A63196B7E4839400F910F9A0E96B8
:107E20001A6B3A431A63196B39400E910E9A0D96EC
:107E30005A6C42F0100159645B6CCDF850C003F0ED
:107E4000100229464FF400730D924FF00708CDE958
:107E5000156713930D9ACDF85C804FF48069F8F79D
:107E6000D7FA12226A48CDF85C80CDE91567CDE9D2
:107E70001392F8F7CDFA324603212520F8F7BEFB1E
:107E80006448D4F828E7D4F8307720264660DEF836
:107E90000C103143CEF80C1058E55C490C970A6B76
:107EA00084F8887642EA080008630B6BDFF8689173
:107EB00003EA08020C920C9A0B97086B40EA08033D
:107EC0000B630A6B02EA08000B900B9A0A970B6B84
:107ED00043EA08020A63086B00EA08030A930A9A55
:107EE00009970A6B42EA080008630B6B03EA080271
:107EF0000992099A0897086C40F480430B64096C56
:107F0000CDF84CB001F48042089229464846089BBF
:107F1000CDE914671696F8F77BFA4FF48063C9F839
:107F200018B013930193F8F773FA0198C9F8180081
:107F30004FF4805B48464FF0050ACDF84CB0F8F797
:107F400067FAC9F818B04FF400521392CDE91487BC
:107F50001696CDF85CA0F8F75BFA4FF40043139344
:107F6000CDE914871696CDF85CA0F8F751FA4FF4D6
:107F70008042CDE9148716961392CDF85CA0F8F7ED
:107F800047FA39463A462420224FF8F737FB1021AA
:107F9000D4F8386679606DE402F0FF060796DBF8E6
:107FA000407084F8386047EA0801CBF84010DBF8ED
:107FB0004000184F00EA08033246079341461C2050
:107FC000079BF8F71BFB4FF080523A600696DBF8F0
:107FD000406046F00201CBF84010DBF8400000F0B2
:107FE0000203424606931D200921069BF8F706FB73
:107FF0004FF000523A602068FFF7FFBB84F8DC8046
:10800000F8F72EFBD4F8A0105FE500BF003802405F
:108010000000024000E100E000040240D4F8BC2768
:10802000BE49D4F88057BE4822F4885626F002078D
:1080300047F00202C4F8BC274E6826F440374F6070
:108040004A682A434A60596821F480755D605E6819
:10805000D4F88C7746EA07225A60596821F04075B7
:108060005D605E68D4F884773E435E609A6822F46F
:10807000006199609D68D4F8886735439D60D4F8A5
:10808000A4778742986820F070629A609D6800F03B
:108090002381D4F8A46735439D609F6827F0405042
:1080A00098609A68D4F8A8572A439A60996821F092
:1080B00002069E609F68D4F8940747EA40029A60DF
:1080C000D4F89C57002D40F0B580596821F4006623
:1080D0005E60DA6AD4F8985722F47006DE62DF6ACE
:1080E00005F1FF3B47EA0B51D962986820F4007212
:1080F0009A609D68D4F8AC6745EA46279F60996806
:1081000021F4806098609A68D4F89057002642EA7B
:1081100085279F60C4F8C067D4F8BC1721F003001E
:1081200040F00102C4F8BC2733E503F58C3EC4F8E7
:10813000C0671196DEF8443084F8B86743F4807065
:10814000CEF84400DEF844107648139701F48072AC
:10815000119203232946119D734D1493CDE91567A0
:10816000F8F756F93246092112204FF48026F8F725
:1081700045FAD4F87C372E6006E5192707FB03F390
:10818000B0FBF3F0C0F30B03002B3FF4DFAD40F482
:108190004043BBE4D4F89C7094F8DD30202B7FF48E
:1081A00029AD3B46192229466048F8F7B5FD00285D
:1081B0007FF420AD94F8DC1001293FF41BADD4F816
:1081C000A02084F8DC501368594923F4006313603D
:1081D000D4F8A0204FF0220C84F8DDC084F8DE60D3
:1081E000C4F8E000C4F8CC10166846F48061116051
:1081F000D4F8A020136843F48076014616603B460D
:108200002A464FF00110F8F787FD60B9D4F8A010A6
:108210004848A0220A613A462946F8F743FD00285B
:108220005ED0D4F8E030D4F8E020434D002184F84B
:10823000DC10E0E45F6847F4006058605A6822F49C
:1082400060455D604FF4604999FAA9F8D4F8A067D9
:108250005F68B8FA88F1701E88403843586038E784
:10826000FBF7A0FBD4F82C17192606FB00FC4B00EB
:108270004FF06409BCFBF3F0B0FBF9F24FEA0218CF
:10828000FBF790FBD4F82C7706FB00F07900B0FBED
:10829000F1FAFBF787FBD4F82C3706FB00F05A0005
:1082A000B0FBF2F0B0FBF9F709FB17A1CB003233BA
:1082B000B3FBF9F2500000F4F87BFBF773FBD4F842
:1082C0002C7706FB00F07900B0FBF1F7FBF76AFBB7
:1082D00082E547F4004319E425F040519960E5E652
:1082E000D4F8A0301390586913909E6913963846BD
:1082F000139BF8F7E9FD30B9D4F8A01008613846AF
:10830000F8F7E2FDD0B1D4F8E030042B8BD1D4F8EB
:10831000A020166846F40070106084E70023014036
:108320000100000F0004024000E100E00200100024
:108330000000FFFF020001006F040120D4F8A0201C
:10834000136843F48076014616603B462A464FF098
:108350000110F8F7E1FC00287FF465AFD4F8A030F5
:108360003A48A1221A6129463A46F8F79BFC0028B0
:108370007FF457AFD4F8A0000025129541691291FF
:10838000866912963846129BF8F766FD014600286A
:1083900058D1D4F8A0301D695A6984F82C5412F0D1
:1083A000040A43D151463B4601222948F8F7B4FC60
:1083B000014600287FF41EACD4F8A060244833683E
:1083C00023F480653560D4F8A0203B46176984F813
:1083D0002D740122F8F7A0FC00287FF40BACD4F830
:1083E000A000016841F400730360D4F8A05094F831
:1083F0002C642A692F6984F82F7400212020FF2E15
:1084000084F8DD0084F82E2484F8DC1084F8DE1073
:10841000104D7FF4F0AB28460121F8F78DFDB4F83C
:108420002D7487427FF4E7ABFFF7F1BB1E69084864
:1084300084F82D643B460122F8F76EFC0028CED06C
:10844000FFF7D8BBD4F8E030FFF7D4BB020001003F
:10845000040001006F040120014BC3F8740770474A
:10846000400001207BB972B90029BEBF00204FF047
:10847000004106E008BF00281CBF6FF000414FF02C
:10848000FF3000F0BDB9ADF1080C6DE904CE002954
:1084900009DB002B1ADB00F04DF8DDF804E0DDE924
:1084A000022304B07047404261EB4101002B1BDB0B
:1084B00000F040F8DDF804E0DDE9022304B04042BA
:1084C00061EB4101524263EB43037047524263EB5D
:1084D000430300F02FF8DDF804E0DDE9022304B0E7
:1084E000404261EB41017047524263EB430300F0AD
:1084F00021F8DDF804E0DDE9022304B0524263EB29
:108500004303704753B94AB9002908BF00281CBF6C
:108510004FF0FF314FF0FF3000F072B9ADF1080CB1
:108520006DE904CE00F006F8DDF804E0DDE9022391
:1085300004B070472DE9F047089E04468846002B9A
:108540004BD18A42154667D9B2FA82F24AB1C2F1DA
:10855000200701FA02F320FA07F7954047EA0308DB
:1085600094404FEA154E230CB8FBFEF71FFA85FC2A
:108570000EFB178843EA084307FB0CF1994209D91F
:10858000EB1807F1FF3080F01B81994240F218810F
:10859000023F2B445B1AA4B2B3FBFEF00EFB103378
:1085A00044EA034400FB0CFCA44509D92C1900F152
:1085B000FF3380F00781A44540F2048102382C4447
:1085C00040EA0740A4EB0C0400271EB1D44000236E
:1085D000C6E900433946BDE8F0878B4209D9002E31
:1085E00000F0EB800027C6E9000138463946BDE8B7
:1085F000F087B3FA83F7002F47D18B4202D3824230
:1086000000F2FA80841A61EB030301209846002EE1
:10861000E0D0C6E90048DDE702B9FFDEB2FA82F237
:10862000002A40F08F80491B4FEA154E1FFA85F84B
:108630000127B1FBFEFC230C0EFB1C1143EA014396
:1086400008FB0CF1994207D9EB180CF1FF3002D26C
:10865000994200F2CD808446591AA3B2B1FBFEF0D4
:108660000EFB101443EA044408FB00F8A04507D9A8
:108670002C1900F1FF3302D2A04500F2B680184653
:10868000A4EB080440EA0C409FE7C7F1200CBB4074
:1086900022FA0CFE4EEA030E01FA07F420FA0CF55A
:1086A00021FA0CF34FEA1E482543B3FBF8F92C0CD2
:1086B00008FB19331FFA8EFA44EA034309FB0AF454
:1086C0009C4202FA07F200FA07F10BD91EEB0303F2
:1086D00009F1FF3080F087809C4240F28480A9F14C
:1086E000020973441B1BADB2B3FBF8F008FB103357
:1086F00045EA034400FB0AFAA24508D91EEB04042C
:1087000000F1FF336BD2A24569D90238744440EAC4
:108710000940A0FB0289A4EB0A044C45C2464B4623
:1087200054D351D0002E69D0B1EB0A0564EB030499
:1087300004FA0CFCFD40FC404CEA0505C6E9005477
:10874000002747E7C2F1200320FA03F7954001FA1A
:1087500002F021FA03F34FEA154E3843010CB3FB44
:10876000FEF71FFA85F80EFB173341EA034107FBBA
:1087700008F38B4204FA02F407D9691807F1FF3CA9
:108780002FD28B422DD9023F2944CB1A81B2B3FBA1
:10879000FEF00EFB103341EA034100FB08F38B426D
:1087A00007D9691800F1FF3C17D28B4215D902385E
:1087B0002944C91A40EA07473BE73746304609E7EC
:1087C0000746E7E61846FBE64145ABD2B8EB020A9E
:1087D00069EB0E0201381346A4E76046E9E7184644
:1087E00095E76746D1E781467CE702382C4447E7A6
:1087F000ACF1020C2B442FE7384608E73746E9E690
:10880000704700BF844641EA000313F003036DD1B3
:10881000403A41D351F8043B40F8043B51F8043B43
:1088200040F8043B51F8043B40F8043B51F8043B4A
:1088300040F8043B51F8043B40F8043B51F8043B3A
:1088400040F8043B51F8043B40F8043B51F8043B2A
:1088500040F8043B51F8043B40F8043B51F8043B1A
:1088600040F8043B51F8043B40F8043B51F8043B0A
:1088700040F8043B51F8043B40F8043B51F8043BFA
:1088800040F8043B51F8043B40F8043B51F8043BEA
:1088900040F8043B403ABDD2303211D351F8043B8A
:1088A00040F8043B51F8043B40F8043B51F8043BCA
:1088B00040F8043B51F8043B40F8043B103AEDD239
:1088C0000C3205D351F8043B40F8043B043AF9D28A
:1088D000043208D0D2071CBF11F8013B00F8013B5D
:1088E00001D30B8803806046704700BF082A13D36A
:1088F0008B078DD010F003038AD0C3F10403D21A82
:10890000DB071CBF11F8013B00F8013B80D331F8B5
:10891000023B20F8023B7BE7043AD9D3013A11F835
:10892000013B00F8013BF9D20B7803704B784370A0
:108930008B788370604670470000000000000000E4
:1089400090F800F06DE9024520F007016FF0000C8F
:1089500010F0070491F820F040F049804FF0000437
:108960006FF00700D1E9002391F840F000F1080012
:1089700082FA4CF2A4FA8CF283FA4CF3A2FA8CF34A
:108980004BBBD1E9022382FA4CF200F10800A4FAB1
:108990008CF283FA4CF3A2FA8CF3E3B9D1E9042305
:1089A00082FA4CF200F10800A4FA8CF283FA4CF33C
:1089B000A2FA8CF37BB9D1E9062301F1200182FAF6
:1089C0004CF200F10800A4FA8CF283FA4CF3A2FAFC
:1089D0008CF3002BC6D0002A04BF04301A4612BA0A
:1089E000B2FA82F2FDE8024500EBD2007047D1E90D
:1089F000002304F00305C4F100004FEAC50514F09C
:108A0000040F91F840F00CFA05F562EA05021CBF6C
:108A100063EA050362464FF00004A9E72DE98048A8
:108A2000CDB072B6FEF7D8FDC14BC24F13F8483C2B
:108A3000002B01F0CA85C04BC7F85C3103F19801E7
:108A400003F5987503F5E47003F51874C7F8601121
:108A5000C7F8645103F53E7103F56475C7F8680102
:108A6000C7F86C4103F5856003F5986403F5AB63C3
:108A7000C7F87C41B14AC7F87011A3F23C54A24632
:108A8000C7F87801C3F89820AD4EAE48AE49AF4A5A
:108A9000C7F87451C3F8A460C4F8E405C4F8E81535
:108AA000C4F8EC25AA4EAB4DAB4CC7F88031CAF8E0
:108AB000F065CAF8F455CAF82446A849A84BA94855
:108AC000A94EAA4AAA4DAB4CCAF8F815CAF82836DE
:108AD000CAF82C06CAF83066CAF83426CAF83856DE
:108AE000CAF83C464FF00A09A349A44EA44BA54836
:108AF000A54DA64AA64CCAF84016CAF84466CAF85C
:108B00004836CAF84C06CAF85456CAF8582687F8A8
:108B10008491A04ECAF874469F4DA04CCAF898663E
:108B2000CAF8A056CAF8B8469D4E9E4D9E4CCAF84B
:108B3000D866CAF8DC56CAF8E4469C499C4B9D4866
:108B40009D4A9E4E9E4D9F4CCAF89C16CAF8A4366C
:108B5000CAF8B406CAF8D426CAF8E067CAF8E857D3
:108B6000CAF8EC479849994B99489A4A9A4E9B4DB6
:108B70009B4CCAF8E016CAF8E836CAF8D407CAF817
:108B8000E427CAF8F467CAF82858CAF83048954963
:108B9000954B9648964A974E974D984CCAF8F017C1
:108BA000CAF8F837CAF82408CAF82C28CAF8346872
:108BB000CAF83C58CAF848489149924B9248934A9F
:108BC000934E944D944CCAF83818CAF84038CAF8F5
:108BD0004408CAF84C28CAF854689049CAF858584A
:108BE0008F4B9048904ECAF89848904A904D914CBF
:108BF000CAF87418CAF89C38CAF8A008CAF8A46859
:108C00008D49CAF8B4288D4ECAF8B8588C4BCAF8AA
:108C1000D4488C488C4D8D4A8D4CCAF8D818CAF867
:108C2000DC68CAF8E038CAF8E408CAF8E858CAF8B4
:108C3000D429C7F8744762B6864D874E95F805B0BB
:108C400001248021A34587F88C41B16187F8E84170
:108C500001F2B084687B012801F2A08401267F4CD8
:108C60007F4BC7F8244740F2012C4FF0400E002103
:108C70002E75A7F822C7A7F820E7C7F80414C7F88D
:108C80001C37784CFCF7F2FF87F87867764EB846C9
:108C9000274890F8D879002F00F08685012F00F042
:108CA000AD85022F01F0948098F81934002B00F064
:108CB000C082D8F81C74D8F81004B8F82024C11B5E
:108CC0008BB29342C0F0B582B8F822B4991A3A44F4
:108CD0000BEB0107B7F5004FA2EB0B094FF0980221
:108CE00088BF89440DEB02004FF0000188BFA8F84F
:108CF000203402F01DFDB8F8200498F818248DF8EF
:108D00009E20010A4FEA1B2C41EA00274CEA0B2A5D
:108D10000520A0238DF89D00ADF8A170ADF89FA0AF
:108D20008DF89A30D8F89C009DF89820A4E000BFF8
:108D300038110120400001201C1101209110000871
:108D4000591C000801520008311C0008891C000849
:108D5000811C00081D1C0008751B0008CD1B0008A5
:108D6000551B0008F5730008B51A0008915B000850
:108D7000E95A0008591A0008C1190008A119000889
:108D800079190008215B0008DD180008B1180008F7
:108D90004D18000871720008556F00081916000878
:108DA000054200080D16000805160008E9700008C5
:108DB000616F00081D1600081516000841550008CF
:108DC000351C000895100008294200083D420008A3
:108DD000E1510008491C0008191C000899100008FE
:108DE0000D1B00082D1C0008091C0008A51B00080D
:108DF000311B0008A9100008791A00087D19000825
:108E00008D1A0008FD1900082D5600086519000884
:108E1000D9180008B910000849180008811800087E
:108E200045180008411800083D18000821160008E0
:108E300059420008D11000081116000861110008FD
:108E400009160008611500085D150008C94F0008E3
:108E5000051000080000002000000240DB1B040099
:108E6000B9A201003022012000ED00E0D8F89C708A
:108E70003B1A642B01F2D58398F86137202BF5D18A
:108E80006E48212740214FF4047E102A88F861772C
:108E90008161A8F8B0EF00F0B78188F8B22F0327FE
:108EA0009DF899106648102907F1010300EB070CA3
:108EB00001F0B8849DF89A00614F8CF800105A1C9C
:108EC000102892B207EB030A00F07A879DF89B10F6
:108ED0008AF800005A48531C10299BB2104406D14E
:108EE000574F02F1020EB954F8181FFA8EF39DF88D
:108EF0009CA0017052495A1CBAF1100F92B2194449
:108F000005D14F4F981C07F803A0B91882B29DF8FD
:108F10009DC081F800A04A49531CBCF1100F9BB2C0
:108F2000114405D1464F901C07F802C0F91883B2CE
:108F30009DF89E0081F800C041495A1C102892B249
:108F4000194406D13E4F03F1020EF854B9181FFA26
:108F50008EF29DF89FA008703949531CBAF1100F8A
:108F60009BB2114405D1364F901C07F802A0F918A6
:108F700083B29DF8A00081F800A031495A1C102846
:108F800092B2194406D12E4F03F1020CF854B918CD
:108F90001FFA8CF29DF8A1E008702949531CBEF11C
:108FA000100F9BB2114405D1254F901C07F802E029
:108FB000F91883B29DF8A20081F800E020495A1CFC
:108FC00010281FFA82FA01EB030C07D11C4F9A1CE0
:108FD000F85407EB0A0C53461FFA82FA991C18FA48
:108FE00081F2C2448CF80000D8F828771448C8F8F9
:108FF0004807033310214FF0030E8AF8B01FA8F87A
:109000004E3782F8B0EFF9680C4B0497C9F30E0A9B
:109010004FF00009CC464FF4800241F08000F86028
:10902000D1469A61DA46E346DA4540F2F58026A950
:109030004FF0020E0091CDF808808CE0000802404D
:10904000F00F0120DA450EF10E0E1FFA83FB01F03E
:10905000FD83704B159333F81900069B11F4004FF4
:109060000CBF89464FF0000909F1010CD8719245F7
:109070004FEA10201FFA8CF198711FFA87FC01F05B
:10908000E5836448099F30F81930FB711B0A11F41D
:10909000004FBB710A9FBDF820C00CBF89464FF03E
:1090A000000909F10101BA458BB201F0CF8330F814
:1090B00019100C9FBDF82CC0F97113F4004F4FEA42
:1090C00011220D99BA7118BF002399468A4503F100
:1090D00001039BB201F0BA8330F819100F9FBDF85D
:1090E00038C0F971090A13F4004FB971109F9946FD
:1090F00018BF4FF0000909F10102BA4593B201F01F
:10910000A58330F81910129ABDF844C0D17113F438
:10911000004F4FEA1127139997710CBF99464FF0F2
:10912000000909F101038A459AB201F08F83394899
:10913000BDF850C030F8197088F8077012F4004F6D
:109140004FEA17230CBF91464FF00009DA4588F823
:10915000063001F07B830BF101032E4A009F32F8A9
:109160001900F8711FFA83FB0BF101018AB2571C39
:10917000BBB20A93013399B20D9101318FB21097AE
:109180000137BBB2009F1393000AB8713846023012
:1091900006900EF1020702300990B81C0890009862
:1091A00006300C900EF106000B90009808300F90DE
:1091B0000EF108000E9000980A3012900EF10A008D
:1091C0001190009809F101081FFA88F900F10C08C4
:1091D0000EF10C0019F4004F1490009818BF4FF0D6
:1091E000000909F1010C0E30BEF1800F1FFA8CF15D
:1091F00003F101031FFA8EFC00907FF423AFDDF82A
:109200000880F44601F025BB41F21002A8F8B22F05
:10921000042745E640000020A969C64A881A0023B1
:109220004710C8F8107488F81934C8F81C3488F846
:10923000183498F8F97D002F41F0F28498F8FC0D6D
:10924000002841F0CD8498F85931002B41F0F78186
:1092500098F82834002B3FF41BADB74F4FF4003083
:109260004FF480214FF0000E4FF4803288F894E6DE
:10927000B861B961BA61D8F80030DF6827F0010041
:10928000D860196A41F2111911EA090F09D11F6A50
:1092900040F2444A17EA0A0F03D11A6822F001008B
:1092A00018601123D8F80000A449C8F80C30F6F76C
:1092B000A7FFD8F80070D8F808103868D8F8102040
:1092C00020F070030B4323F4407111433960D8F848
:1092D0000070D8F80C00D8F80430F8620122BB62A4
:1092E0007A61F96841F00100F8603B6843F00102DF
:1092F0003A6072B6924F6F6362B68F4898F88C11DD
:10930000009100234FF4000288F88C31826198F8B4
:109310006177212FFBD0884B8A498B4F8B484FF4C4
:10932000801E4FF4000C4FF4002B4FF480024FF0DE
:109330008059C3F818B04FF0040A9A614FF0000B3F
:10934000C3F818904022C3F818E04FF00309C1F8A1
:1093500000C026A9CDE92629CDF8A8A0CDE928BBD3
:10936000F7F756F8802326A978482693CDE9279B5E
:10937000CDE929BAF7F74CF8396C744821F400129A
:109380003A6426A94FF4007ACDE9279BCDF8A4B022
:10939000CDF898A0F7F73CF84FF4806326A96B4806
:1093A0002693F7F735F84FF4805226A9674826929E
:1093B0004FF00509F7F72CF84FF4005326A963483E
:1093C0002693CDF8A890F7F723F84FF4004226A98A
:1093D0005E482692CDF8A890F7F71AF84FF480432C
:1093E00026A95A482693CDF8A890F7F711F8786C7B
:1093F000574A20F480517964136823F0020010600A
:109400009AFAAAF1B1FA81FC0CF1845303F56030A9
:10941000830001214F481960036823F003030B43C5
:109420000360306940F00403336130BF306920F0DD
:10943000040333619AFAAAF0B0FA80FA0AF1845C64
:109440000CF560339B000F20C3F800B0136843F0A5
:1094500002031360CDF85CB03A6C42F080533B6479
:109460003A6C269002F080501790179B3B685B0384
:1094700041F11A83CDF89C903349334F0A6812F0BA
:10948000010018BF01202990F8213B6891FAA1FB47
:10949000BBFA8BF203F0F800D0402A90396F4807EE
:1094A00041F1B881052228922748274B416FDFF808
:1094B00098A011F0010718BF01272B971868C20167
:1094C0004CBF022001202C90DAF8042002F4800125
:1094D0002D91DAF8047007F03F032E93DAF80400B8
:1094E00047F6C07191FAA1F9B9FA89F20840D04063
:1094F0002F90DAF804704FF4403393FAA3F007F496
:10950000403C0CF58031B0FA80F24F00D7403097E4
:10951000DAF804304FF0706090FAA0F1B1FA81F7F8
:1095200003F07062FA403192DAF804304FF0E04014
:1095300012E000BF40000020000002404400012073
:109540007D10000800E100E0003802400004024005
:1095500010E000E00070004090FAA0F1B1FA81F74D
:1095600003F0E042FA404FF0010B022726A83292A6
:109570002C97CDE926BBF9F739FF0F231A93DAF8B8
:109580000800934A00F003011B91DAF8083003F059
:10959000F0001C90DAF8081001F4E0531D93DAF89B
:1095A0000800C10801F4E0531E931068CDE91AB712
:1095B000176800F00F0107F00F0A8A45C1F02081FB
:1095C0001AA8FAF7C5F8834983484FF40007C1F891
:1095D00080704FF000094FF0400E04274FF0120B3F
:1095E0001FA9CDE91FEB2397CDE92199F6F710FFCD
:1095F000802201231FA978482397784F1F92229336
:10960000CDF880B0CDF88490F6F702FFCDF86490E5
:109610003A6C7348734942F400133B643F6CC8F8DA
:10962000A00007F400121992199B98F8DD30C8F8D1
:10963000B4904FF480425E27FE20C8F8BC90C8F872
:10964000C09003F0FF0CC8F8B020C8E92912C8F890
:10965000AC70C8F8B8001BB988F8DCC0F7F700F8A0
:10966000D8F8A0205D4F242188F8DD10136823F07E
:1096700001001060B9684FF4E05292FAA2FA5A4819
:109680005A4ABAFA8AF301F4E057DF400744EB6A1A
:1096900097F89470D8F8A000554923FA07FBBBFB54
:1096A000F2FEC0F804E0D8F8A4308B4201F2458203
:1096B0005900BBFBF1F3C3F30B070EF10102032FBB
:1096C000026298BF0423C361D8E92F373B4303608C
:1096D000D8E92B23D8F8A0004049DFF8FC901343C9
:1096E0008360D8E92D721743C760076847F001020D
:1096F000026000232020C8F8E03088F8DD00C8F8B8
:10970000D03088F8DE3018934F6C47F480524A64AA
:10971000496C219301F4805018904FF4007B484627
:109720001FA94FF0010A189A2293CDE91FBA4FF4EE
:109730008067F6F76DFEC9F818B01FA91F974FF4A0
:10974000805BF6F765FEC9F818701FA90527CDF8EC
:109750007CB0F6F75DFE4FF4005CC9F818B0022348
:109760001FA9CDE91FC32397F6F752FE4FF400421D
:109770001FA91F922397F6F74BFE4FF480431FA9B2
:1097800023971F93F6F744FE1A481021816172B6A1
:10979000FCF76CFA009F002F41F09C81002288F8B2
:1097A000282462B6FFF774BA39464FF4006200F617
:1097B000DC1001F0BDFF3846C4F8E470FAF70CF98C
:1097C0000D49012081F8D809FCF750FAFFF76CBA6F
:1097D000003C024000E100E000040240003802408A
:1097E00000540040801A060000BD000840420F00EF
:1097F000A086010000000240381101206F782B8CF8
:10980000AA6A0D974FF480400C9392FBF0F1C14689
:109810000B914FF0000BD9F8FC21D9F80072BA4235
:1098200000F0ED8199F88C01D9F8883150B1D9F860
:1098300004243AB1D9F808145F1A142F00D89047BD
:10984000C9F804B4D9F80C04D9F8FC21D9F80032CD
:1098500001309A420490C9F80C0400F0DD81D9F877
:109860000002C2B2043209EB420EBEF8FC31D9F854
:1098700000121FFA83F80FFA88F787FB0723900B73
:10988000013140EA834202970692C9F80012D9F8E2
:109890001034A969DB4A99F86C7AA1F80080013389
:1098A000C3F30E0002EB40010097C9F81034A96120
:1098B000B4F8E8809FB1009B049A03F1FF3A0AEBE9
:1098C0008A0709EB870CDCF8D007111AB1F5806F15
:1098D00005D94046FAF780F899F86C3A0093D9F820
:1098E000947AD9F8982A3946B81CC9F8940A31F9FB
:1098F000040BC9F8941AB7F90210C34F4FEA0813C2
:1099000007EB030A029FBAF902E007FB01F107FB2C
:1099100000F0BD4FFF5E40F38F3041F38F31A0EB7D
:10992000070CD9F8787AA1EB0E0EBE44B64FC9F8F1
:1099300078EAF852D9F8743AAAF802100CEB03004E
:10994000134602F1020CC9F898CAC9F8740A33F92F
:1099500004EBC9F8983AB2F902200298BAF9043037
:10996000BAF9061000FB0EFC00FB02F24FEA880079
:10997000089001304CF38F3C27F820C0ACEB030E6D
:1099800042F38F32D9F89CCAD9F87C3A07EB8000B1
:10999000D9F8807A4280511A3944624673440CF1F6
:1099A000020EC9F8801AC9F87C3AC9F89CEA32F963
:1099B000040BC9F89C2A029FBCF90210BAF90830BE
:1099C000D9F8842ABAF90AC007FB00F04FEA480820
:1099D00008F1010840F38F3007FB01F18A4FA0EB3B
:1099E000030E27F83800D9F8883A07EBC80041F38E
:1099F0008F319644D9F8A02A4180A1EB0C0CC9F80C
:109A000084EA9C449646931C08988049C9F888CA01
:109A1000C9F8A03A3EF9043BC9F8A0EA0144069807
:109A2000B2F90220BAF90CE0BAF90EC0D1F8DCA9FB
:109A3000C1F8DC0902994FEA480001FB02F201304B
:109A400001FB03F141F38F3127F8201042F38F38E7
:109A500007EB8000D9F88C2A069FD4F8E430A0F8F0
:109A60000280A1EB0E010A44A7EB0A0E0099D9F877
:109A7000907AC9F88C2A7344A8EB0C0CBC4401F111
:109A8000010A03F58072C9F890CAC4F8E4301FFADD
:109A900081FC09928E46CDF838A0CDF828A0CDF8EB
:109AA0003CA04F460EE0D2F8CC070130C2F8CC07FC
:109AB0000CF101020A981FFA82FC8445E64660DC3C
:109AC000DDF83CA05FFA8CF303F0010007EB00180F
:109AD0004FEA8E01D8F8742AD8F8789A089382FB56
:109AE00002230291910B41EA834189FB0923CDE9CD
:109AF0000623D8F87C0AD8F8808A079B88FB088957
:109B0000920BCDE9068942EA83430B440799029AF6
:109B10004FEA983848EA814980FB0001CDE9060107
:109B20007244079907EB8202800B40EA8148D2F821
:109B3000C4070999C844434493FBF1F38342B2DD5F
:109B400010B90499C2F8D4170299089A049871447C
:109B5000013207EB8109D1B25145C9F8D007C9F8E4
:109B6000C43789F8C8B7C9F8CCB7A1DC01EB8108C4
:109B7000013107EB8803C9B25145C3F8C4B7F5DD1D
:109B800096E7B946009F0B9AB4F8E81007EB870AEE
:109B900009EB8A08D8F8C4379A4245DD0131C1F390
:109BA0000801A4F8E81000297FF435AE184B99F8A5
:109BB00070BA99F8718A174F9B4498449BF8ACA6E9
:109BC00098F8B0269BF8AEE698F8B2C607EB8A0084
:109BD00007EB8E0107EB820B07EB8C08DBF8AC2060
:109BE000D0F8AC70D8F8AC30D1F8AC00C9F8947AA1
:109BF000C9F8980AC9F89C2AC9F8A03A09E6C846E3
:109C0000FFF752B8400000205824012038110120ED
:109C1000D022010800BD000800214FF0FF37069157
:109C200002974FF6FF7832E6D8F8CC770C9AB14B12
:109C3000B148C9F824079742C9F81C370BD2009ADB
:109C4000002AABD0009BD9F8D07704985B02C21BE6
:109C500080339A42A2D9009FA84B17F0010A09EB62
:109C60000A0C14BF04224FF480229A619CF8700AF7
:109C7000A34F0130C2B207EB8A0E022A8CF8702A79
:109C8000DEF8A43004BF8CF870BA00220131985C71
:109C900007EB8008C1F30807D8F8ACE0BF0009EB78
:109CA000CA0C1A440EEB0703CCF8943A9078944A05
:109CB00002EB80080FFA8AF2D8F8AC301F44CCF8D7
:109CC000987A904B904FD00003440744A3F800B01B
:109CD000A3F802B0A3F804B0A3F806B0A3F810B03C
:109CE000A3F812B0A3F814B0A3F816B0A3F820B0EC
:109CF000A3F822B0A3F824B0A3F826B0A3F830B09C
:109D0000A3F832B0A3F834B0A3F836B0A3F840B04B
:109D1000A3F842B0A3F844B0A3F846B0A3F850B0FB
:109D2000A3F852B0A3F854B0A3F856B0A3F860B0AB
:109D3000A3F862B0A3F864B0A3F866B0A3F870B05B
:109D400003F1700A80339F42AAF802B0AAF804B067
:109D5000AAF806B0BAD16D48009F120183181F2FD0
:109D600040F802B0C3E901BBC3F80CB006D809EB58
:109D7000470EBEF8A8210132AEF8A8219DF8383070
:109D80000D9F89F86C3A03EB830009EB800CBB4212
:109D9000CCF8CCB7FFF403AF0020D9F8D017C846F1
:109DA0008346142201305A4F5FFA80FA534502FB72
:109DB000007940F25386D9F80C707F1ABB44F1E762
:109DC000544F991C07EB020AF8548AB2FFF77EB889
:109DD000D8F8FC21D8F800329A4239D098F88C1182
:109DE000D8F8880159B1D8F8047447B1D8F80824D4
:109DF000831A142B00D8B8470021C8F80414D8F8E7
:109E00000C04D8F8FC71D8F8002201309742C8F849
:109E10000C0400F03186D8F80032D9B2043108EBD6
:109E2000410ABAF8FC01D8F8007201371FFA80F92C
:109E3000C8F80072D8F810243749AB690132C2F370
:109E40000E0B01EB4B00C8F81024A861A3F800909A
:109E5000D4F8EC70D8F80C2497427EF425AFB8F80B
:109E6000923126482D4A4FF400010133A8F892316F
:109E7000816198F818744FF0000C022F82F8D8C94D
:109E800000F0FE851D4A02279761697895F815E074
:109E9000AF6A234A1A920131BEEB010348BF033374
:109EA00098100130C1B2002FB8BF07F57F570A9153
:109EB000B8BF3F370A98BB130D93002800F06283A8
:109EC0000021184A184B04910C910020CDE908009C
:109ED0000DF1690101270B910697CDE91F2300229F
:109EE000C4F8E420CDE92622CDE928224FF40079F8
:109EF0007DE000BFB9A20100DB1B040000080240A6
:109F000000BD00085824012058440120B40A012053
:109F100004080120F00F012040000020381101202A
:109F200001000001A0D60008A0F60008D8F8000241
:109F3000C1B2043108EB410BBBF8FC21D8F8000298
:109F40001FFA82FA0FFA8AF787FB0723910B013079
:109F500041EA834CC8F80002AA69D8F81034A2F884
:109F600000A01F98279902460133009332F9043B61
:109F70001F9207FB03FA269B4AF38F321A4426925C
:109F8000B0F902B0009B2098C8F8103407FB0BF31F
:109F900043F38F3A8346514427913BF9043BCDF874
:109FA00080B007FB03F343F38F3A289B9A44CDF824
:109FB000A0A0B0F90200D4F8E430029307FB00F748
:109FC00009F1FF30009B1FFA80F9299847F38F377A
:109FD000C3F30E0B07445D4B0298299703EB4B0329
:109FE0006044AB61C4F8E400B9F1000F36D0D8F892
:109FF000FC01D8F80032984224D098F88C11D8F897
:10A00000883159B1D8F8047447B1D8F80824981A9F
:10A01000142800D8B8470021C8F80414D8F80C74E4
:10A02000D8F8FC21D8F8003207F1010E9A42C8F89E
:10A030000CE47FF47BAF4FF0000C4FF0FF374FF68E
:10A04000FF7A89E7316921F00407376130BFD8F81A
:10A05000FC21D8F800028242CFD1F3E78AFB0AAB99
:10A06000BC46CDE902AB8CFB0CBCCDE900BCDDE904
:10A0700002AB074608465146890B41EA8B4180FBFB
:10A0800000AB0098019B800B40EA834082FB0223D7
:10A090004FEA9A3C920B9A4642EA8A4A01444CEAB9
:10A0A0008B4C06980D9B089AE24407F58077514443
:10A0B00091FBF7F18B42C8BF0020069002B30999CB
:10A0C0000B9B1BAF81F001009F42CDE908901A461F
:10A0D0001DD012F801CB1E4F09980B9207EB8C0E86
:10A0E000DEF8A430191813F8009091F802A007EBDD
:10A0F000890B07EB8A0CDBF8AC20DCF8AC30ECE623
:10A1000001270B9B08971BAF9F421A46E1D1069986
:10A1100001BB04980A9B0130C7B29F4204900C9780
:10A1200080F030820A499DF8682001EB8209D9F855
:10A13000A400877890F800E001EB870C01EB8E0B10
:10A14000DCF8AC30DBF8AC20BFE600BF40000020FC
:10A1500000BD0008B8F894310C9A0133062A7746FE
:10A16000A8F8943107D8049908EB410ABAF8EC0131
:10A170000130AAF8EC01D8F88831D8F8FC21D8F8D9
:10A180000012E86B521A9B1AB84A4FF400319161E1
:10A1900098220021C4F8F03001F0CAFA4FF4897215
:10A1A0000021B34801F0C4FA022288F8AE2AAF4A6F
:10A1B00095F800A088F8A5AA4FF0040C002388F8B1
:10A1C000B8CA4FF0FF094FF400214FF480109446B5
:10A1D0004FF0030BA8F8C83BC8F8B03AC8F8B43A37
:10A1E000C8F8A83A88F8AD3A88F8AC9A88F8AFBAB7
:10A1F0004FF4800391614FF4001990614FF4000116
:10A200009B48C2F818909361CCF8181000220023E4
:10A21000C4F8F470A86340E903231B27F9F78CFC0A
:10A22000013F1FFA87FBF9F787FCF9F785FC0BF173
:10A23000FF331FFA83FAF9F77FFC0AF1FF321FFAA6
:10A2400082F9F9F779FC09F1FF318FB2F9F774FC63
:10A25000781E1FFA80FBF9F76FFC0BF1FF331FFA32
:10A2600083FAF9F769FC0AF1FF321FFA82F9F9F76C
:10A2700063FC09F1FF318FB2F9F75EFC781E87B2FB
:10A28000002FCDD1794A0021202393618C460823E9
:10A290000A910846029109910491009174490D9325
:10A2A000BE46BB460B970697089780230C9791F8FC
:10A2B00000A00C9A13EA0A0F4FEA420218BF42F0BC
:10A2C00001025B0808BF013192B291F800A00C9224
:10A2D0000A9A08BF802313EA0A0F4FEA420218BF06
:10A2E00042F001025B0808BF013192B20A920A787B
:10A2F00008BF802313424FEA4E0E18BF4EF0010EE6
:10A300005FEA530A04BF01314FF0800A0B784FEA2D
:10A310004C021AEA030F18BF42F001025FEA5A0A20
:10A3200004BF01314FF0800A0B787F001AEA030F57
:10A3300018BF47F001071FFA82FC5FEA5A0204BF08
:10A34000013180220B7840001A4218BF40F0010012
:10A35000520804BF013180220B784FEA4B0B1A429E
:10A3600018BF4BF0010B530808BF0131029A91F856
:10A3700000A008BF802313EA0A0F4FEA420218BF69
:10A3800042F001025B0808BF013192B291F80090DF
:10A3900002920B9A08BF802313EA090F4FEA420288
:10A3A00018BF42F001025B0808BF013192B291F878
:10A3B00000A00B92099A08BF802313EA0A0F4FEA04
:10A3C000420218BF42F001025B0808BF013192B29D
:10A3D00091F800A00992069A08BF802313EA0A0F99
:10A3E0004FEA420218BF42F001025B0808BF013188
:10A3F00092B291F800A00692049A08BF802313EA53
:10A400000A0F4FEA420218BF42F001025B0808BF80
:10A41000013192B291F800A00492089A08BF8023FB
:10A4200013EA0A0F4FEA420218BF42F001025B082A
:10A4300008BF013192B2089291F800A0009A08BFBB
:10A44000802313EA0A0F4FEA420218BF42F00102CA
:10A4500092B25B081FFA8EFEBFB280B21FFA8BFB6E
:10A46000009207D10131802304E000BF00080240C0
:10A470000C0C01200D9A013A12F0FF020D927FF4AC
:10A4800016AF0C9B0A99ADF88470ADF88600029F58
:10A490000B98ADF87C30ADF87E10ADF88A70ADF851
:10A4A0008C00099A069B0499089F0098ADF888B023
:10A4B000ADF880E0ADF882C0ADF88E20ADF89030F8
:10A4C000ADF89210ADF89470ADF896000DF17C0BDC
:10A4D0000DF1980A37E0BDF85AC0BCF1000F13D057
:10A4E000D5F83CE0B8F89A319EF88870674453FA82
:10A4F0008CF08EF88870CE4FA8F89A017B6983F0B3
:10A50000400040F48003BB613BF8020BF6F726FFE6
:10A5100048B3BDF85A1091B1EF6BB8F89A0197F8AB
:10A52000882050FA81F90A44C14987F88820A8F8A0
:10A530009A914B6983F0400747F48000886126AA0E
:10A540005A4500F01B8551460DF15A023BF8020BAB
:10A55000F6F704FF0AF102090DF15A02494609F122
:10A56000020A0028B7D1B248436983F0800747F454
:10A5700000018161B8F89C210132A8F89C21AC4B04
:10A5800002209861AA4AAB4FAB49C8F824774FF430
:10A590000030C8F81C179061FEF786BB2A690120BD
:10A5A000117AFBF7AFF900283EF458AB01262E7361
:10A5B000FEF754BBAB680020197AFBF7A3F900281B
:10A5C0003EF448AB2C71FEF745BB9C4C0521A4F131
:10A5D000440201251846C7F85421C7F8581104F859
:10A5E000485CD7F8546146F82300013397F8584186
:10A5F000DBB29C42F5D8924AC7F8F42D052100241D
:10A60000C7F8F81D25460FFA84F8D7F8F40D40F87E
:10A610002850013497F8F86DE4B2A642F3D8FEF75B
:10A620000ABA884E08254FF40064402080214FF478
:10A630008052B561B461B061B161B261FEE798F872
:10A640005B1198F858C14A1CD7B2BC4588F85B71B9
:10A6500098BF88F85B01581ED8F8543188F8590122
:10A6600053F8217097F802A01AF0800F40F0098487
:10A67000962200210DF19A0001F05AF898F82FB4B3
:10A680008DF898B0FF218DF89A107A788DF899207E
:10A6900038798DF89C00D946D8F89C0005E0D8F8A8
:10A6A0009C100B1A642B00F2078298F86137202B5C
:10A6B000F5D15F4B212140224FF40470B9F1100F06
:10A6C00088F861179A61A8F8B00F00F0E78108F6E2
:10A6D000B27E03239DF899205B498EF80090102AE2
:10A6E00003F1010C01EB030006D157488246604498
:10A6F0000AF8032003F1020C9DF89AB00270524A46
:10A700000CF1010EBBF1100F1FFA8EF3624406D15B
:10A710004D490CF1020001F80CB0CA1883B29DF843
:10A720009BC0494882F800B0BCF1100F03F1010250
:10A7300092B2184407D1444903F1020A01F803C058
:10A7400088181FFA8AF29DF89CB080F800C03E4835
:10A75000531CBBF1100F9BB2104407D13A4902F1D0
:10A76000020E01F802B0C8181FFA8EF39DF89DC0C2
:10A7700080F800B034485A1CBCF1100F1FFA82FA5E
:10A7800000EB030B08D130499A1C01F803C001EB20
:10A790000A0B53461FFA82FA981CC24418FA80F03A
:10A7A00010228BF800C003338AF8B02F4FF0030E4D
:10A7B000D8F828272449C8F8481780F8B0EFA8F837
:10A7C0004E37D3681A4943F080004FF4800CD060B4
:10A7D000C1F818C0384687F80090FBF7D9FB144A37
:10A7E0008023936198F88431092B3EF631AD08EB54
:10A7F000830B0133CBF85C7188F88431FEF728BDF8
:10A80000CBB21370126802F00F0088427EF4DBAE08
:10A81000FEF7D6BE3F6F17F0010318BF0123289340
:10A82000FEF742BE00EB030CC155BB1CFEF742BB5A
:10A8300000080240DB1B0400B9A20100381101200E
:10A840000811012000000240F00F0120DDF808800F
:10A85000D3465FFA8CF18A1DD8F89C008DF89D10C4
:10A860005FFA82FE009006E0D8F89C10009A8F1ADA
:10A87000642F00F2E58098F86177202FF4D126ABA1
:10A88000DA43C74F4FF021017244402088F8611726
:10A8900012F00302B8614FF4047726A94FF00203C7
:10A8A000A8F8B07F02924BD026A9BE4F11F8010B39
:10A8B00010284FF0030207F1020C06D1B87011F80E
:10A8C000010C07EB020C1346042226AFCF1BFFB28C
:10A8D000BE458CF8000040F29880FC2A134600F236
:10A8E00084809DF9080001282AD0022813D09DF801
:10A8F0009900AC4F531C102801F101019BB2174481
:10A9000006D1A84FB854023211F8010C1F4493B27B
:10A91000FC2B387069D811F8010BA24F5A1C102873
:10A920001FFA82FC1F4407D19E4FF854023311F8DE
:10A93000010C67441FFA83FC6346FC2B387054D823
:10A9400011F8010B974F5A1C102892B207EB030C19
:10A9500008D1F8549F1C934B11F8010C03EB020C27
:10A960001346BAB226AFCF1BFFB2BE458CF800002B
:10A970004BD9FC2A39D80F46531C17F8010B029704
:10A98000884F10289BB207EB020C07D1B8540298ED
:10A99000023210F8010C07EB030C93B2FC2B8CF87D
:10A9A000000022D848787F4F5A1C102892B21F44CA
:10A9B00005D17C4FF8540233487817449AB2FC2AE8
:10A9C000387012D88878774F531C10289BB201F149
:10A9D0000301174406D1734FB854023211F8010C29
:10A9E0001F4493B2FC2B3870AAD96D486D4AC8F841
:10A9F00048274FF000014FF020074FF48003A8F8DC
:10AA00004E1788F8617783612EE7991C424418FA43
:10AA100081FE102082F8B00F0499624FC8F8487781
:10AA2000032203338EF8B02FA8F84E37C86840F0E1
:10AA30008002CA605A494FF480078F61FEF7F4BA6A
:10AA4000594E08254FF40064402080234FF4805174
:10AA5000B561B461B061B361B161FEE7BBFBF3FE08
:10AA6000013301EB0321514A71440220C4F8EC1078
:10AA700082F8D809FEF718B94FF6FF79FFF7DAB96F
:10AA800098F81934002B7FF4FDA90121D8F810049F
:10AA900088F81914C8F81C04FFF7F4B988F8B29FB5
:10AAA00008F6B37E042315E63F6817F4803E08BF1E
:10AAB00071462791FEF7E0BC3B4E08254FF4006439
:10AAC000402780204FF48052B561B461B761B06116
:10AAD000B261FEE7344A88F88CA18023936198F82C
:10AAE000E891B9F1000F74D188F8E8A198F8E891DD
:10AAF0002F4895F805E04FEA4907C21992F84CA093
:10AB0000D6455BD82A49687B0F4497F84D70B84208
:10AB10002AD840F2012B402100232648264F85F8F1
:10AB20001490A8F822B7A8F82017C8F80434C8F879
:10AB30002407C8F81C77FEF731BE4FF49677D8F893
:10AB4000A81007FB0EF94FF47A72B9FBF2F7013740
:10AB50000762B9B903EB430ABBFBFAF7C7F30B0271
:10AB600062B90123FEF7AFBD2A69012012F8371040
:10AB7000FAF7C8FE0028CCD02F73CAE747F4004389
:10AB8000FEF7A1BD192101FB03F1BBFBF1FCCCF3E6
:10AB90000B03002BE5D04CF44043FEF794BD00BFFF
:10ABA00000080240F00F012000000240381101208F
:10ABB00000BD0008DB1B0400B9A20100AB68002047
:10ABC00013F83A10FAF79EFE00289BD085F804A0EF
:10ABD00098E7B9F1110F8BD9112188F8E81185E7B1
:10ABE000D8F814244FF0000C88F8FCCD82B1D8F8C6
:10ABF0008871D8F88831D91B8A4209D9306920F088
:10AC00000403336130BFD8F88811C81B8242F5D8DD
:10AC1000CE48FBF7BDF9CE4A80279761FEF718BBF7
:10AC200098F8FB1D98F8F83DD8F8F42D481C5FFA09
:10AC300080FC634588F8FBCD07F1FF3798BF4FF0E4
:10AC4000000C88F8F97D98BF88F8FBCD52F82110E8
:10AC500091F805A08E468A445EF8863FCAF8063011
:10AC6000BEF80400D8F89C70AAF80A00029701F117
:10AC7000FF3A06E0D8F89C00029A831A642B00F28F
:10AC80006F8198F86127202AF4D14B794FF0210089
:10AC900003F10C0788F86107FAB2AD484027052A8E
:10ACA000876140F2CE800B3351FA83FCAAEB0C0390
:10ACB000DA434FF4047012F00302A8F8B00FD6463E
:10ACC0004FF0020333D00878A24F10288E464FF081
:10ACD000030307F1020704D1023FB87008781F444C
:10ACE0000423FC2B387000F2AC80012A1FD0022A0A
:10ACF0000ED01EF8012F97485F1C102A1FFA87F903
:10AD0000184400F0B6804B46FC2B027000F299808C
:10AD10001EF8012F8F485F1C102A1FFA87FB18446A
:10AD200000F09F805B46FC2B027000F28A8000914D
:10AD300034E002461846BC458BF8009044D0FC2A0B
:10AD40007ED878788349531C10281FFA83FB11445E
:10AD500000F0F2805B46FC2B087071D8BA787D4910
:10AD6000581C102A1FFA80FB01EB030E00F0DC8058
:10AD70005B46FC2B8EF8002062D8FA787548591C87
:10AD8000102A1FFA81FB07F1030E00EB030900F004
:10AD9000C3805B46FC2B89F8002051D89EF80190B7
:10ADA0006C4A591CB9F1100F88B20EF1010702EB81
:10ADB000030BBED102F80390114602339EF80190B6
:10ADC0009AB201EB000BB6E7831C424418FA83FAEF
:10ADD000102382F8B03F0330D8F828275D4FA8F839
:10ADE0004E0703238AF8B03FC8F84877D768009920
:10ADF00047F08003D360564A4FF48000906198F882
:10AE00008471092F06D808EB870E0137CEF85C1144
:10AE100088F8847198F8F91D00297EF40FAA98F833
:10AE2000260401287EF40AAA01F1804C0CF50239AF
:10AE30004FF0006288F82714C9F81820FEF7FEB911
:10AE40000099434B4348C8F848074FF00007A8F85B
:10AE50004E774FF020024FF4800788F861279F61FA
:10AE600008E73C48C25402339EF800209BB2584485
:10AE700059E73848C25402339EF800209BB2484438
:10AE800042E7354B8AF0800103EB8109D9F8D4B54C
:10AE9000BBF1000F00F037813846D8479822824630
:10AEA000002800F0FD8000210DEB020000F040FCC6
:10AEB00097F802C0D9F8D4278DF89AC00DF19E00FA
:10AEC0009047831D411D8DF89D0026AAD8B2D8F861
:10AED0009C30029052FA81F104934FF021094FF017
:10AEE000000B4FF0200A98F86107202800F0A2809C
:10AEF000D8F89C00049A831A642BF4D9174E0825BD
:10AF00004FF40064402780214FF48050B561B46154
:10AF1000B761B161B061FEE70E49CA540233FA78F5
:10AF20009BB201EB0B0935E70A48C2540233BA78E9
:10AF30009BB200EB0B0E1CE7064B98549E46023268
:10AF4000787893B20EEB0B0105E700BF400E0120AD
:10AF500000080240F00F01203811012000000240DB
:10AF6000CF4E08254FF40064402780214FF48050D5
:10AF7000B561B461B761B161B061FEE700211A91BA
:10AF80008E460846CDF86B100DF196071AA93AE0E7
:10AF90001FFA82FB09F0070EC3F3800A4AEA4B024C
:10AFA00000F1020CBEF1070F12B21FFA8CF900F08B
:10AFB0002A821FFA82FBC3F3400242EA4B0A09F0DD
:10AFC00007020FFA8AF3072A08BF0B7000F1030E7D
:10AFD000B7F800901FFA8EFC14BF9BB2002309F053
:10AFE000010B0CF0070A08BF013104304BEA4302A1
:10AFF000BAF1070F80B213B200F00B821FFA83FE82
:10B00000382800F0E18037F8023F00F0070CC3F366
:10B01000C00B4BEA4E0ABCF1070F00F1010E0FFA0C
:10B020008AF21FFA8EF9B3D10A703B8801314FF0D2
:10B03000000BAFE79B4B88F8619740229A6102981A
:10B04000052821D94FF4047EA8F8B0EF02230DF1B2
:10B05000970E00911EF801CFBCF1100F08BF924966
:10B0600003F1010292B214BF1A4601F803C008EBC3
:10B070000201531C81F8B0CF00998E459BB200F0BD
:10B08000F180FC2BE6D900998648874AA8F84EB78C
:10B090004FF48003C8F8482788F861A7836127E741
:10B0A00001460DEB020097F8029000F041FBFE20F4
:10B0B0000122D8F89C108DF89E90CDF808A08DF84C
:10B0C0009A008DF89D2000914FF021094FF4047BE8
:10B0D0004FF0200A98F86137202B00F0E780D8F86D
:10B0E0009C00009A831A642BF4D96D4E08254FF406
:10B0F0000064402780214FF48050B561B461B7618E
:10B10000B161B061FEE7982259460DEB020000F0F4
:10B110000FFBFE200122D8F89C108DF89EA0CDF8E0
:10B1200008B08DF89A008DF89D2000914FF021090C
:10B130004FF4047B4FF0200A98F86137202B13D08E
:10B14000D8F89C3000981A1A642AF5D9544E08256C
:10B150004FF40064402780214FF48053B561B461FF
:10B16000B761B161B361FEE74E4B88F86197402249
:10B170009A610DF197000223A8F8B0BF10F801CF33
:10B18000BCF1100F08BF484903F1010292B214BF8D
:10B190001A4601F803C0511C08EB020E8BB20DF1E8
:10B1A0009E0181428EF8B0CF5CD0FC2BE6D9029A8A
:10B1B0003C48A8F84E273C4BC8F848374FF480026B
:10B1C00088F861A78261BBE70DF1670C00231CF8CA
:10B1D000012F534013F0800F4FEA430018BF80F057
:10B1E0009700C3B2590013F0800F18BF81F0970188
:10B1F000CFB27A0017F0800F18BF82F09702D0B25A
:10B20000430010F0800F18BF83F09703D9B24F00AE
:10B2100011F0800F18BF87F09707FAB2500012F0B4
:10B22000800F18BF80F09700C3B213F0800F4FEA71
:10B23000430118BF81F09701CFB217F0800F4FEA9A
:10B2400047020DF16E0018BF82F097026045D3B23D
:10B25000BDD1002B5AD0B8F898210132A8F8982116
:10B26000FFF78DB9901C434418FA80F910210E485D
:10B27000C8F8480783F8B01FD8F8281703324FF0F2
:10B28000030AA8F84E2789F8B0AFCB6843F08000D6
:10B29000C86004494FF480028A61FFF7A3BA00BF77
:10B2A0000000024000080240F00F0120C04B88F867
:10B2B000619740229A610DF197000223A8F8B0BF70
:10B2C00010F801CFBCF1100F08BFBA4903F1010219
:10B2D00092B214BF1A4601F803C0511C08EB020ECB
:10B2E0008BB20DF19E0181428EF8B0CFBAD0FC2B0B
:10B2F000E6D9029BAE48A8F84E37AE4AC8F84827B0
:10B300004FF4800388F861A78361E8E6EF6B1A9930
:10B310003960A748BDF86C20BA804FF400118161F4
:10B320007F792FB10C2F8CBF022301233B44DB001C
:10B33000EA6992F8009051784B44581E90FBF9F757
:10B3400011FB07F3703399B2B1F5096F3FF617A9F6
:10B3500098F8B82A881800F1FF3B9BFBF2FAAAF193
:10B360001C0E1FFA8EFA4FF0000B1FFA8BFCE24501
:10B3700004D9F8F7E1FB0BF1010BF6E7F9F79CFBB9
:10B3800000283FF4FCA8D8F8B41AD4F8F430D8F860
:10B390000C2498F8B89AEF6B81FB0101800B40EA0E
:10B3A000814ED8F8B01A08468346D21AC917BEFB98
:10B3B000F2FABBEB0A034FEA490C61F100010846BF
:10B3C0004FEAEC719E4603FB01F30CFB003BAEFB26
:10B3D0000C0100235944FDF745F8002871F10003E2
:10B3E00060DB4FF0010C6FF0004B0022834572EBE5
:10B3F000010E13DA83084FEA4C0C43EA81705FFABE
:10B400008CFC8910F2E70A703B8801314FF0000B89
:10B41000D1E50B704FF0000E0131F1E58A0342EAED
:10B42000904B4FEA803A00224FF08043910841EA66
:10B43000837292454FEAA3037BEB0301F6DB002006
:10B440000021CDE90001CDE902AB52EA03014FD062
:10B45000DDE90001DDE902ABCDE9040180185941C5
:10B4600082457BEB010E11DBBAEB000A6BEB010BA3
:10B47000CDE902ABDDE904AB12EB020E43EB0300B6
:10B480001AEB0E0A4BEB000BCDE900ABDDE9000136
:10B49000920849104FEA300042EA8372CDE9000178
:10B4A0009B10D2E70022FF2AB8F8C83B4248069317
:10B4B00028BFFF2287F88620D0E900011A46002322
:10B4C000FCF7D0FF002871F1000377DB4FF0010C8F
:10B4D0006FF0004B0022834572EB010E22DA8308E5
:10B4E0004FEA4C0C43EA81705FFA8CFC8910F2E75A
:10B4F00000988CFB00AB4FF0640CAAFB0C12CDE95A
:10B5000000120CFB0B210191DDE90012002972F100
:10B510000003C7DB11F5005042F10001830B43EA41
:10B520008142C0E7890341EA904B4FEA803A00220A
:10B530004FF08043920842EA837292454FEAA30398
:10B540007BEB0301F6DB00200021CDE90001CDE912
:10B5500002AB52EA030100F0E180DDE90001DDE920
:10B5600002ABCDE904018018594182457BEB010E05
:10B5700011DBBAEB000A6BEB010BCDE902ABDDE9A5
:10B5800004AB12EB020E43EB03001AEB0E0A4BEB7B
:10B59000000BCDE900ABDDE90001920849104FEA4C
:10B5A000300042EA8372CDE900019B10D1E700BF71
:10B5B00000080240F00F0120000C01204FF0FF3A7C
:10B5C0004FF0FF3BC820AAFB002300FB0B3E5FFAB5
:10B5D00089F3A2FB03AB03FB0EB0BAF1000F70F1CD
:10B5E000000305DA40F2FF1200211AEB020A48417B
:10B5F0004FEA5A2343EAC0524FEA602A002A7AF1FE
:10B600000001C0F2898012F500504AF1000B810B55
:10B6100041EA8B4395F815C0D4F8F020D8F8A81A61
:10B6200000910CF10400A2EB4020069998F8A5AA1D
:10B63000C7F89000FF2B98F8AC0A87F88A0028BF5B
:10B64000FF230AFB01F0009987F887307B79C7F860
:10B650008C2001FB09FEBEFBF0FB98F8AD0A87F8D1
:10B6600089B087F88B003BB10C2B8CBF4FF0020BDD
:10B670004FF0010B5B44DB00D5F81CC029499CF856
:10B6800000E09CF80100D1F8D419734403F1FF3BAA
:10B690009BFBFEF300FB03F0703009F1FF330AFB64
:10B6A0000030B0FBF9F902EB4922C7F8942049B108
:10B6B0001D4A536983F0080040F400239361384623
:10B6C0008847E863B8F8967118484FF400210137AD
:10B6D0004FF48012A8F896714FF4001381614FF473
:10B6E000800782614FF400010222836187618161DA
:10B6F000826198F8180498F8193403287EF442AF50
:10B70000002B7EF43FAF0127D8F8101488F8197485
:10B71000C8F81C14FEF736BF00237BE700988CFBAB
:10B7200000AB4FE738110120000002400008024042
:10B73000F0B4860743D0541E002A3ED0CAB2034656
:10B7400002E014F1FF3438D303F8012B9D07F8D140
:10B75000032C2BD9CDB245EA05250F2C45EA05452A
:10B7600016D9A4F110073F0903F1200606EB0716CE
:10B7700003F1100242E9045542E902551032B24287
:10B78000F8D104F00F040137032C03EB07130DD994
:10B790001E462246043A032A46F8045BFAD8221FC2
:10B7A00022F003020432134404F003042CB1C9B2A2
:10B7B0001C4403F8011B9C42FBD1F0BC70471446AB
:10B7C0000346C5E740EA01039B0770B42AD1032A68
:10B7D00028D90C460346214654F8046BA6F10135DE
:10B7E00025EA060515F0803F06D1043A032A43F8FE
:10B7F000046B2146EFD89AB10C781C70013A0133E2
:10B800003CB16AB111F8014F03F8014B013A002C29
:10B81000F7D12AB11A44002103F8011B9342FBD14E
:08B8200070BC70470346E6E727
:10B82800034AD2F89C300133C2F89C30704700BFFD
:10B838004000012008B5F6F70DFA00BF80B50B4BA4
:10B848000B4A96B01968914200AF15D1094C1C609B
:10B85800A3F5CA3CACF5847E8EF30888AEF5953521
:10B86800A5F1F40630688047FEE700BF00C001205C
:10B87800AD700DB0EFBEADDEBD48BE4ED0F888400D
:10B88800BD4ABE4D44F47003C0F8883031680024C6
:10B8980041F001033360B460316821F0847C2CF4FA
:10B8A8008033336072603268B54B22F480214FF0E8
:10B8B80000623160F46082608560D0F88860B14DC4
:10B8C80046F47004AB42C0F8884055D20335181DC1
:10B8D800291A21F003021518EE1A341FA1080131A4
:10B8E80011F00702A84C29D0012A21D0022A1BD026
:10B8F800032A15D0042A0FD0052A09D0062A03D016
:10B9080054F8046B1E60034654F8040B43F8040B08
:10B9180054F8041B43F8041B54F8042B43F8042B75
:10B9280054F8046B43F8046B54F8040B43F8040B05
:10B9380054F8041B43F8041BAB421DD0A6469C4692
:10B948005EF8042BE068DEF800104CF8042BA668BB
:10B9580059602269A1697860203454F80C0CCCF83D
:10B9680004601A617E6854F8042CDE60DA61C3E969
:10B9780005012033AB42E1D1844B854DAB4238D22F
:10B9880003351C1D281B20F003062644F11A0A1F44
:10B998009508013515F007014FF000001BD001296B
:10B9A80015D0022911D003290DD0042909D0052961
:10B9B80005D0062901D01860234643F8040B43F844
:10B9C800040B43F8040B43F8040B43F8040B43F847
:10B9D800040BB3420DD09E464EF8040B5860CEF8C7
:10B9E8000400D861C3E90300C3E905002033B3426A
:10B9F800F1D1684E684D34685D49684844F4007276
:10BA080032603468EB6A44F480623260346844F42B
:10BA180080723260CE684FF6FF0426404FF47A7C7D
:10BA2800B3FBFCFE0EF1FF333043B3F1807FC860F7
:10BA380008D25B4AF02600200724536081F823606F
:10BA48009060146000220F214FF0FF30F4F7D2FD10
:10BA58000024484AFC60116C524B534E41F0805010
:10BA68001064126C02F08051F960FA68BC601868C2
:10BA780040F440421A601B6803F44041B960012356
:10BA88004FF48000BA68336010214FF4B47C02266A
:10BA98003864072207F12400C7E909337964C7E944
:10BAA80012C6FE633A65F7F79DFC4FF4A0514FF4B8
:10BAB800805CC7E9071C0F20364B7E61BC6138618A
:10BAC8001C680440042C40F20681052107F110008F
:10BAD800F7F73AFE274B996801F00C04082C00F0A0
:10BAE800E480324EEE62234E3149B068314B324C1D
:10BAF800EA6AC0F3031E71441E1B91F8B416002EA7
:10BB080022FA01F2EA624FEAA60576DD681E54F8C9
:10BB1800043B7D6000F00706984779680125A94233
:10BB28006BDD002E51D0012E48D0022E1BD0032EE3
:10BB380015D0042E0FD0052E09D0062E03D054F8A8
:10BB4800045BA847022554F8042B9047013554F8A4
:10BB5800040B8047013554F8043B9847013554F8E5
:10BB6800046BB047013554F8041B8847013525E0BC
:10BB780000ED00E00038024010300024000000080A
:10BB88000000002040000120F812030840000120B6
:10BB980058440120003C0240000000200003FA0540
:10BBA80010E000E0007000404C0047420024F40020
:10BBB800D0220108F8120308F812030854F8042BDD
:10BBC800904778680135A84217DD2646083556F8AB
:10BBD800043B98476168884772689047E0688047E7
:10BBE8002669B04763699847A1698847E269904721
:10BBF8007868A84204F12004E7DC3B4D3B4C2E1B3F
:10BC0800002E4FEAA6034EDD591E54F8040B7B6044
:10BC180001F0070680477B680125AB4243DD56B338
:10BC2800012E21D0022E1BD0032E15D0042E0FD0AA
:10BC3800052E09D0062E03D054F8045BA847022528
:10BC480054F8042B9047013554F8041B88470135F4
:10BC580054F8040B8047013554F8046BB04701359C
:10BC680054F8043B9847013554F8042B90477968F9
:10BC78000135A94217DD2646083556F8040B8047DA
:10BC88006368984772689047E16888472669B047B3
:10BC980060698047A3699847E26990477968A94233
:10BCA80004F12004E7DCFCF7B5FE59685A685968C6
:10BCB8000F4B02F03F000F4AB3FBF0F45068C1F39A
:10BCC8008816C0F30141013104FB06F44B00B4FBB4
:10BCD800F3F4EC6207E705261E701A6802F00F00FD
:10BCE800B0427FF4F7AEF0E6F8120308F812030842
:08BCF8000024F40000380240B2
:10BD000000061016000610160D000B0008000700B4
:10BD10000400020001000E00AAAA66661E1EFE01B3
:10BD2000FFFF0000AA0066001E00FF00D506B30555
:10BD300000048F030002000180007F00400020000B
:10BD40001000080004000200010069070100010161
:10BD500001020103010401050106010701080109AF
:10BD6000010A010B010C010D010E010F011001115F
:10BD70000112000004080000C50F00085D13000850
:10BD80000B100000051400082912000800800000B4
:10BD9000AAAA00000000000001020304010203043B
:10BDA000060708097C290108802901083C0A0308C4
:10BDB000A0CE00083C0203083CFA0208A0DE0008FE
:10BDC00070BE000870C600083CF202083CEA020897
:10BDD000A0E600083CE202083CDA02083CD2020875
:10BDE0003CCA0208A0D600083CC202083CBA0208BD
:10BDF0003CB202083CAA0208A0F600083CA20208D5
:10BE00003C9A02083C9202083C8A0208A0060108FB
:10BE10003C8202083C7A02083C7202083C6A020832
:10BE2000A0FE00083C6202083C5A0208A0EE00088E
:10BE30003C5202083C4A02083C4202083C3A0208D2
:10BE40003C3202083C2A02083C2202083C1A020842
:10BE50003C1202083C0A02083C0202083CFA0108B3
:10BE60003CF201083CEA01083CE201083CDA010826
:10BE70000000004074325F27143E74F0EF197EC555
:10BE8000D5E18FC7F2C00FF595D0FA2AB504D33F9C
:10BE900036358E23C53CEDEB8F15BEC3C3DDEEC931
:10BEA0004FC0BBF9DFD35A2E64094E3FAF378B1F0B
:10BEB000203B83E7111152C2E1D999CC05C06EFE37
:10BEC00067D77931050E713EDA395D1B2A393AE3BD
:10BED0007C0C3BC133D68ACF14C0230326DB5334FA
:10BEE00094123E3DB63B0817E53619DFD5077CC0F6
:10BEF000BFD2BFD27CC0D50719DFE5360817B63BE5
:10BF00003E3D9412533426DB230314C08ACF33D62C
:10BF10003BC17C0C3AE32A395D1BDA39713E050ED0
:10BF2000793167D76EFE05C099CCE1D952C21111A3
:10BF300083E7203B8B1FAF374E3F64095A2EDFD378
:10BF4000BBF94FC0EEC9C3DDBEC38F15EDEBC53CD9
:10BF50008E233635D33FB504FA2A95D00FF5F2C0BB
:10BF60008FC7D5E17EC5EF1974F0143E5F27743298
:10BF7000004000005F278CCD74F0ECC17EC511E657
:10BF80008FC72B1E0FF50E3FFA2A6B2FD33F4BFBAB
:10BF90008E23CACAEDEB3BC3BEC371EAEEC93D2294
:10BFA000BBF9B13F5A2E212C4E3F9CF68B1F51C836
:10BFB00083E7E0C452C2EFEE99CC1F266EFEFB3F32
:10BFC00079319928713EFBF15D1B26C63AE3D6C64E
:10BFD0003BC184F38ACFCD292303EC3F5334DA24C9
:10BFE0003E3D6CED08174AC419DF1BC97CC02BF815
:10BFF000BFD2412DD507843FE536E720B63BF8E8B0
:10C000009412C2C226DBADCB14C0DDFC33D6763031
:10C010007C0CC53E2A39C61CDA39A3E4050E8FC153
:10C0200067D787CE05C09201E1D967331111AE3DC4
:10C03000203B7D18AF3775E06409B2C0DFD3A6D1CD
:10C040004FC04506C3DD12368F15423CC53C131464
:10C05000363572DCB5042DC095D006D5F2C0F10A94
:10C06000D5E17138EF19823A143E8C0F7432A1D8A1
:10C07000000000C08CCDA1D8ECC18C0F11E6823A33
:10C080002B1E71380E3FF10A6B2F06D54BFB2DC0CE
:10C09000CACA72DC3BC3131471EA423C3D22123619
:10C0A000B13F4506212CA6D19CF6B2C051C875E01F
:10C0B000E0C47D18EFEEAE3D1F266733FB3F9201D3
:10C0C000992887CEFBF18FC126C6A3E4D6C6C61C2D
:10C0D00084F3C53ECD297630EC3FDDFCDA24ADCBD0
:10C0E0006CEDC2C24AC4F8E81BC9E7202BF8843FB4
:10C0F000412D412D843F2BF8E7201BC9F8E84AC4A5
:10C10000C2C26CEDADCBDA24DDFCEC3F7630CD293C
:10C11000C53E84F3C61CD6C6A3E426C68FC1FBF178
:10C1200087CE99289201FB3F67331F26AE3DEFEE85
:10C130007D18E0C475E051C8B2C09CF6A6D1212C90
:10C140004506B13F12363D22423C71EA13143BC30F
:10C1500072DCCACA2DC04BFB06D56B2FF10A0E3F0D
:10C1600071382B1E823A11E68C0FECC1A1D88CCD10
:10C1700000C00000A1D874328C0F143E823AEF192F
:10C180007138D5E1F10AF2C006D595D02DC0B504BD
:10C1900072DC36351314C53C423C8F151236C3DDB4
:10C1A00045064FC0A6D1DFD3B2C0640975E0AF37F2
:10C1B0007D18203BAE3D11116733E1D9920105C0D6
:10C1C00087CE67D78FC1050EA3E4DA39C61C2A399A
:10C1D000C53E7C0C763033D6DDFC14C0ADCB26DBFF
:10C1E000C2C29412F8E8B63BE720E536843FD50793
:10C1F000412DBFD22BF87CC01BC919DF4AC40817D8
:10C200006CED3E3DDA245334EC3F2303CD298ACF35
:10C2100084F33BC1D6C63AE326C65D1BFBF1713EF3
:10C2200099287931FB3F6EFE1F2699CCEFEE52C262
:10C23000E0C483E751C88B1F9CF64E3F212C5A2E39
:10C24000B13FBBF93D22EEC971EABEC33BC3EDEB82
:10C25000CACA8E234BFBD33F6B2FFA2A0E3F0FF532
:10C260002B1E8FC711E67EC5ECC174F08CCD5F2705
:10C270000000004074325F27143E74F0EF197EC551
:10C28000D5E18FC7F2C00FF595D0FA2AB504D33F98
:10C2900036358E23C53CEDEB8F15BEC3C3DDEEC92D
:10C2A0004FC0BBF9DFD35A2E64094E3FAF378B1F07
:10C2B000203B83E7111152C2E1D999CC05C06EFE33
:10C2C00067D77931050E713EDA395D1B2A393AE3B9
:10C2D0007C0C3BC133D68ACF14C0230326DB5334F6
:10C2E00094123E3DB63B0817E53619DFD5077CC0F2
:10C2F000BFD2BFD27CC0D50719DFE5360817B63BE1
:10C300003E3D9412533426DB230314C08ACF33D628
:10C310003BC17C0C3AE32A395D1BDA39713E050ECC
:10C32000793167D76EFE05C099CCE1D952C211119F
:10C3300083E7203B8B1FAF374E3F64095A2EDFD374
:10C34000BBF94FC0EEC9C3DDBEC38F15EDEBC53CD5
:10C350008E233635D33FB504FA2A95D00FF5F2C0B7
:10C360008FC7D5E17EC5EF1974F0143E5F27743294
:10C37000004000005F278CCD74F0ECC17EC511E653
:10C380008FC72B1E0FF50E3FFA2A6B2FD33F4BFBA7
:10C390008E23CACAEDEB3BC3BEC371EAEEC93D2290
:10C3A000BBF9B13F5A2E212C4E3F9CF68B1F51C832
:10C3B00083E7E0C452C2EFEE99CC1F266EFEFB3F2E
:10C3C00079319928713EFBF15D1B26C63AE3D6C64A
:10C3D0003BC184F38ACFCD292303EC3F5334DA24C5
:10C3E0003E3D6CED08174AC419DF1BC97CC02BF811
:10C3F000BFD2412DD507843FE536E720B63BF8E8AC
:10C400009412C2C226DBADCB14C0DDFC33D676302D
:10C410007C0CC53E2A39C61CDA39A3E4050E8FC14F
:10C4200067D787CE05C09201E1D967331111AE3DC0
:10C43000203B7D18AF3775E06409B2C0DFD3A6D1C9
:10C440004FC04506C3DD12368F15423CC53C131460
:10C45000363572DCB5042DC095D006D5F2C0F10A90
:10C46000D5E17138EF19823A143E8C0F7432A1D89D
:10C47000000000C08CCDA1D8ECC18C0F11E6823A2F
:10C480002B1E71380E3FF10A6B2F06D54BFB2DC0CA
:10C49000CACA72DC3BC3131471EA423C3D22123615
:10C4A000B13F4506212CA6D19CF6B2C051C875E01B
:10C4B000E0C47D18EFEEAE3D1F266733FB3F9201CF
:10C4C000992887CEFBF18FC126C6A3E4D6C6C61C29
:10C4D00084F3C53ECD297630EC3FDDFCDA24ADCBCC
:10C4E0006CEDC2C24AC4F8E81BC9E7202BF8843FB0
:10C4F000412D412D843F2BF8E7201BC9F8E84AC4A1
:10C50000C2C26CEDADCBDA24DDFCEC3F7630CD2938
:10C51000C53E84F3C61CD6C6A3E426C68FC1FBF174
:10C5200087CE99289201FB3F67331F26AE3DEFEE81
:10C530007D18E0C475E051C8B2C09CF6A6D1212C8C
:10C540004506B13F12363D22423C71EA13143BC30B
:10C5500072DCCACA2DC04BFB06D56B2FF10A0E3F09
:10C5600071382B1E823A11E68C0FECC1A1D88CCD0C
:10C5700000C00000A1D874328C0F143E823AEF192B
:10C580007138D5E1F10AF2C006D595D02DC0B504B9
:10C5900072DC36351314C53C423C8F151236C3DDB0
:10C5A00045064FC0A6D1DFD3B2C0640975E0AF37EE
:10C5B0007D18203BAE3D11116733E1D9920105C0D2
:10C5C00087CE67D78FC1050EA3E4DA39C61C2A3996
:10C5D000C53E7C0C763033D6DDFC14C0ADCB26DBFB
:10C5E000C2C29412F8E8B63BE720E536843FD5078F
:10C5F000412DBFD22BF87CC01BC919DF4AC40817D4
:10C600006CED3E3DDA245334EC3F2303CD298ACF31
:10C6100084F33BC1D6C63AE326C65D1BFBF1713EEF
:10C6200099287931FB3F6EFE1F2699CCEFEE52C25E
:10C63000E0C483E751C88B1F9CF64E3F212C5A2E35
:10C64000B13FBBF93D22EEC971EABEC33BC3EDEB7E
:10C65000CACA8E234BFBD33F6B2FFA2A0E3F0FF52E
:10C660002B1E8FC711E67EC5ECC174F08CCD5F2701
:10C670000000004067331F263E3D6CED8F15BEC3A2
:10C6800072DCCACA14C0DDFC67D779318C0F143E46
:10C69000203B7D18E53619DF45064FC095D006D5FD
:10C6A0003BC17C0CA3E4DA392B1E71384E3F640980
:10C6B000412DBFD29CF6B2C08FC7D5E126C65D1B07
:10C6C00084F3C53EFA2A6B2FB13FBBF9E7201BC9A3
:10C6D00083E7E0C4ECC174F087CE99282303EC3FD4
:10C6E00036358E23423C71EA9412C2C2E1D999CC0C
:10C6F00000C00000E1D9673394123E3D423C8F15E3
:10C70000363572DC230314C087CE67D7ECC18C0F9B
:10C7100083E7203BE720E536B13F4506FA2A95D06E
:10C7200084F33BC126C6A3E48FC72B1E9CF64E3F65
:10C73000412D412D4E3F9CF62B1E8FC7A3E426C6EC
:10C740003BC184F395D0FA2A4506B13FE536E72090
:10C75000203B83E78C0FECC167D787CE14C023033F
:10C7600072DC36358F15423C3E3D94126733E1D979
:10C77000000000C099CCE1D9C2C2941271EA423CD7
:10C780008E233635EC3F2303992887CE74F0ECC115
:10C79000E0C483E71BC9E720BBF9B13F6B2FFA2A3E
:10C7A000C53E84F35D1B26C6D5E18FC7B2C09CF69B
:10C7B000BFD2412D64094E3F71382B1EDA39A3E4F4
:10C7C0007C0C3BC106D595D04FC0450619DFE53638
:10C7D0007D18203B143E8C0F793167D7DDFC14C0E7
:10C7E000CACA72DCBEC38F156CED3E3D1F2667338F
:10C7F000004000001F2699CC6CEDC2C2BEC371EA96
:10C80000CACA8E23DDFCEC3F79319928143E74F0BE
:10C810007D18E0C419DF1BC94FC0BBF906D56B2FCB
:10C820007C0CC53EDA395D1B7138D5E16409B2C0B4
:10C83000BFD2BFD2B2C06409D5E171385D1BDA390D
:10C84000C53E7C0C6B2F06D5BBF94FC01BC919DF49
:10C85000E0C47D1874F0143E99287931EC3FDDFC7A
:10C860008E23CACA71EABEC3C2C26CED99CC1F2620
:10C870000000004067331F263E3D6CED8F15BEC3A0
:10C8800072DCCACA14C0DDFC67D779318C0F143E44
:10C89000203B7D18E53619DF45064FC095D006D5FB
:10C8A0003BC17C0CA3E4DA392B1E71384E3F64097E
:10C8B000412DBFD29CF6B2C08FC7D5E126C65D1B05
:10C8C00084F3C53EFA2A6B2FB13FBBF9E7201BC9A1
:10C8D00083E7E0C4ECC174F087CE99282303EC3FD2
:10C8E00036358E23423C71EA9412C2C2E1D999CC0A
:10C8F00000C00000E1D9673394123E3D423C8F15E1
:10C90000363572DC230314C087CE67D7ECC18C0F99
:10C9100083E7203BE720E536B13F4506FA2A95D06C
:10C9200084F33BC126C6A3E48FC72B1E9CF64E3F63
:10C93000412D412D4E3F9CF62B1E8FC7A3E426C6EA
:10C940003BC184F395D0FA2A4506B13FE536E7208E
:10C95000203B83E78C0FECC167D787CE14C023033D
:10C9600072DC36358F15423C3E3D94126733E1D977
:10C97000000000C099CCE1D9C2C2941271EA423CD5
:10C980008E233635EC3F2303992887CE74F0ECC113
:10C99000E0C483E71BC9E720BBF9B13F6B2FFA2A3C
:10C9A000C53E84F35D1B26C6D5E18FC7B2C09CF699
:10C9B000BFD2412D64094E3F71382B1EDA39A3E4F2
:10C9C0007C0C3BC106D595D04FC0450619DFE53636
:10C9D0007D18203B143E8C0F793167D7DDFC14C0E5
:10C9E000CACA72DCBEC38F156CED3E3D1F2667338D
:10C9F000004000001F2699CC6CEDC2C2BEC371EA94
:10CA0000CACA8E23DDFCEC3F79319928143E74F0BC
:10CA10007D18E0C419DF1BC94FC0BBF906D56B2FC9
:10CA20007C0CC53EDA395D1B7138D5E16409B2C0B2
:10CA3000BFD2BFD2B2C06409D5E171385D1BDA390B
:10CA4000C53E7C0C6B2F06D5BBF94FC01BC919DF47
:10CA5000E0C47D1874F0143E99287931EC3FDDFC78
:10CA60008E23CACA71EABEC3C2C26CED99CC1F261E
:10CA70000000004067331F263E3D6CED8F15BEC39E
:10CA800072DCCACA14C0DDFC67D779318C0F143E42
:10CA9000203B7D18E53619DF45064FC095D006D5F9
:10CAA0003BC17C0CA3E4DA392B1E71384E3F64097C
:10CAB000412DBFD29CF6B2C08FC7D5E126C65D1B03
:10CAC00084F3C53EFA2A6B2FB13FBBF9E7201BC99F
:10CAD00083E7E0C4ECC174F087CE99282303EC3FD0
:10CAE00036358E23423C71EA9412C2C2E1D999CC08
:10CAF00000C00000E1D9673394123E3D423C8F15DF
:10CB0000363572DC230314C087CE67D7ECC18C0F97
:10CB100083E7203BE720E536B13F4506FA2A95D06A
:10CB200084F33BC126C6A3E48FC72B1E9CF64E3F61
:10CB3000412D412D4E3F9CF62B1E8FC7A3E426C6E8
:10CB40003BC184F395D0FA2A4506B13FE536E7208C
:10CB5000203B83E78C0FECC167D787CE14C023033B
:10CB600072DC36358F15423C3E3D94126733E1D975
:10CB7000000000C099CCE1D9C2C2941271EA423CD3
:10CB80008E233635EC3F2303992887CE74F0ECC111
:10CB9000E0C483E71BC9E720BBF9B13F6B2FFA2A3A
:10CBA000C53E84F35D1B26C6D5E18FC7B2C09CF697
:10CBB000BFD2412D64094E3F71382B1EDA39A3E4F0
:10CBC0007C0C3BC106D595D04FC0450619DFE53634
:10CBD0007D18203B143E8C0F793167D7DDFC14C0E3
:10CBE000CACA72DCBEC38F156CED3E3D1F2667338B
:10CBF000004000001F2699CC6CEDC2C2BEC371EA92
:10CC0000CACA8E23DDFCEC3F79319928143E74F0BA
:10CC10007D18E0C419DF1BC94FC0BBF906D56B2FC7
:10CC20007C0CC53EDA395D1B7138D5E16409B2C0B0
:10CC3000BFD2BFD2B2C06409D5E171385D1BDA3909
:10CC4000C53E7C0C6B2F06D5BBF94FC01BC919DF45
:10CC5000E0C47D1874F0143E99287931EC3FDDFC76
:10CC60008E23CACA71EABEC3C2C26CED99CC1F261C
:10CC70000000004067331F263E3D6CED8F15BEC39C
:10CC800072DCCACA14C0DDFC67D779318C0F143E40
:10CC9000203B7D18E53619DF45064FC095D006D5F7
:10CCA0003BC17C0CA3E4DA392B1E71384E3F64097A
:10CCB000412DBFD29CF6B2C08FC7D5E126C65D1B01
:10CCC00084F3C53EFA2A6B2FB13FBBF9E7201BC99D
:10CCD00083E7E0C4ECC174F087CE99282303EC3FCE
:10CCE00036358E23423C71EA9412C2C2E1D999CC06
:10CCF00000C00000E1D9673394123E3D423C8F15DD
:10CD0000363572DC230314C087CE67D7ECC18C0F95
:10CD100083E7203BE720E536B13F4506FA2A95D068
:10CD200084F33BC126C6A3E48FC72B1E9CF64E3F5F
:10CD3000412D412D4E3F9CF62B1E8FC7A3E426C6E6
:10CD40003BC184F395D0FA2A4506B13FE536E7208A
:10CD5000203B83E78C0FECC167D787CE14C0230339
:10CD600072DC36358F15423C3E3D94126733E1D973
:10CD7000000000C099CCE1D9C2C2941271EA423CD1
:10CD80008E233635EC3F2303992887CE74F0ECC10F
:10CD9000E0C483E71BC9E720BBF9B13F6B2FFA2A38
:10CDA000C53E84F35D1B26C6D5E18FC7B2C09CF695
:10CDB000BFD2412D64094E3F71382B1EDA39A3E4EE
:10CDC0007C0C3BC106D595D04FC0450619DFE53632
:10CDD0007D18203B143E8C0F793167D7DDFC14C0E1
:10CDE000CACA72DCBEC38F156CED3E3D1F26673389
:10CDF000004000001F2699CC6CEDC2C2BEC371EA90
:10CE0000CACA8E23DDFCEC3F79319928143E74F0B8
:10CE10007D18E0C419DF1BC94FC0BBF906D56B2FC5
:10CE20007C0CC53EDA395D1B7138D5E16409B2C0AE
:10CE3000BFD2BFD2B2C06409D5E171385D1BDA3907
:10CE4000C53E7C0C6B2F06D5BBF94FC01BC919DF43
:10CE5000E0C47D1874F0143E99287931EC3FDDFC74
:10CE60008E23CACA71EABEC3C2C26CED99CC1F261A
:10CE700001000201000201000201000200030102A0
:10CE800001030100020302000306080B0D10121536
:10CE9000171A1C1F0205070A0C0F111416191B1E66
:10CEA000000000405A2E212CEC3FDDFCCD298ACF1A
:10CEB000BBF94FC08CCDA1D8B2C0640926DB533476
:10CEC0007C0CC53E12363D22143E74F08B1F51C8B7
:10CED0006CEDC2C2D6C63AE3BEC38F1511E6823AE4
:10CEE0007D18203BB63B0817DA39A3E413143BC383
:10CEF000D5E18FC752C2EFEE1BC9E720FBF1713EAF
:10CF00008E2336350E3FF10A6733E1D9D5077CC051
:10CF100067D787CE2DC04BFB95D0FA2A6EFEFB3F1C
:10CF2000412D412DFB3F6EFEFA2A95D04BFB2DC0C3
:10CF300087CE67D77CC0D507E1D96733F10A0E3FAA
:10CF400036358E23713EFBF1E7201BC9EFEE52C24E
:10CF50008FC7D5E13BC31314A3E4DA390817B63BF6
:10CF6000203B7D18823A11E68F15BEC33AE3D6C640
:10CF7000C2C26CED51C88B1F74F0143E3D221236B4
:10CF8000C53E7C0C533426DB6409B2C0A1D88CCDDD
:10CF90004FC0BBF98ACFCD29DDFCEC3F212C5A2EA6
:10CFA00000400000212CA6D1DDFC14C08ACF33D66E
:10CFB0004FC04506A1D8743264094E3F5334DA2479
:10CFC000C53E84F33D22EEC974F0ECC151C875E052
:10CFD000C2C294123AE32A398F15423C823AEF19C1
:10CFE000203B83E708174AC4A3E426C63BC3EDEB06
:10CFF0008FC72B1EEFEEAE3DE720E536713E050EE6
:10D00000363572DCF10AF2C0E1D999CC7CC02BF83C
:10D0100087CE99284BFBD33FFA2A6B2FFB3F920117
:10D02000412DBFD26EFE05C095D006D52DC0B504EA
:10D0300067D77931D507843F67331F260E3F0FF539
:10D040008E23CACAFBF18FC11BC919DF52C211114D
:10D05000D5E171381314C53CDA395D1BB63BF8E8ED
:10D060007D18E0C411E67EC5BEC371EAD6C6C61CF3
:10D070006CED3E3D8B1FAF37143E8C0F1236C3DD77
:10D080007C0C3BC126DBADCBB2C09CF68CCD5F27C0
:10D09000BBF9B13FCD297630EC3F23035A2EDFD3C5
:10D0A000000000C0A6D1DFD314C0230333D67630EE
:10D0B0004506B13F74325F274E3F9CF6DA24ADCB74
:10D0C00084F33BC1EEC9C3DDECC18C0F75E0AF3713
:10D0D00094123E3D2A39C61C423C71EAEF197EC5C6
:10D0E00083E7E0C44AC4F8E826C65D1BEDEBC53C07
:10D0F0002B1E7138AE3D1111E53619DF050E8FC1BB
:10D1000072DCCACAF2C00FF599CC1F262BF8843FF7
:10D1100099287931D33FB5046B2F06D5920105C00C
:10D12000BFD2BFD205C0920106D56B2FB504D33F45
:10D1300079319928843F2BF81F2699CC0FF5F2C03E
:10D14000CACA72DC8FC1050E19DFE5361111AE3D7A
:10D1500071382B1EC53CEDEB5D1B26C6F8E84AC4B2
:10D16000E0C483E77EC5EF1971EA423CC61C2A3948
:10D170003E3D9412AF3775E08C0FECC1C3DDEEC9B4
:10D180003BC184F3ADCBDA249CF64E3F5F2774326B
:10D19000B13F4506763033D6230314C0DFD3A6D182
:10D1A00000C00000DFD35A2E2303EC3F7630CD2998
:10D1B000B13FBBF95F278CCD9CF6B2C0ADCB26DB6F
:10D1C0003BC17C0CC3DD12368C0F143EAF378B1F76
:10D1D0003E3D6CEDC61CD6C671EABEC37EC511E6E7
:10D1E000E0C47D18F8E8B63B5D1BDA39C53C131482
:10D1F0007138D5E1111152C219DF1BC98FC1FBF182
:10D20000CACA8E230FF50E3F1F266733843FD5070A
:10D21000793167D7B5042DC006D595D005C06EFE0F
:10D22000BFD2412D9201FB3F6B2FFA2AD33F4BFB1C
:10D23000992887CE2BF87CC099CCE1D9F2C0F10AAD
:10D2400072DC3635050E713EE536E720AE3DEFEE79
:10D250002B1E8FC7EDEB3BC326C6A3E44AC40817B9
:10D2600083E7203BEF19823A423C8F152A393AE393
:10D270009412C2C275E051C8ECC174F0EEC93D22EF
:10D2800084F3C53EDA2453344E3F64097432A1D886
:10D2900045064FC033D68ACF14C0DDFCA6D1212C61
:10D2A000000000405A2E212CEC3FDDFCCD298ACF16
:10D2B000BBF94FC08CCDA1D8B2C0640926DB533472
:10D2C0007C0CC53E12363D22143E74F08B1F51C8B3
:10D2D0006CEDC2C2D6C63AE3BEC38F1511E6823AE0
:10D2E0007D18203BB63B0817DA39A3E413143BC37F
:10D2F000D5E18FC752C2EFEE1BC9E720FBF1713EAB
:10D300008E2336350E3FF10A6733E1D9D5077CC04D
:10D3100067D787CE2DC04BFB95D0FA2A6EFEFB3F18
:10D32000412D412DFB3F6EFEFA2A95D04BFB2DC0BF
:10D3300087CE67D77CC0D507E1D96733F10A0E3FA6
:10D3400036358E23713EFBF1E7201BC9EFEE52C24A
:10D350008FC7D5E13BC31314A3E4DA390817B63BF2
:10D36000203B7D18823A11E68F15BEC33AE3D6C63C
:10D37000C2C26CED51C88B1F74F0143E3D221236B0
:10D38000C53E7C0C533426DB6409B2C0A1D88CCDD9
:10D390004FC0BBF98ACFCD29DDFCEC3F212C5A2EA2
:10D3A00000400000212CA6D1DDFC14C08ACF33D66A
:10D3B0004FC04506A1D8743264094E3F5334DA2475
:10D3C000C53E84F33D22EEC974F0ECC151C875E04E
:10D3D000C2C294123AE32A398F15423C823AEF19BD
:10D3E000203B83E708174AC4A3E426C63BC3EDEB02
:10D3F0008FC72B1EEFEEAE3DE720E536713E050EE2
:10D40000363572DCF10AF2C0E1D999CC7CC02BF838
:10D4100087CE99284BFBD33FFA2A6B2FFB3F920113
:10D42000412DBFD26EFE05C095D006D52DC0B504E6
:10D4300067D77931D507843F67331F260E3F0FF535
:10D440008E23CACAFBF18FC11BC919DF52C2111149
:10D45000D5E171381314C53CDA395D1BB63BF8E8E9
:10D460007D18E0C411E67EC5BEC371EAD6C6C61CEF
:10D470006CED3E3D8B1FAF37143E8C0F1236C3DD73
:10D480007C0C3BC126DBADCBB2C09CF68CCD5F27BC
:10D49000BBF9B13FCD297630EC3F23035A2EDFD3C1
:10D4A000000000C0A6D1DFD314C0230333D67630EA
:10D4B0004506B13F74325F274E3F9CF6DA24ADCB70
:10D4C00084F33BC1EEC9C3DDECC18C0F75E0AF370F
:10D4D00094123E3D2A39C61C423C71EAEF197EC5C2
:10D4E00083E7E0C44AC4F8E826C65D1BEDEBC53C03
:10D4F0002B1E7138AE3D1111E53619DF050E8FC1B7
:10D5000072DCCACAF2C00FF599CC1F262BF8843FF3
:10D5100099287931D33FB5046B2F06D5920105C008
:10D52000BFD2BFD205C0920106D56B2FB504D33F41
:10D5300079319928843F2BF81F2699CC0FF5F2C03A
:10D54000CACA72DC8FC1050E19DFE5361111AE3D76
:10D5500071382B1EC53CEDEB5D1B26C6F8E84AC4AE
:10D56000E0C483E77EC5EF1971EA423CC61C2A3944
:10D570003E3D9412AF3775E08C0FECC1C3DDEEC9B0
:10D580003BC184F3ADCBDA249CF64E3F5F27743267
:10D59000B13F4506763033D6230314C0DFD3A6D17E
:10D5A00000C00000DFD35A2E2303EC3F7630CD2994
:10D5B000B13FBBF95F278CCD9CF6B2C0ADCB26DB6B
:10D5C0003BC17C0CC3DD12368C0F143EAF378B1F72
:10D5D0003E3D6CEDC61CD6C671EABEC37EC511E6E3
:10D5E000E0C47D18F8E8B63B5D1BDA39C53C13147E
:10D5F0007138D5E1111152C219DF1BC98FC1FBF17E
:10D60000CACA8E230FF50E3F1F266733843FD50706
:10D61000793167D7B5042DC006D595D005C06EFE0B
:10D62000BFD2412D9201FB3F6B2FFA2AD33F4BFB18
:10D63000992887CE2BF87CC099CCE1D9F2C0F10AA9
:10D6400072DC3635050E713EE536E720AE3DEFEE75
:10D650002B1E8FC7EDEB3BC326C6A3E44AC40817B5
:10D6600083E7203BEF19823A423C8F152A393AE38F
:10D670009412C2C275E051C8ECC174F0EEC93D22EB
:10D6800084F3C53EDA2453344E3F64097432A1D882
:10D6900045064FC033D68ACF14C0DDFCA6D1212C5D
:10D6A00000000040DA395D1B793167D774F0ECC1B6
:10D6B0003BC184F3E1D967332B1E7138EC3FDDFCAD
:10D6C0007D18E0C406D595D0C2C294129CF64E3F98
:10D6D00036358E23E53619DFBBF94FC0BEC371EA7C
:10D6E000BFD2412D8F15423CB13F4506E7201BC9F3
:10D6F00072DCCACAB2C064096CED3E3D6B2FFA2AD7
:10D70000203B83E7230314C08FC7D5E199CC1F26A4
:10D710007C0CC53E143E8C0F992887CEA3E426C608
:10D7200000C00000A3E4DA3999287931143E74F07E
:10D730007C0C3BC199CCE1D98FC72B1E2303EC3F56
:10D74000203B7D186B2F06D56CEDC2C2B2C09CF693
:10D7500072DC3635E720E536B13FBBF98F15BEC325
:10D76000BFD2BFD2BEC38F15BBF9B13FE536E720AC
:10D77000363572DC9CF6B2C0C2C26CED06D56B2F9A
:10D780007D18203BEC3F23032B1E8FC7E1D999CC9A
:10D790003BC17C0C74F0143E79319928DA39A3E44A
:10D7A000000000C026C6A3E487CE99288C0F143E43
:10D7B000C53E7C0C1F2699CCD5E18FC714C023032E
:10D7C00083E7203BFA2A6B2F3E3D6CED6409B2C023
:10D7D000CACA72DC1BC9E7204506B13F423C8F151F
:10D7E000412DBFD271EABEC34FC0BBF919DFE53688
:10D7F0008E2336354E3F9CF69412C2C295D006D584
:10D80000E0C47D18DDFCEC3F71382B1E6733E1D995
:10D8100084F33BC1ECC174F067D779315D1BDA3911
:10D82000004000005D1B26C667D787CEECC18C0F79
:10D8300084F3C53E67331F267138D5E1DDFC14C083
:10D84000E0C483E795D0FA2A94123E3D4E3F640926
:10D850008E23CACA19DF1BC94FC0450671EA423C74
:10D86000412D412D423C71EA45064FC01BC919DFCD
:10D87000CACA8E2364094E3F3E3D9412FA2A95D0BF
:10D8800083E7E0C414C0DDFCD5E171381F2667339F
:10D89000C53E84F38C0FECC187CE67D726C65D1BCF
:10D8A00000000040DA395D1B793167D774F0ECC1B4
:10D8B0003BC184F3E1D967332B1E7138EC3FDDFCAB
:10D8C0007D18E0C406D595D0C2C294129CF64E3F96
:10D8D00036358E23E53619DFBBF94FC0BEC371EA7A
:10D8E000BFD2412D8F15423CB13F4506E7201BC9F1
:10D8F00072DCCACAB2C064096CED3E3D6B2FFA2AD5
:10D90000203B83E7230314C08FC7D5E199CC1F26A2
:10D910007C0CC53E143E8C0F992887CEA3E426C606
:10D9200000C00000A3E4DA3999287931143E74F07C
:10D930007C0C3BC199CCE1D98FC72B1E2303EC3F54
:10D94000203B7D186B2F06D56CEDC2C2B2C09CF691
:10D9500072DC3635E720E536B13FBBF98F15BEC323
:10D96000BFD2BFD2BEC38F15BBF9B13FE536E720AA
:10D97000363572DC9CF6B2C0C2C26CED06D56B2F98
:10D980007D18203BEC3F23032B1E8FC7E1D999CC98
:10D990003BC17C0C74F0143E79319928DA39A3E448
:10D9A000000000C026C6A3E487CE99288C0F143E41
:10D9B000C53E7C0C1F2699CCD5E18FC714C023032C
:10D9C00083E7203BFA2A6B2F3E3D6CED6409B2C021
:10D9D000CACA72DC1BC9E7204506B13F423C8F151D
:10D9E000412DBFD271EABEC34FC0BBF919DFE53686
:10D9F0008E2336354E3F9CF69412C2C295D006D582
:10DA0000E0C47D18DDFCEC3F71382B1E6733E1D993
:10DA100084F33BC1ECC174F067D779315D1BDA390F
:10DA2000004000005D1B26C667D787CEECC18C0F77
:10DA300084F3C53E67331F267138D5E1DDFC14C081
:10DA4000E0C483E795D0FA2A94123E3D4E3F640924
:10DA50008E23CACA19DF1BC94FC0450671EA423C72
:10DA6000412D412D423C71EA45064FC01BC919DFCB
:10DA7000CACA8E2364094E3F3E3D9412FA2A95D0BD
:10DA800083E7E0C414C0DDFCD5E171381F2667339D
:10DA9000C53E84F38C0FECC187CE67D726C65D1BCD
:10DAA00000000040DA395D1B793167D774F0ECC1B2
:10DAB0003BC184F3E1D967332B1E7138EC3FDDFCA9
:10DAC0007D18E0C406D595D0C2C294129CF64E3F94
:10DAD00036358E23E53619DFBBF94FC0BEC371EA78
:10DAE000BFD2412D8F15423CB13F4506E7201BC9EF
:10DAF00072DCCACAB2C064096CED3E3D6B2FFA2AD3
:10DB0000203B83E7230314C08FC7D5E199CC1F26A0
:10DB10007C0CC53E143E8C0F992887CEA3E426C604
:10DB200000C00000A3E4DA3999287931143E74F07A
:10DB30007C0C3BC199CCE1D98FC72B1E2303EC3F52
:10DB4000203B7D186B2F06D56CEDC2C2B2C09CF68F
:10DB500072DC3635E720E536B13FBBF98F15BEC321
:10DB6000BFD2BFD2BEC38F15BBF9B13FE536E720A8
:10DB7000363572DC9CF6B2C0C2C26CED06D56B2F96
:10DB80007D18203BEC3F23032B1E8FC7E1D999CC96
:10DB90003BC17C0C74F0143E79319928DA39A3E446
:10DBA000000000C026C6A3E487CE99288C0F143E3F
:10DBB000C53E7C0C1F2699CCD5E18FC714C023032A
:10DBC00083E7203BFA2A6B2F3E3D6CED6409B2C01F
:10DBD000CACA72DC1BC9E7204506B13F423C8F151B
:10DBE000412DBFD271EABEC34FC0BBF919DFE53684
:10DBF0008E2336354E3F9CF69412C2C295D006D580
:10DC0000E0C47D18DDFCEC3F71382B1E6733E1D991
:10DC100084F33BC1ECC174F067D779315D1BDA390D
:10DC2000004000005D1B26C667D787CEECC18C0F75
:10DC300084F3C53E67331F267138D5E1DDFC14C07F
:10DC4000E0C483E795D0FA2A94123E3D4E3F640922
:10DC50008E23CACA19DF1BC94FC0450671EA423C70
:10DC6000412D412D423C71EA45064FC01BC919DFC9
:10DC7000CACA8E2364094E3F3E3D9412FA2A95D0BB
:10DC800083E7E0C414C0DDFCD5E171381F2667339B
:10DC9000C53E84F38C0FECC187CE67D726C65D1BCB
:10DCA00000000040DA395D1B793167D774F0ECC1B0
:10DCB0003BC184F3E1D967332B1E7138EC3FDDFCA7
:10DCC0007D18E0C406D595D0C2C294129CF64E3F92
:10DCD00036358E23E53619DFBBF94FC0BEC371EA76
:10DCE000BFD2412D8F15423CB13F4506E7201BC9ED
:10DCF00072DCCACAB2C064096CED3E3D6B2FFA2AD1
:10DD0000203B83E7230314C08FC7D5E199CC1F269E
:10DD10007C0CC53E143E8C0F992887CEA3E426C602
:10DD200000C00000A3E4DA3999287931143E74F078
:10DD30007C0C3BC199CCE1D98FC72B1E2303EC3F50
:10DD4000203B7D186B2F06D56CEDC2C2B2C09CF68D
:10DD500072DC3635E720E536B13FBBF98F15BEC31F
:10DD6000BFD2BFD2BEC38F15BBF9B13FE536E720A6
:10DD7000363572DC9CF6B2C0C2C26CED06D56B2F94
:10DD80007D18203BEC3F23032B1E8FC7E1D999CC94
:10DD90003BC17C0C74F0143E79319928DA39A3E444
:10DDA000000000C026C6A3E487CE99288C0F143E3D
:10DDB000C53E7C0C1F2699CCD5E18FC714C0230328
:10DDC00083E7203BFA2A6B2F3E3D6CED6409B2C01D
:10DDD000CACA72DC1BC9E7204506B13F423C8F1519
:10DDE000412DBFD271EABEC34FC0BBF919DFE53682
:10DDF0008E2336354E3F9CF69412C2C295D006D57E
:10DE0000E0C47D18DDFCEC3F71382B1E6733E1D98F
:10DE100084F33BC1ECC174F067D779315D1BDA390B
:10DE2000004000005D1B26C667D787CEECC18C0F73
:10DE300084F3C53E67331F267138D5E1DDFC14C07D
:10DE4000E0C483E795D0FA2A94123E3D4E3F640920
:10DE50008E23CACA19DF1BC94FC0450671EA423C6E
:10DE6000412D412D423C71EA45064FC01BC919DFC7
:10DE7000CACA8E2364094E3F3E3D9412FA2A95D0B9
:10DE800083E7E0C414C0DDFCD5E171381F26673399
:10DE9000C53E84F38C0FECC187CE67D726C65D1BC9
:10DEA0000000004079319928C53E84F32B1E8FC7AE
:10DEB00083E7E0C4C2C26CEDCACA8E23BBF9B13F8E
:10DEC000412D412DB13FBBF98E23CACA6CEDC2C2B0
:10DED000E0C483E78FC72B1E84F3C53E99287931B0
:10DEE00000400000992887CE84F33BC18FC7D5E15D
:10DEF000E0C47D186CED3E3D8E233635B13F4506BE
:10DF0000412DBFD2BBF94FC0CACA72DCC2C2941243
:10DF100083E7203B2B1E7138C53E7C0C793167D7D7
:10DF2000000000C087CE67D73BC17C0CD5E17138BB
:10DF30007D18203B3E3D9412363572DC45064FC0BD
:10DF4000BFD2BFD24FC0450672DC363594123E3D7B
:10DF5000203B7D187138D5E17C0C3BC167D787CE5B
:10DF600000C0000067D779317C0CC53E71382B1E8C
:10DF7000203B83E79412C2C272DCCACA4FC0BBF90D
:10DF8000BFD2412D4506B13F36358E233E3D6CED67
:10DF90007D18E0C4D5E18FC73BC184F387CE9928B3
:10DFA0000000004079319928C53E84F32B1E8FC7AD
:10DFB00083E7E0C4C2C26CEDCACA8E23BBF9B13F8D
:10DFC000412D412DB13FBBF98E23CACA6CEDC2C2AF
:10DFD000E0C483E78FC72B1E84F3C53E99287931AF
:10DFE00000400000992887CE84F33BC18FC7D5E15C
:10DFF000E0C47D186CED3E3D8E233635B13F4506BD
:10E00000412DBFD2BBF94FC0CACA72DCC2C2941242
:10E0100083E7203B2B1E7138C53E7C0C793167D7D6
:10E02000000000C087CE67D73BC17C0CD5E17138BA
:10E030007D18203B3E3D9412363572DC45064FC0BC
:10E04000BFD2BFD24FC0450672DC363594123E3D7A
:10E05000203B7D187138D5E17C0C3BC167D787CE5A
:10E0600000C0000067D779317C0CC53E71382B1E8B
:10E07000203B83E79412C2C272DCCACA4FC0BBF90C
:10E08000BFD2412D4506B13F36358E233E3D6CED66
:10E090007D18E0C4D5E18FC73BC184F387CE9928B2
:10E0A0000000004079319928C53E84F32B1E8FC7AC
:10E0B00083E7E0C4C2C26CEDCACA8E23BBF9B13F8C
:10E0C000412D412DB13FBBF98E23CACA6CEDC2C2AE
:10E0D000E0C483E78FC72B1E84F3C53E99287931AE
:10E0E00000400000992887CE84F33BC18FC7D5E15B
:10E0F000E0C47D186CED3E3D8E233635B13F4506BC
:10E10000412DBFD2BBF94FC0CACA72DCC2C2941241
:10E1100083E7203B2B1E7138C53E7C0C793167D7D5
:10E12000000000C087CE67D73BC17C0CD5E17138B9
:10E130007D18203B3E3D9412363572DC45064FC0BB
:10E14000BFD2BFD24FC0450672DC363594123E3D79
:10E15000203B7D187138D5E17C0C3BC167D787CE59
:10E1600000C0000067D779317C0CC53E71382B1E8A
:10E17000203B83E79412C2C272DCCACA4FC0BBF90B
:10E18000BFD2412D4506B13F36358E233E3D6CED65
:10E190007D18E0C4D5E18FC73BC184F387CE9928B1
:10E1A0000000004079319928C53E84F32B1E8FC7AB
:10E1B00083E7E0C4C2C26CEDCACA8E23BBF9B13F8B
:10E1C000412D412DB13FBBF98E23CACA6CEDC2C2AD
:10E1D000E0C483E78FC72B1E84F3C53E99287931AD
:10E1E00000400000992887CE84F33BC18FC7D5E15A
:10E1F000E0C47D186CED3E3D8E233635B13F4506BB
:10E20000412DBFD2BBF94FC0CACA72DCC2C2941240
:10E2100083E7203B2B1E7138C53E7C0C793167D7D4
:10E22000000000C087CE67D73BC17C0CD5E17138B8
:10E230007D18203B3E3D9412363572DC45064FC0BA
:10E24000BFD2BFD24FC0450672DC363594123E3D78
:10E25000203B7D187138D5E17C0C3BC167D787CE58
:10E2600000C0000067D779317C0CC53E71382B1E89
:10E27000203B83E79412C2C272DCCACA4FC0BBF90A
:10E28000BFD2412D4506B13F36358E233E3D6CED64
:10E290007D18E0C4D5E18FC73BC184F387CE9928B0
:10E2A0000000004079319928C53E84F32B1E8FC7AA
:10E2B00083E7E0C4C2C26CEDCACA8E23BBF9B13F8A
:10E2C000412D412DB13FBBF98E23CACA6CEDC2C2AC
:10E2D000E0C483E78FC72B1E84F3C53E99287931AC
:10E2E00000400000992887CE84F33BC18FC7D5E159
:10E2F000E0C47D186CED3E3D8E233635B13F4506BA
:10E30000412DBFD2BBF94FC0CACA72DCC2C294123F
:10E3100083E7203B2B1E7138C53E7C0C793167D7D3
:10E32000000000C087CE67D73BC17C0CD5E17138B7
:10E330007D18203B3E3D9412363572DC45064FC0B9
:10E34000BFD2BFD24FC0450672DC363594123E3D77
:10E35000203B7D187138D5E17C0C3BC167D787CE57
:10E3600000C0000067D779317C0CC53E71382B1E88
:10E37000203B83E79412C2C272DCCACA4FC0BBF909
:10E38000BFD2412D4506B13F36358E233E3D6CED63
:10E390007D18E0C4D5E18FC73BC184F387CE9928AF
:10E3A0000000004079319928C53E84F32B1E8FC7A9
:10E3B00083E7E0C4C2C26CEDCACA8E23BBF9B13F89
:10E3C000412D412DB13FBBF98E23CACA6CEDC2C2AB
:10E3D000E0C483E78FC72B1E84F3C53E99287931AB
:10E3E00000400000992887CE84F33BC18FC7D5E158
:10E3F000E0C47D186CED3E3D8E233635B13F4506B9
:10E40000412DBFD2BBF94FC0CACA72DCC2C294123E
:10E4100083E7203B2B1E7138C53E7C0C793167D7D2
:10E42000000000C087CE67D73BC17C0CD5E17138B6
:10E430007D18203B3E3D9412363572DC45064FC0B8
:10E44000BFD2BFD24FC0450672DC363594123E3D76
:10E45000203B7D187138D5E17C0C3BC167D787CE56
:10E4600000C0000067D779317C0CC53E71382B1E87
:10E47000203B83E79412C2C272DCCACA4FC0BBF908
:10E48000BFD2412D4506B13F36358E233E3D6CED62
:10E490007D18E0C4D5E18FC73BC184F387CE9928AE
:10E4A0000000004079319928C53E84F32B1E8FC7A8
:10E4B00083E7E0C4C2C26CEDCACA8E23BBF9B13F88
:10E4C000412D412DB13FBBF98E23CACA6CEDC2C2AA
:10E4D000E0C483E78FC72B1E84F3C53E99287931AA
:10E4E00000400000992887CE84F33BC18FC7D5E157
:10E4F000E0C47D186CED3E3D8E233635B13F4506B8
:10E50000412DBFD2BBF94FC0CACA72DCC2C294123D
:10E5100083E7203B2B1E7138C53E7C0C793167D7D1
:10E52000000000C087CE67D73BC17C0CD5E17138B5
:10E530007D18203B3E3D9412363572DC45064FC0B7
:10E54000BFD2BFD24FC0450672DC363594123E3D75
:10E55000203B7D187138D5E17C0C3BC167D787CE55
:10E5600000C0000067D779317C0CC53E71382B1E86
:10E57000203B83E79412C2C272DCCACA4FC0BBF907
:10E58000BFD2412D4506B13F36358E233E3D6CED61
:10E590007D18E0C4D5E18FC73BC184F387CE9928AD
:10E5A0000000004079319928C53E84F32B1E8FC7A7
:10E5B00083E7E0C4C2C26CEDCACA8E23BBF9B13F87
:10E5C000412D412DB13FBBF98E23CACA6CEDC2C2A9
:10E5D000E0C483E78FC72B1E84F3C53E99287931A9
:10E5E00000400000992887CE84F33BC18FC7D5E156
:10E5F000E0C47D186CED3E3D8E233635B13F4506B7
:10E60000412DBFD2BBF94FC0CACA72DCC2C294123C
:10E6100083E7203B2B1E7138C53E7C0C793167D7D0
:10E62000000000C087CE67D73BC17C0CD5E17138B4
:10E630007D18203B3E3D9412363572DC45064FC0B6
:10E64000BFD2BFD24FC0450672DC363594123E3D74
:10E65000203B7D187138D5E17C0C3BC167D787CE54
:10E6600000C0000067D779317C0CC53E71382B1E85
:10E67000203B83E79412C2C272DCCACA4FC0BBF906
:10E68000BFD2412D4506B13F36358E233E3D6CED60
:10E690007D18E0C4D5E18FC73BC184F387CE9928AC
:10E6A0000000004012363D22DA39A3E4D5077CC0D1
:10E6B00087CE67D73BC3131474F0143E212C5A2E17
:10E6C000C53E84F308174AC4E1D999CC2DC0B504DE
:10E6D000D5E171388B1FAF37EC3F2303DA24ADCB84
:10E6E00083E7E0C4F2C00FF506D56B2F1111AE3DE4
:10E6F0003E3D9412763033D69CF6B2C07EC511E60C
:10E70000CACA8E239201FB3FE536E7202A393AE355
:10E7100045064FC08CCDA1D8BEC38F15FBF1713E0D
:10E72000412D412D713EFBF18F15BEC3A1D88CCD7B
:10E730004FC045063AE32A39E720E536FB3F920110
:10E740008E23CACA11E67EC5B2C09CF633D6763097
:10E7500094123E3DAE3D11116B2F06D50FF5F2C060
:10E76000E0C483E7ADCBDA242303EC3FAF378B1F44
:10E770007138D5E1B5042DC099CCE1D94AC4081748
:10E7800084F3C53E5A2E212C143E74F013143BC35F
:10E7900067D787CE7CC0D507A3E4DA393D2212368D
:10E7A000004000003D22EEC9A3E426C67CC02BF841
:10E7B00067D779311314C53C143E8C0F5A2EDFD322
:10E7C00084F33BC14AC4F8E899CC1F26B504D33F73
:10E7D00071382B1EAF3775E0230314C0ADCB26DB99
:10E7E000E0C47D180FF50E3F6B2FFA2AAE3DEFEE19
:10E7F0009412C2C233D68ACFB2C0640911E6823AFB
:10E800008E233635FB3F6EFEE7201BC93AE3D6C6A2
:10E810004FC0BBF9A1D874328F15423C713E050E32
:10E82000412DBFD2FBF18FC1BEC371EA8CCD5F27F2
:10E830004506B13F2A39C61CE53619DF920105C0ED
:10E84000CACA72DC7EC5EF199CF64E3F7630CD29E0
:10E850003E3D6CED111152C206D595D0F2C0F10AC1
:10E8600083E7203BDA245334EC3FDDFC8B1F51C897
:10E87000D5E18FC72DC04BFBE1D967330817B63BF5
:10E88000C53E7C0C212CA6D174F0ECC13BC3EDEB52
:10E8900087CE9928D507843FDA395D1B1236C3DD50
:10E8A000000000C0EEC9C3DD26C65D1B2BF8843F07
:10E8B00079319928C53CEDEB8C0FECC1DFD3A6D1A3
:10E8C0003BC17C0CF8E8B63B1F266733D33F4BFBBC
:10E8D0002B1E8FC775E051C814C0DDFC26DB5334F6
:10E8E0007D18203B0E3FF10AFA2A95D0EFEE52C276
:10E8F000C2C26CED8ACFCD2964094E3F823AEF192E
:10E90000363572DC6EFE05C01BC919DFD6C6C61CC3
:10E91000BBF9B13F74325F27423C71EA050E8FC1EB
:10E92000BFD2BFD28FC1050E71EA423C5F2774325D
:10E93000B13FBBF9C61CD6C619DF1BC905C06EFEA8
:10E9400072DC3635EF19823A4E3F6409CD298ACF01
:10E950006CEDC2C252C2EFEE95D0FA2AF10A0E3F18
:10E96000203B7D18533426DBDDFC14C051C875E014
:10E970008FC72B1E4BFBD33F67331F26B63BF8E8F0
:10E980007C0C3BC1A6D1DFD3ECC18C0FEDEBC53CB9
:10E9900099287931843F2BF85D1B26C6C3DDEEC96B
:10E9A00000C00000C3DD12365D1BDA39843FD50795
:10E9B000992887CEEDEB3BC3ECC174F0A6D1212C96
:10E9C0007C0CC53EB63B08176733E1D94BFB2DC025
:10E9D0008FC7D5E151C88B1FDDFCEC3F5334DA24DF
:10E9E000203B83E7F10AF2C095D006D552C211113F
:10E9F0006CED3E3DCD2976304E3F9CF6EF197EC53D
:10EA000072DCCACA05C0920119DFE536C61C2A3974
:10EA1000B13F45065F278CCD71EABEC38FC1FBF1C4
:10EA2000BFD2412D050E713E423C8F157432A1D8E4
:10EA3000BBF94FC0D6C63AE31BC9E7206EFEFB3FC9
:10EA400036358E23823A11E66409B2C08ACF33D6B6
:10EA5000C2C29412EFEEAE3DFA2A6B2F0E3F0FF5B5
:10EA60007D18E0C426DBADCB14C0230375E0AF37BF
:10EA70002B1E7138D33FB5041F2699CCF8E84AC441
:10EA80003BC184F3DFD35A2E8C0F143EC53C1314C4
:10EA9000793167D72BF87CC026C6A3E4EEC93D22A6
:10EAA0000000004012363D22DA39A3E4D5077CC0CD
:10EAB00087CE67D73BC3131474F0143E212C5A2E13
:10EAC000C53E84F308174AC4E1D999CC2DC0B504DA
:10EAD000D5E171388B1FAF37EC3F2303DA24ADCB80
:10EAE00083E7E0C4F2C00FF506D56B2F1111AE3DE0
:10EAF0003E3D9412763033D69CF6B2C07EC511E608
:10EB0000CACA8E239201FB3FE536E7202A393AE351
:10EB100045064FC08CCDA1D8BEC38F15FBF1713E09
:10EB2000412D412D713EFBF18F15BEC3A1D88CCD77
:10EB30004FC045063AE32A39E720E536FB3F92010C
:10EB40008E23CACA11E67EC5B2C09CF633D6763093
:10EB500094123E3DAE3D11116B2F06D50FF5F2C05C
:10EB6000E0C483E7ADCBDA242303EC3FAF378B1F40
:10EB70007138D5E1B5042DC099CCE1D94AC4081744
:10EB800084F3C53E5A2E212C143E74F013143BC35B
:10EB900067D787CE7CC0D507A3E4DA393D22123689
:10EBA000004000003D22EEC9A3E426C67CC02BF83D
:10EBB00067D779311314C53C143E8C0F5A2EDFD31E
:10EBC00084F33BC14AC4F8E899CC1F26B504D33F6F
:10EBD00071382B1EAF3775E0230314C0ADCB26DB95
:10EBE000E0C47D180FF50E3F6B2FFA2AAE3DEFEE15
:10EBF0009412C2C233D68ACFB2C0640911E6823AF7
:10EC00008E233635FB3F6EFEE7201BC93AE3D6C69E
:10EC10004FC0BBF9A1D874328F15423C713E050E2E
:10EC2000412DBFD2FBF18FC1BEC371EA8CCD5F27EE
:10EC30004506B13F2A39C61CE53619DF920105C0E9
:10EC4000CACA72DC7EC5EF199CF64E3F7630CD29DC
:10EC50003E3D6CED111152C206D595D0F2C0F10ABD
:10EC600083E7203BDA245334EC3FDDFC8B1F51C893
:10EC7000D5E18FC72DC04BFBE1D967330817B63BF1
:10EC8000C53E7C0C212CA6D174F0ECC13BC3EDEB4E
:10EC900087CE9928D507843FDA395D1B1236C3DD4C
:10ECA000000000C0EEC9C3DD26C65D1B2BF8843F03
:10ECB00079319928C53CEDEB8C0FECC1DFD3A6D19F
:10ECC0003BC17C0CF8E8B63B1F266733D33F4BFBB8
:10ECD0002B1E8FC775E051C814C0DDFC26DB5334F2
:10ECE0007D18203B0E3FF10AFA2A95D0EFEE52C272
:10ECF000C2C26CED8ACFCD2964094E3F823AEF192A
:10ED0000363572DC6EFE05C01BC919DFD6C6C61CBF
:10ED1000BBF9B13F74325F27423C71EA050E8FC1E7
:10ED2000BFD2BFD28FC1050E71EA423C5F27743259
:10ED3000B13FBBF9C61CD6C619DF1BC905C06EFEA4
:10ED400072DC3635EF19823A4E3F6409CD298ACFFD
:10ED50006CEDC2C252C2EFEE95D0FA2AF10A0E3F14
:10ED6000203B7D18533426DBDDFC14C051C875E010
:10ED70008FC72B1E4BFBD33F67331F26B63BF8E8EC
:10ED80007C0C3BC1A6D1DFD3ECC18C0FEDEBC53CB5
:10ED900099287931843F2BF85D1B26C6C3DDEEC967
:10EDA00000C00000C3DD12365D1BDA39843FD50791
:10EDB000992887CEEDEB3BC3ECC174F0A6D1212C92
:10EDC0007C0CC53EB63B08176733E1D94BFB2DC021
:10EDD0008FC7D5E151C88B1FDDFCEC3F5334DA24DB
:10EDE000203B83E7F10AF2C095D006D552C211113B
:10EDF0006CED3E3DCD2976304E3F9CF6EF197EC539
:10EE000072DCCACA05C0920119DFE536C61C2A3970
:10EE1000B13F45065F278CCD71EABEC38FC1FBF1C0
:10EE2000BFD2412D050E713E423C8F157432A1D8E0
:10EE3000BBF94FC0D6C63AE31BC9E7206EFEFB3FC5
:10EE400036358E23823A11E66409B2C08ACF33D6B2
:10EE5000C2C29412EFEEAE3DFA2A6B2F0E3F0FF5B1
:10EE60007D18E0C426DBADCB14C0230375E0AF37BB
:10EE70002B1E7138D33FB5041F2699CCF8E84AC43D
:10EE80003BC184F3DFD35A2E8C0F143EC53C1314C0
:10EE9000793167D72BF87CC026C6A3E4EEC93D22A2
:10EEA0000000004000400000000000C000C0000062
:10EEB0000000004000400000000000C000C0000052
:10EEC0000000004000400000000000C000C0000042
:10EED0000000004000400000000000C000C0000032
:10EEE0000000004000400000000000C000C0000022
:10EEF0000000004000400000000000C000C0000012
:10EF00000000004000400000000000C000C0000001
:10EF10000000004000400000000000C000C00000F1
:10EF20000000004000400000000000C000C00000E1
:10EF30000000004000400000000000C000C00000D1
:10EF40000000004000400000000000C000C00000C1
:10EF50000000004000400000000000C000C00000B1
:10EF60000000004000400000000000C000C00000A1
:10EF70000000004000400000000000C000C0000091
:10EF80000000004000400000000000C000C0000081
:10EF90000000004000400000000000C000C0000071
:10EFA0000000004000400000000000C000C0000061
:10EFB0000000004000400000000000C000C0000051
:10EFC0000000004000400000000000C000C0000041
:10EFD0000000004000400000000000C000C0000031
:10EFE0000000004000400000000000C000C0000021
:10EFF0000000004000400000000000C000C0000011
:10F000000000004000400000000000C000C0000000
:10F010000000004000400000000000C000C00000F0
:10F020000000004000400000000000C000C00000E0
:10F030000000004000400000000000C000C00000D0
:10F040000000004000400000000000C000C00000C0
:10F050000000004000400000000000C000C00000B0
:10F060000000004000400000000000C000C00000A0
:10F070000000004000400000000000C000C0000090
:10F080000000004000400000000000C000C0000080
:10F090000000004000400000000000C000C0000070
:10F0A0000000004000400000000000C000C0000060
:10F0B0000000004000400000000000C000C0000050
:10F0C0000000004000400000000000C000C0000040
:10F0D0000000004000400000000000C000C0000030
:10F0E0000000004000400000000000C000C0000020
:10F0F0000000004000400000000000C000C0000010
:10F100000000004000400000000000C000C00000FF
:10F110000000004000400000000000C000C00000EF
:10F120000000004000400000000000C000C00000DF
:10F130000000004000400000000000C000C00000CF
:10F140000000004000400000000000C000C00000BF
:10F150000000004000400000000000C000C00000AF
:10F160000000004000400000000000C000C000009F
:10F170000000004000400000000000C000C000008F
:10F180000000004000400000000000C000C000007F
:10F190000000004000400000000000C000C000006F
:10F1A0000000004000400000000000C000C000005F
:10F1B0000000004000400000000000C000C000004F
:10F1C0000000004000400000000000C000C000003F
:10F1D0000000004000400000000000C000C000002F
:10F1E0000000004000400000000000C000C000001F
:10F1F0000000004000400000000000C000C000000F
:10F200000000004000400000000000C000C00000FE
:10F210000000004000400000000000C000C00000EE
:10F220000000004000400000000000C000C00000DE
:10F230000000004000400000000000C000C00000CE
:10F240000000004000400000000000C000C00000BE
:10F250000000004000400000000000C000C00000AE
:10F260000000004000400000000000C000C000009E
:10F270000000004000400000000000C000C000008E
:10F280000000004000400000000000C000C000007E
:10F290000000004000400000000000C000C000006E
:10F2A0000000004000400000000000C000C000005E
:10F2B0000000004000400000000000C000C000004E
:10F2C0000000004000400000000000C000C000003E
:10F2D0000000004000400000000000C000C000002E
:10F2E0000000004000400000000000C000C000001E
:10F2F0000000004000400000000000C000C000000E
:10F300000000004000400000000000C000C00000FD
:10F310000000004000400000000000C000C00000ED
:10F320000000004000400000000000C000C00000DD
:10F330000000004000400000000000C000C00000CD
:10F340000000004000400000000000C000C00000BD
:10F350000000004000400000000000C000C00000AD
:10F360000000004000400000000000C000C000009D
:10F370000000004000400000000000C000C000008D
:10F380000000004000400000000000C000C000007D
:10F390000000004000400000000000C000C000006D
:10F3A0000000004000400000000000C000C000005D
:10F3B0000000004000400000000000C000C000004D
:10F3C0000000004000400000000000C000C000003D
:10F3D0000000004000400000000000C000C000002D
:10F3E0000000004000400000000000C000C000001D
:10F3F0000000004000400000000000C000C000000D
:10F400000000004000400000000000C000C00000FC
:10F410000000004000400000000000C000C00000EC
:10F420000000004000400000000000C000C00000DC
:10F430000000004000400000000000C000C00000CC
:10F440000000004000400000000000C000C00000BC
:10F450000000004000400000000000C000C00000AC
:10F460000000004000400000000000C000C000009C
:10F470000000004000400000000000C000C000008C
:10F480000000004000400000000000C000C000007C
:10F490000000004000400000000000C000C000006C
:10F4A0000000004000400000000000C000C000005C
:10F4B0000000004000400000000000C000C000004C
:10F4C0000000004000400000000000C000C000003C
:10F4D0000000004000400000000000C000C000002C
:10F4E0000000004000400000000000C000C000001C
:10F4F0000000004000400000000000C000C000000C
:10F500000000004000400000000000C000C00000FB
:10F510000000004000400000000000C000C00000EB
:10F520000000004000400000000000C000C00000DB
:10F530000000004000400000000000C000C00000CB
:10F540000000004000400000000000C000C00000BB
:10F550000000004000400000000000C000C00000AB
:10F560000000004000400000000000C000C000009B
:10F570000000004000400000000000C000C000008B
:10F580000000004000400000000000C000C000007B
:10F590000000004000400000000000C000C000006B
:10F5A0000000004000400000000000C000C000005B
:10F5B0000000004000400000000000C000C000004B
:10F5C0000000004000400000000000C000C000003B
:10F5D0000000004000400000000000C000C000002B
:10F5E0000000004000400000000000C000C000001B
:10F5F0000000004000400000000000C000C000000B
:10F600000000004000400000000000C000C00000FA
:10F610000000004000400000000000C000C00000EA
:10F620000000004000400000000000C000C00000DA
:10F630000000004000400000000000C000C00000CA
:10F640000000004000400000000000C000C00000BA
:10F650000000004000400000000000C000C00000AA
:10F660000000004000400000000000C000C000009A
:10F670000000004000400000000000C000C000008A
:10F680000000004000400000000000C000C000007A
:10F690000000004000400000000000C000C000006A
:10F6A00000000040C53C13141F2699CC26DBADCBCF
:10F6B000C2C294126EFEFB3F423C8F155F278CCD79
:10F6C00072DCCACA52C21111DDFCEC3FB63B08170E
:10F6D000992887CEC3DDEEC9ECC18C0F4BFBD33F1D
:10F6E000203B7D18CD298ACF19DF1BC98FC1050E9C
:10F6F000BBF9B13F823AEF19FA2A95D075E051C8AB
:10F700003BC17C0C2BF8843FDA395D1B212CA6D140
:10F71000D5E18FC7F2C0F10A9CF64E3F2A39C61CCC
:10F72000412DBFD23AE3D6C6B2C064090FF50E3FF1
:10F7300071382B1E5A2EDFD3A3E426C67CC0D50712
:10F7400084F3C53EAF378B1F6B2F06D511E67EC500
:10F750004FC04506FBF1713EE536E720763033D6E3
:10F7600083E7E0C42DC0B50474F0143E12363D2288
:10F77000793167D7F8E84AC414C02303EFEEAE3DF1
:10F7800036358E237432A1D871EABEC305C092010A
:10F790006CED3E3D5334DA246733E1D9EDEB3BC3E6
:10F7A00000C00000EDEBC53C67331F26533426DB59
:10F7B0006CEDC2C205C06EFE71EA423C74325F2736
:10F7C000363572DCEFEE52C214C0DDFCF8E8B63B11
:10F7D000793199281236C3DD74F0ECC12DC04BFB92
:10F7E00083E7203B7630CD29E53619DFFBF18FC169
:10F7F0004FC0BBF911E6823A6B2FFA2AAF3775E09A
:10F8000084F33BC17CC02BF8A3E4DA395A2E212CB7
:10F810007138D5E10FF5F2C0B2C09CF63AE32A394F
:10F82000412D412D2A393AE39CF6B2C0F2C00FF5C2
:10F83000D5E17138212C5A2EDA39A3E42BF87CC09B
:10F840003BC184F375E0AF37FA2A6B2F823A11E699
:10F85000BBF94FC08FC1FBF119DFE536CD297630FA
:10F86000203B83E74BFB2DC0ECC174F0C3DD1236A7
:10F8700099287931B63BF8E8DDFC14C052C2EFEEAE
:10F8800072DC36355F277432423C71EA6EFE05C089
:10F89000C2C26CED26DB53341F266733C53CEDEB4B
:10F8A000000000C03BC3EDEBE1D96733DA245334E9
:10F8B0003E3D6CED920105C0BEC371EAA1D8743221
:10F8C0008E233635AE3DEFEE230314C04AC4F8E86C
:10F8D00067D779313D221236143E74F0B5042DC03D
:10F8E000E0C483E733D67630E720E536713EFBF19E
:10F8F00045064FC07EC511E606D56B2F8B1FAF376F
:10F90000C53E84F3D5077CC026C6A3E4DFD35A2EB8
:10F910002B1E71380E3F0FF56409B2C0D6C63AE30C
:10F92000BFD2412DC61C2A394E3F9CF6F10AF2C0C7
:10F930008FC7D5E1A6D1212C5D1BDA39843F2BF886
:10F940007C0C3BC151C875E095D0FA2AEF19823A78
:10F95000B13FBBF9050E8FC11BC919DF8ACFCD2975
:10F960007D18203BD33F4BFB8C0FECC1EEC9C3DDB0
:10F9700087CE99280817B63BEC3FDDFC111152C227
:10F98000CACA72DC8CCD5F278F15423CFB3F6EFEEE
:10F990009412C2C2ADCB26DB99CC1F261314C53CF2
:10F9A0000040000013143BC399CCE1D9ADCBDA245D
:10F9B00094123E3DFB3F92018F15BEC38CCDA1D862
:10F9C000CACA8E231111AE3DEC3F230308174AC467
:10F9D00087CE67D7EEC93D228C0F143ED33FB504C6
:10F9E0007D18E0C48ACF33D61BC9E720050E713ECF
:10F9F000B13F4506EF197EC595D006D551C88B1F7E
:10FA00007C0CC53E843FD5075D1B26C6A6D1DFD33F
:10FA10008FC72B1EF10A0E3F4E3F6409C61CD6C687
:10FA2000BFD2BFD2D6C6C61C64094E3F0E3FF10AF4
:10FA30002B1E8FC7DFD3A6D126C65D1BD507843FFB
:10FA4000C53E7C0C8B1F51C806D595D07EC5EF19DD
:10FA50004506B13F713E050EE7201BC933D68ACF5C
:10FA6000E0C47D18B504D33F143E8C0F3D22EEC98F
:10FA700067D787CE4AC408172303EC3FAE3D111168
:10FA80008E23CACAA1D88CCDBEC38F159201FB3F6D
:10FA90003E3D9412DA24ADCBE1D999CC3BC313148B
:10FAA00000000040C53C13141F2699CC26DBADCBCB
:10FAB000C2C294126EFEFB3F423C8F155F278CCD75
:10FAC00072DCCACA52C21111DDFCEC3FB63B08170A
:10FAD000992887CEC3DDEEC9ECC18C0F4BFBD33F19
:10FAE000203B7D18CD298ACF19DF1BC98FC1050E98
:10FAF000BBF9B13F823AEF19FA2A95D075E051C8A7
:10FB00003BC17C0C2BF8843FDA395D1B212CA6D13C
:10FB1000D5E18FC7F2C0F10A9CF64E3F2A39C61CC8
:10FB2000412DBFD23AE3D6C6B2C064090FF50E3FED
:10FB300071382B1E5A2EDFD3A3E426C67CC0D5070E
:10FB400084F3C53EAF378B1F6B2F06D511E67EC5FC
:10FB50004FC04506FBF1713EE536E720763033D6DF
:10FB600083E7E0C42DC0B50474F0143E12363D2284
:10FB7000793167D7F8E84AC414C02303EFEEAE3DED
:10FB800036358E237432A1D871EABEC305C0920106
:10FB90006CED3E3D5334DA246733E1D9EDEB3BC3E2
:10FBA00000C00000EDEBC53C67331F26533426DB55
:10FBB0006CEDC2C205C06EFE71EA423C74325F2732
:10FBC000363572DCEFEE52C214C0DDFCF8E8B63B0D
:10FBD000793199281236C3DD74F0ECC12DC04BFB8E
:10FBE00083E7203B7630CD29E53619DFFBF18FC165
:10FBF0004FC0BBF911E6823A6B2FFA2AAF3775E096
:10FC000084F33BC17CC02BF8A3E4DA395A2E212CB3
:10FC10007138D5E10FF5F2C0B2C09CF63AE32A394B
:10FC2000412D412D2A393AE39CF6B2C0F2C00FF5BE
:10FC3000D5E17138212C5A2EDA39A3E42BF87CC097
:10FC40003BC184F375E0AF37FA2A6B2F823A11E695
:10FC5000BBF94FC08FC1FBF119DFE536CD297630F6
:10FC6000203B83E74BFB2DC0ECC174F0C3DD1236A3
:10FC700099287931B63BF8E8DDFC14C052C2EFEEAA
:10FC800072DC36355F277432423C71EA6EFE05C085
:10FC9000C2C26CED26DB53341F266733C53CEDEB47
:10FCA000000000C03BC3EDEBE1D96733DA245334E5
:10FCB0003E3D6CED920105C0BEC371EAA1D874321D
:10FCC0008E233635AE3DEFEE230314C04AC4F8E868
:10FCD00067D779313D221236143E74F0B5042DC039
:10FCE000E0C483E733D67630E720E536713EFBF19A
:10FCF00045064FC07EC511E606D56B2F8B1FAF376B
:10FD0000C53E84F3D5077CC026C6A3E4DFD35A2EB4
:10FD10002B1E71380E3F0FF56409B2C0D6C63AE308
:10FD2000BFD2412DC61C2A394E3F9CF6F10AF2C0C3
:10FD30008FC7D5E1A6D1212C5D1BDA39843F2BF882
:10FD40007C0C3BC151C875E095D0FA2AEF19823A74
:10FD5000B13FBBF9050E8FC11BC919DF8ACFCD2971
:10FD60007D18203BD33F4BFB8C0FECC1EEC9C3DDAC
:10FD700087CE99280817B63BEC3FDDFC111152C223
:10FD8000CACA72DC8CCD5F278F15423CFB3F6EFEEA
:10FD90009412C2C2ADCB26DB99CC1F261314C53CEE
:10FDA0000040000013143BC399CCE1D9ADCBDA2459
:10FDB00094123E3DFB3F92018F15BEC38CCDA1D85E
:10FDC000CACA8E231111AE3DEC3F230308174AC463
:10FDD00087CE67D7EEC93D228C0F143ED33FB504C2
:10FDE0007D18E0C48ACF33D61BC9E720050E713ECB
:10FDF000B13F4506EF197EC595D006D551C88B1F7A
:10FE00007C0CC53E843FD5075D1B26C6A6D1DFD33B
:10FE10008FC72B1EF10A0E3F4E3F6409C61CD6C683
:10FE2000BFD2BFD2D6C6C61C64094E3F0E3FF10AF0
:10FE30002B1E8FC7DFD3A6D126C65D1BD507843FF7
:10FE4000C53E7C0C8B1F51C806D595D07EC5EF19D9
:10FE50004506B13F713E050EE7201BC933D68ACF58
:10FE6000E0C47D18B504D33F143E8C0F3D22EEC98B
:10FE700067D787CE4AC408172303EC3FAE3D111164
:10FE80008E23CACAA1D88CCDBEC38F159201FB3F69
:10FE90003E3D9412DA24ADCBE1D999CC3BC3131487
:10FEA00000000040D33FB5046409B2C08FC1FBF12C
:10FEB0006CED3E3DB63B08175D1B26C651C875E08C
:10FEC00072DC363574325F27FA2A95D0DFD3A6D19B
:10FED00087CE9928DA245334E53619DF3AE3D6C6BB
:10FEE000E0C47D181314C53C143E74F00FF5F2C045
:10FEF0004FC045069201FB3FEC3F2303D5077CC072
:10FF00003BC184F3EFEEAE3D423C8F15EF197EC549
:10FF10008FC7D5E1C3DD123667331F26CD298ACFBF
:10FF2000BFD2BFD28ACFCD291F2667331236C3DD99
:10FF3000D5E18FC77EC5EF198F15423CAE3DEFEE80
:10FF400084F33BC17CC0D5072303EC3FFB3F920108
:10FF500045064FC0F2C00FF574F0143EC53C1314B3
:10FF60007D18E0C4D6C63AE319DFE5365334DA2407
:10FF7000992887CEA6D1DFD395D0FA2A5F2774328D
:10FF8000363572DC75E051C826C65D1B0817B63BD6
:10FF90003E3D6CEDFBF18FC1B2C06409B504D33FA7
:10FFA00000400000B5042DC0B2C09CF6FBF1713ECC
:10FFB0003E3D941208174AC426C6A3E475E0AF3745
:10FFC00036358E235F278CCD95D006D5A6D1212C32
:10FFD00099287931533426DB19DF1BC9D6C6C61CD4
:10FFE0007D18203BC53CEDEB74F0ECC1F2C0F10A8A
:10FFF0004506B13FFB3F6EFE230314C07CC02BF8C7
:020000040801F1
:1000000084F3C53EAE3D11118F15BEC37EC511E60A
:10001000D5E1713812363D221F2699CC8ACF33D6CE
:10002000BFD2412DCD2976306733E1D9C3DDEEC98A
:100030008FC72B1EEF19823A423C71EAEFEE52C293
:100040003BC17C0CD507843FEC3FDDFC920105C031
:100050004FC0BBF90FF50E3F143E8C0F13143BC37A
:10006000E0C483E73AE32A39E536E720DA24ADCB6A
:1000700087CE67D7DFD35A2EFA2A6B2F7432A1D8D6
:1000800072DCCACA51C88B1F5D1BDA39B63BF8E86F
:100090006CEDC2C28FC1050E64094E3FD33F4BFBCE
:1000A000000000C02DC04BFB9CF64E3F713E050E7C
:1000B0009412C2C24AC4F8E8A3E4DA39AF378B1FFE
:1000C0008E23CACA8CCDA1D806D56B2F212C5A2ECF
:1000D000793167D726DBADCB1BC9E720C61C2A398F
:1000E000203B83E7EDEB3BC3ECC18C0FF10A0E3FE5
:1000F000B13FBBF96EFE05C014C0DDFC2BF8843F98
:10010000C53E7C0C111152C2BEC371EA11E6823A9F
:1001100071382B1E3D22EEC999CCE1D933D6763009
:10012000412D412D763033D6E1D999CCEEC93D220F
:100130002B1E7138823A11E671EABEC352C2111108
:100140007C0CC53E843F2BF8DDFC14C005C06EFE60
:10015000BBF9B13F0E3FF10A8C0FECC13BC3EDEB95
:1001600083E7203B2A39C61CE7201BC9ADCB26DB21
:1001700067D779315A2E212C6B2F06D5A1D88CCD7B
:10018000CACA8E238B1FAF37DA39A3E4F8E84AC412
:10019000C2C29412050E713E4E3F9CF64BFB2DC021
:1001A00000C000004BFBD33F4E3F6409050E8FC1DA
:1001B000C2C26CEDF8E8B63BDA395D1B8B1F51C843
:1001C000CACA72DCA1D874326B2FFA2A5A2EDFD336
:1001D00067D787CEADCBDA24E720E5362A393AE374
:1001E00083E7E0C43BC313148C0F143E0E3F0FF59E
:1001F000BBF94FC005C09201DDFCEC3F843FD50741
:100200007C0C3BC152C2EFEE71EA423C823AEF19DC
:100210002B1E8FC7EEC9C3DDE1D967337630CD29F8
:10022000412DBFD233D68ACF99CC1F263D2212361C
:100230007138D5E111E67EC5BEC38F151111AE3DF3
:10024000C53E84F32BF87CC014C023036EFEFB3F35
:10025000B13F4506F10AF2C0ECC174F0EDEBC53CCC
:10026000203B7D18C61CD6C61BC919DF26DB5334BC
:1002700079319928212CA6D106D595D08CCD5F2730
:100280008E233635AF3775E0A3E426C64AC4081777
:1002900094123E3D713EFBF19CF6B2C02DC0B504F8
:1002A00000000040D33FB5046409B2C08FC1FBF128
:1002B0006CED3E3DB63B08175D1B26C651C875E088
:1002C00072DC363574325F27FA2A95D0DFD3A6D197
:1002D00087CE9928DA245334E53619DF3AE3D6C6B7
:1002E000E0C47D181314C53C143E74F00FF5F2C041
:1002F0004FC045069201FB3FEC3F2303D5077CC06E
:100300003BC184F3EFEEAE3D423C8F15EF197EC545
:100310008FC7D5E1C3DD123667331F26CD298ACFBB
:10032000BFD2BFD28ACFCD291F2667331236C3DD95
:10033000D5E18FC77EC5EF198F15423CAE3DEFEE7C
:1003400084F33BC17CC0D5072303EC3FFB3F920104
:1003500045064FC0F2C00FF574F0143EC53C1314AF
:100360007D18E0C4D6C63AE319DFE5365334DA2403
:10037000992887CEA6D1DFD395D0FA2A5F27743289
:10038000363572DC75E051C826C65D1B0817B63BD2
:100390003E3D6CEDFBF18FC1B2C06409B504D33FA3
:1003A00000400000B5042DC0B2C09CF6FBF1713EC8
:1003B0003E3D941208174AC426C6A3E475E0AF3741
:1003C00036358E235F278CCD95D006D5A6D1212C2E
:1003D00099287931533426DB19DF1BC9D6C6C61CD0
:1003E0007D18203BC53CEDEB74F0ECC1F2C0F10A86
:1003F0004506B13FFB3F6EFE230314C07CC02BF8C3
:1004000084F3C53EAE3D11118F15BEC37EC511E606
:10041000D5E1713812363D221F2699CC8ACF33D6CA
:10042000BFD2412DCD2976306733E1D9C3DDEEC986
:100430008FC72B1EEF19823A423C71EAEFEE52C28F
:100440003BC17C0CD507843FEC3FDDFC920105C02D
:100450004FC0BBF90FF50E3F143E8C0F13143BC376
:10046000E0C483E73AE32A39E536E720DA24ADCB66
:1004700087CE67D7DFD35A2EFA2A6B2F7432A1D8D2
:1004800072DCCACA51C88B1F5D1BDA39B63BF8E86B
:100490006CEDC2C28FC1050E64094E3FD33F4BFBCA
:1004A000000000C02DC04BFB9CF64E3F713E050E78
:1004B0009412C2C24AC4F8E8A3E4DA39AF378B1FFA
:1004C0008E23CACA8CCDA1D806D56B2F212C5A2ECB
:1004D000793167D726DBADCB1BC9E720C61C2A398B
:1004E000203B83E7EDEB3BC3ECC18C0FF10A0E3FE1
:1004F000B13FBBF96EFE05C014C0DDFC2BF8843F94
:10050000C53E7C0C111152C2BEC371EA11E6823A9B
:1005100071382B1E3D22EEC999CCE1D933D6763005
:10052000412D412D763033D6E1D999CCEEC93D220B
:100530002B1E7138823A11E671EABEC352C2111104
:100540007C0CC53E843F2BF8DDFC14C005C06EFE5C
:10055000BBF9B13F0E3FF10A8C0FECC13BC3EDEB91
:1005600083E7203B2A39C61CE7201BC9ADCB26DB1D
:1005700067D779315A2E212C6B2F06D5A1D88CCD77
:10058000CACA8E238B1FAF37DA39A3E4F8E84AC40E
:10059000C2C29412050E713E4E3F9CF64BFB2DC01D
:1005A00000C000004BFBD33F4E3F6409050E8FC1D6
:1005B000C2C26CEDF8E8B63BDA395D1B8B1F51C83F
:1005C000CACA72DCA1D874326B2FFA2A5A2EDFD332
:1005D00067D787CEADCBDA24E720E5362A393AE370
:1005E00083E7E0C43BC313148C0F143E0E3F0FF59A
:1005F000BBF94FC005C09201DDFCEC3F843FD5073D
:100600007C0C3BC152C2EFEE71EA423C823AEF19D8
:100610002B1E8FC7EEC9C3DDE1D967337630CD29F4
:10062000412DBFD233D68ACF99CC1F263D22123618
:100630007138D5E111E67EC5BEC38F151111AE3DEF
:10064000C53E84F32BF87CC014C023036EFEFB3F31
:10065000B13F4506F10AF2C0ECC174F0EDEBC53CC8
:10066000203B7D18C61CD6C61BC919DF26DB5334B8
:1006700079319928212CA6D106D595D08CCD5F272C
:100680008E233635AF3775E0A3E426C64AC4081773
:1006900094123E3D713EFBF19CF6B2C02DC0B504F4
:1006A00000000040C53E7C0C7D18E0C4CACA72DC64
:1006B000BFD2412D8E233635203B83E784F33BC1E7
:1006C00000C0000084F3C53E203B7D188E23CACABB
:1006D000BFD2BFD2CACA8E237D18203BC53E84F349
:1006E000000000C03BC184F383E7203B36358E23F6
:1006F000412DBFD272DCCACAE0C47D187C0CC53E55
:10070000004000007C0C3BC1E0C483E772DC36355E
:10071000412D412D363572DC83E7E0C43BC17C0CB2
:1007200000000040C53E7C0C7D18E0C4CACA72DCE3
:10073000BFD2412D8E233635203B83E784F33BC166
:1007400000C0000084F3C53E203B7D188E23CACA3A
:10075000BFD2BFD2CACA8E237D18203BC53E84F3C8
:10076000000000C03BC184F383E7203B36358E2375
:10077000412DBFD272DCCACAE0C47D187C0CC53ED4
:10078000004000007C0C3BC1E0C483E772DC3635DE
:10079000412D412D363572DC83E7E0C43BC17C0C32
:1007A00000000040C53E7C0C7D18E0C4CACA72DC63
:1007B000BFD2412D8E233635203B83E784F33BC1E6
:1007C00000C0000084F3C53E203B7D188E23CACABA
:1007D000BFD2BFD2CACA8E237D18203BC53E84F348
:1007E000000000C03BC184F383E7203B36358E23F5
:1007F000412DBFD272DCCACAE0C47D187C0CC53E54
:10080000004000007C0C3BC1E0C483E772DC36355D
:10081000412D412D363572DC83E7E0C43BC17C0CB1
:1008200000000040C53E7C0C7D18E0C4CACA72DCE2
:10083000BFD2412D8E233635203B83E784F33BC165
:1008400000C0000084F3C53E203B7D188E23CACA39
:10085000BFD2BFD2CACA8E237D18203BC53E84F3C7
:10086000000000C03BC184F383E7203B36358E2374
:10087000412DBFD272DCCACAE0C47D187C0CC53ED3
:10088000004000007C0C3BC1E0C483E772DC3635DD
:10089000412D412D363572DC83E7E0C43BC17C0C31
:1008A00000000040C53E7C0C7D18E0C4CACA72DC62
:1008B000BFD2412D8E233635203B83E784F33BC1E5
:1008C00000C0000084F3C53E203B7D188E23CACAB9
:1008D000BFD2BFD2CACA8E237D18203BC53E84F347
:1008E000000000C03BC184F383E7203B36358E23F4
:1008F000412DBFD272DCCACAE0C47D187C0CC53E53
:10090000004000007C0C3BC1E0C483E772DC36355C
:10091000412D412D363572DC83E7E0C43BC17C0CB0
:1009200000000040C53E7C0C7D18E0C4CACA72DCE1
:10093000BFD2412D8E233635203B83E784F33BC164
:1009400000C0000084F3C53E203B7D188E23CACA38
:10095000BFD2BFD2CACA8E237D18203BC53E84F3C6
:10096000000000C03BC184F383E7203B36358E2373
:10097000412DBFD272DCCACAE0C47D187C0CC53ED2
:10098000004000007C0C3BC1E0C483E772DC3635DC
:10099000412D412D363572DC83E7E0C43BC17C0C30
:1009A00000000040C53E7C0C7D18E0C4CACA72DC61
:1009B000BFD2412D8E233635203B83E784F33BC1E4
:1009C00000C0000084F3C53E203B7D188E23CACAB8
:1009D000BFD2BFD2CACA8E237D18203BC53E84F346
:1009E000000000C03BC184F383E7203B36358E23F3
:1009F000412DBFD272DCCACAE0C47D187C0CC53E52
:100A0000004000007C0C3BC1E0C483E772DC36355B
:100A1000412D412D363572DC83E7E0C43BC17C0CAF
:100A200000000040C53E7C0C7D18E0C4CACA72DCE0
:100A3000BFD2412D8E233635203B83E784F33BC163
:100A400000C0000084F3C53E203B7D188E23CACA37
:100A5000BFD2BFD2CACA8E237D18203BC53E84F3C5
:100A6000000000C03BC184F383E7203B36358E2372
:100A7000412DBFD272DCCACAE0C47D187C0CC53ED1
:100A8000004000007C0C3BC1E0C483E772DC3635DB
:100A9000412D412D363572DC83E7E0C43BC17C0C2F
:100AA00000000040C53E7C0C7D18E0C4CACA72DC60
:100AB000BFD2412D8E233635203B83E784F33BC1E3
:100AC00000C0000084F3C53E203B7D188E23CACAB7
:100AD000BFD2BFD2CACA8E237D18203BC53E84F345
:100AE000000000C03BC184F383E7203B36358E23F2
:100AF000412DBFD272DCCACAE0C47D187C0CC53E51
:100B0000004000007C0C3BC1E0C483E772DC36355A
:100B1000412D412D363572DC83E7E0C43BC17C0CAE
:100B200000000040C53E7C0C7D18E0C4CACA72DCDF
:100B3000BFD2412D8E233635203B83E784F33BC162
:100B400000C0000084F3C53E203B7D188E23CACA36
:100B5000BFD2BFD2CACA8E237D18203BC53E84F3C4
:100B6000000000C03BC184F383E7203B36358E2371
:100B7000412DBFD272DCCACAE0C47D187C0CC53ED0
:100B8000004000007C0C3BC1E0C483E772DC3635DA
:100B9000412D412D363572DC83E7E0C43BC17C0C2E
:100BA00000000040C53E7C0C7D18E0C4CACA72DC5F
:100BB000BFD2412D8E233635203B83E784F33BC1E2
:100BC00000C0000084F3C53E203B7D188E23CACAB6
:100BD000BFD2BFD2CACA8E237D18203BC53E84F344
:100BE000000000C03BC184F383E7203B36358E23F1
:100BF000412DBFD272DCCACAE0C47D187C0CC53E50
:100C0000004000007C0C3BC1E0C483E772DC363559
:100C1000412D412D363572DC83E7E0C43BC17C0CAD
:100C200000000040C53E7C0C7D18E0C4CACA72DCDE
:100C3000BFD2412D8E233635203B83E784F33BC161
:100C400000C0000084F3C53E203B7D188E23CACA35
:100C5000BFD2BFD2CACA8E237D18203BC53E84F3C3
:100C6000000000C03BC184F383E7203B36358E2370
:100C7000412DBFD272DCCACAE0C47D187C0CC53ECF
:100C8000004000007C0C3BC1E0C483E772DC3635D9
:100C9000412D412D363572DC83E7E0C43BC17C0C2D
:100CA00000000040C53E7C0C7D18E0C4CACA72DC5E
:100CB000BFD2412D8E233635203B83E784F33BC1E1
:100CC00000C0000084F3C53E203B7D188E23CACAB5
:100CD000BFD2BFD2CACA8E237D18203BC53E84F343
:100CE000000000C03BC184F383E7203B36358E23F0
:100CF000412DBFD272DCCACAE0C47D187C0CC53E4F
:100D0000004000007C0C3BC1E0C483E772DC363558
:100D1000412D412D363572DC83E7E0C43BC17C0CAC
:100D200000000040C53E7C0C7D18E0C4CACA72DCDD
:100D3000BFD2412D8E233635203B83E784F33BC160
:100D400000C0000084F3C53E203B7D188E23CACA34
:100D5000BFD2BFD2CACA8E237D18203BC53E84F3C2
:100D6000000000C03BC184F383E7203B36358E236F
:100D7000412DBFD272DCCACAE0C47D187C0CC53ECE
:100D8000004000007C0C3BC1E0C483E772DC3635D8
:100D9000412D412D363572DC83E7E0C43BC17C0C2C
:100DA00000000040C53E7C0C7D18E0C4CACA72DC5D
:100DB000BFD2412D8E233635203B83E784F33BC1E0
:100DC00000C0000084F3C53E203B7D188E23CACAB4
:100DD000BFD2BFD2CACA8E237D18203BC53E84F342
:100DE000000000C03BC184F383E7203B36358E23EF
:100DF000412DBFD272DCCACAE0C47D187C0CC53E4E
:100E0000004000007C0C3BC1E0C483E772DC363557
:100E1000412D412D363572DC83E7E0C43BC17C0CAB
:100E200000000040C53E7C0C7D18E0C4CACA72DCDC
:100E3000BFD2412D8E233635203B83E784F33BC15F
:100E400000C0000084F3C53E203B7D188E23CACA33
:100E5000BFD2BFD2CACA8E237D18203BC53E84F3C1
:100E6000000000C03BC184F383E7203B36358E236E
:100E7000412DBFD272DCCACAE0C47D187C0CC53ECD
:100E8000004000007C0C3BC1E0C483E772DC3635D7
:100E9000412D412D363572DC83E7E0C43BC17C0C2B
:100EA000BC120308C0120308CC120308D4120308B2
:100EB000E0120308055085ABC5D8E5EEF5FAFD0054
:100EC00000000040000000C000000040000000C022
:100ED00000000040000000C000000040000000C012
:100EE00000000040000000C000000040000000C002
:100EF00000000040000000C000000040000000C0F2
:100F000000000040000000C000000040000000C0E1
:100F100000000040000000C000000040000000C0D1
:100F200000000040000000C000000040000000C0C1
:100F300000000040000000C000000040000000C0B1
:100F400000000040000000C000000040000000C0A1
:100F500000000040000000C000000040000000C091
:100F600000000040000000C000000040000000C081
:100F700000000040000000C000000040000000C071
:100F800000000040000000C000000040000000C061
:100F900000000040000000C000000040000000C051
:100FA00000000040000000C000000040000000C041
:100FB00000000040000000C000000040000000C031
:100FC00000000040000000C000000040000000C021
:100FD00000000040000000C000000040000000C011
:100FE00000000040000000C000000040000000C001
:100FF00000000040000000C000000040000000C0F1
:1010000000000040000000C000000040000000C0E0
:1010100000000040000000C000000040000000C0D0
:1010200000000040000000C000000040000000C0C0
:1010300000000040000000C000000040000000C0B0
:1010400000000040000000C000000040000000C0A0
:1010500000000040000000C000000040000000C090
:1010600000000040000000C000000040000000C080
:1010700000000040000000C000000040000000C070
:1010800000000040000000C000000040000000C060
:1010900000000040000000C000000040000000C050
:1010A00000000040000000C000000040000000C040
:1010B00000000040000000C000000040000000C030
:1010C00000000040000000C000000040000000C020
:1010D00000000040000000C000000040000000C010
:1010E00000000040000000C000000040000000C000
:1010F00000000040000000C000000040000000C0F0
:1011000000000040000000C000000040000000C0DF
:1011100000000040000000C000000040000000C0CF
:1011200000000040000000C000000040000000C0BF
:1011300000000040000000C000000040000000C0AF
:1011400000000040000000C000000040000000C09F
:1011500000000040000000C000000040000000C08F
:1011600000000040000000C000000040000000C07F
:1011700000000040000000C000000040000000C06F
:1011800000000040000000C000000040000000C05F
:1011900000000040000000C000000040000000C04F
:1011A00000000040000000C000000040000000C03F
:1011B00000000040000000C000000040000000C02F
:1011C00000000040000000C000000040000000C01F
:1011D00000000040000000C000000040000000C00F
:1011E00000000040000000C000000040000000C0FF
:1011F00000000040000000C000000040000000C0EF
:1012000000000040000000C000000040000000C0DE
:1012100000000040000000C000000040000000C0CE
:1012200000000040000000C000000040000000C0BE
:1012300000000040000000C000000040000000C0AE
:1012400000000040000000C000000040000000C09E
:1012500000000040000000C000000040000000C08E
:1012600000000040000000C000000040000000C07E
:1012700000000040000000C000000040000000C06E
:1012800000000040000000C000000040000000C05E
:1012900000000040000000C000000040000000C04E
:1012A00000000040000000C000000040000000C03E
:1012B00000000040000000C000000040000000C02E
:1012C00000005A2EEC3FCD29BBF98CCDB2C026DBF5
:1012D0007C0C1236143E8B1F6CEDD6C6BEC311E6D5
:1012E0007D18B63BDA391314D5E152C21BC9FBF1A4
:1012F0008E230E3F6733D50767D72DC095D06EFE7E
:10130000412DFB3FFA2A4BFB87CE7CC0E1D9F10A85
:101310003635713EE720EFEE8FC73BC3A3E40817D5
:10132000203B823A8F153AE3C2C251C874F03D2285
:10133000C53E53346409A1D84FC08ACFDDFC212CAF
:101340000040212CDDFC8ACF4FC0A1D86409533462
:10135000C53E3D2274F051C8C2C23AE38F15823AAD
:10136000203B0817A3E43BC38FC7EFEEE720713E95
:101370003635F10AE1D97CC087CE4BFBFA2AFB3F18
:10138000412D6EFE95D02DC067D7D50767330E3F30
:101390008E23FBF11BC952C2D5E11314DA39B63BD7
:1013A0007D1811E6BEC3D6C66CED8B1F143E1236F7
:1013B0007C0C26DBB2C08CCDBBF9CD29EC3F5A2E7C
:1013C0000000A6D114C033D6450674324E3FDA244D
:1013D00084F3EEC9ECC175E094122A39423CEF194E
:1013E00083E74AC426C6EDEB2B1EAE3DE536050E5F
:1013F00072DCF2C099CC2BF89928D33F6B2F920165
:10140000BFD205C006D5B5047931843F1F260FF53C
:10141000CACA8FC119DF11117138C53C5D1BF8E8CC
:10142000E0C47EC571EAC61C3E3DAF378C0FC3DDFC
:101430003BC1ADCB9CF65F27B13F76302303DFD3B2
:1014400000C0DFD323037630B13F5F279CF6ADCBDE
:101450003BC1C3DD8C0FAF373E3DC61C71EA7EC574
:10146000E0C4F8E85D1BC53C7138111119DF8FC16C
:10147000CACA0FF51F26843F7931B50406D505C0C9
:10148000BFD292016B2FD33F99282BF899CCF2C091
:1014900072DC050EE536AE3D2B1EEDEB26C64AC4CA
:1014A00083E7EF19423C2A39941275E0ECC1EEC98A
:1014B00084F3DA244E3F7432450633D614C0A6D1E5
:1014C00000005A2EEC3FCD29BBF98CCDB2C026DBF3
:1014D0007C0C1236143E8B1F6CEDD6C6BEC311E6D3
:1014E0007D18B63BDA391314D5E152C21BC9FBF1A2
:1014F0008E230E3F6733D50767D72DC095D06EFE7C
:10150000412DFB3FFA2A4BFB87CE7CC0E1D9F10A83
:101510003635713EE720EFEE8FC73BC3A3E40817D3
:10152000203B823A8F153AE3C2C251C874F03D2283
:10153000C53E53346409A1D84FC08ACFDDFC212CAD
:101540000040212CDDFC8ACF4FC0A1D86409533460
:10155000C53E3D2274F051C8C2C23AE38F15823AAB
:10156000203B0817A3E43BC38FC7EFEEE720713E93
:101570003635F10AE1D97CC087CE4BFBFA2AFB3F16
:10158000412D6EFE95D02DC067D7D50767330E3F2E
:101590008E23FBF11BC952C2D5E11314DA39B63BD5
:1015A0007D1811E6BEC3D6C66CED8B1F143E1236F5
:1015B0007C0C26DBB2C08CCDBBF9CD29EC3F5A2E7A
:1015C0000000A6D114C033D6450674324E3FDA244B
:1015D00084F3EEC9ECC175E094122A39423CEF194C
:1015E00083E74AC426C6EDEB2B1EAE3DE536050E5D
:1015F00072DCF2C099CC2BF89928D33F6B2F920163
:10160000BFD205C006D5B5047931843F1F260FF53A
:10161000CACA8FC119DF11117138C53C5D1BF8E8CA
:10162000E0C47EC571EAC61C3E3DAF378C0FC3DDFA
:101630003BC1ADCB9CF65F27B13F76302303DFD3B0
:1016400000C0DFD323037630B13F5F279CF6ADCBDC
:101650003BC1C3DD8C0FAF373E3DC61C71EA7EC572
:10166000E0C4F8E85D1BC53C7138111119DF8FC16A
:10167000CACA0FF51F26843F7931B50406D505C0C7
:10168000BFD292016B2FD33F99282BF899CCF2C08F
:1016900072DC050EE536AE3D2B1EEDEB26C64AC4C8
:1016A00083E7EF19423C2A39941275E0ECC1EEC988
:1016B00084F3DA244E3F7432450633D614C0A6D1E3
:1016C0000000C53C1F2626DBC2C26EFE423C5F27DF
:1016D00072DC52C2DDFCB63B9928C3DDECC14BFB8A
:1016E000203BCD2919DF8FC1BBF9823AFA2A75E078
:1016F0003BC12BF8DA39212CD5E1F2C09CF62A390E
:10170000412D3AE3B2C00FF571385A2EA3E47CC0E4
:1017100084F3AF376B2F11E64FC0FBF1E53676301F
:1017200083E72DC074F012367931F8E814C0EFEE7B
:101730003635743271EA05C06CED53346733EDEB26
:1017400000C0EDEB673353346CED05C071EA7432C1
:101750003635EFEE14C0F8E87931123674F02DC04A
:1017600083E77630E536FBF14FC011E66B2FAF37DC
:1017700084F37CC0A3E45A2E71380FF5B2C03AE36B
:10178000412D2A399CF6F2C0D5E1212CDA392BF80B
:101790003BC175E0FA2A823ABBF98FC119DFCD2926
:1017A000203B4BFBECC1C3DD9928B63BDDFC52C2AC
:1017B00072DC5F27423C6EFEC2C226DB1F26C53CA0
:1017C00000003BC3E1D9DA243E3D9201BEC3A1D85B
:1017D0008E23AE3D23034AC467D73D22143EB50491
:1017E000E0C433D6E720713E45067EC506D58B1F83
:1017F000C53ED50726C6DFD32B1E0E3F6409D6C6CD
:10180000BFD2C61C4E3FF10A8FC7A6D15D1B843FD5
:101810007C0C51C895D0EF19B13F050E1BC98ACF7A
:101820007D18D33F8C0FEEC987CE0817EC3F1111FE
:10183000CACA8CCD8F15FB3F9412ADCB99CC131433
:101840000040131499CCADCB9412FB3F8F158CCD77
:10185000CACA1111EC3F081787CEEEC98C0FD33FCF
:101860007D188ACF1BC9050EB13FEF1995D051C81D
:101870007C0C843F5D1BA6D18FC7F10A4E3FC61C6E
:10188000BFD2D6C664090E3F2B1EDFD326C6D507AE
:10189000C53E8B1F06D57EC54506713EE72033D673
:1018A000E0C4B504143E3D2267D74AC42303AE3DCD
:1018B0008E23A1D8BEC392013E3DDA24E1D93BC3B9
:1018C0000000C53C1F2626DBC2C26EFE423C5F27DD
:1018D00072DC52C2DDFCB63B9928C3DDECC14BFB88
:1018E000203BCD2919DF8FC1BBF9823AFA2A75E076
:1018F0003BC12BF8DA39212CD5E1F2C09CF62A390C
:10190000412D3AE3B2C00FF571385A2EA3E47CC0E2
:1019100084F3AF376B2F11E64FC0FBF1E53676301D
:1019200083E72DC074F012367931F8E814C0EFEE79
:101930003635743271EA05C06CED53346733EDEB24
:1019400000C0EDEB673353346CED05C071EA7432BF
:101950003635EFEE14C0F8E87931123674F02DC048
:1019600083E77630E536FBF14FC011E66B2FAF37DA
:1019700084F37CC0A3E45A2E71380FF5B2C03AE369
:10198000412D2A399CF6F2C0D5E1212CDA392BF809
:101990003BC175E0FA2A823ABBF98FC119DFCD2924
:1019A000203B4BFBECC1C3DD9928B63BDDFC52C2AA
:1019B00072DC5F27423C6EFEC2C226DB1F26C53C9E
:1019C00000003BC3E1D9DA243E3D9201BEC3A1D859
:1019D0008E23AE3D23034AC467D73D22143EB5048F
:1019E000E0C433D6E720713E45067EC506D58B1F81
:1019F000C53ED50726C6DFD32B1E0E3F6409D6C6CB
:101A0000BFD2C61C4E3FF10A8FC7A6D15D1B843FD3
:101A10007C0C51C895D0EF19B13F050E1BC98ACF78
:101A20007D18D33F8C0FEEC987CE0817EC3F1111FC
:101A3000CACA8CCD8F15FB3F9412ADCB99CC131431
:101A40000040131499CCADCB9412FB3F8F158CCD75
:101A5000CACA1111EC3F081787CEEEC98C0FD33FCD
:101A60007D188ACF1BC9050EB13FEF1995D051C81B
:101A70007C0C843F5D1BA6D18FC7F10A4E3FC61C6C
:101A8000BFD2D6C664090E3F2B1EDFD326C6D507AC
:101A9000C53E8B1F06D57EC54506713EE72033D671
:101AA000E0C4B504143E3D2267D74AC42303AE3DCB
:101AB0008E23A1D8BEC392013E3DDA24E1D93BC3B7
:101AC0000000DA39793174F03BC1E1D92B1EEC3FCB
:101AD0007D1806D5C2C29CF63635E536BBF9BEC3C5
:101AE000BFD28F15B13FE72072DCB2C06CED6B2F17
:101AF000203B23038FC799CC7C0C143E9928A3E488
:101B000000C0A3E49928143E7C0C99CC8FC7230312
:101B1000203B6B2F6CEDB2C072DCE720B13F8F151C
:101B2000BFD2BEC3BBF9E53636359CF6C2C206D578
:101B30007D18EC3F2B1EE1D93BC174F07931DA39C5
:101B4000000026C687CE8C0FC53E1F26D5E114C0E7
:101B500083E7FA2A3E3D6409CACA1BC94506423CCE
:101B6000412D71EA4FC019DF8E234E3F941295D05C
:101B7000E0C4DDFC7138673384F3ECC167D75D1BCB
:101B800000405D1B67D7ECC184F367337138DDFC1F
:101B9000E0C495D094124E3F8E2319DF4FC071EAF6
:101BA000412D423C45061BC9CACA64093E3DFA2A7A
:101BB00083E714C0D5E11F26C53E8C0F87CE26C60D
:101BC0000000DA39793174F03BC1E1D92B1EEC3FCA
:101BD0007D1806D5C2C29CF63635E536BBF9BEC3C4
:101BE000BFD28F15B13FE72072DCB2C06CED6B2F16
:101BF000203B23038FC799CC7C0C143E9928A3E487
:101C000000C0A3E49928143E7C0C99CC8FC7230311
:101C1000203B6B2F6CEDB2C072DCE720B13F8F151B
:101C2000BFD2BEC3BBF9E53636359CF6C2C206D577
:101C30007D18EC3F2B1EE1D93BC174F07931DA39C4
